:020000040000FA
:040000006FD00400B9
:101000006F10C000000000000000000090200020D1
:10101000AA220020A9BDF9F56C23002000000000E1
:10102000000000006C230020902000200000000041
:101030000000000090200020000000009020002010
:101040000000000090200020902000209020002030
:1010500090200020902000207C2F0020822400205F
:101060000000000090200020902000200C24002090
:1010700090200020D22300209020002090200020EB
:101080009020002090200020902000209020002020
:101090009020002001A04111B7170040985F3AC688
:1010A000945F3247E39CE6FE3245410182800111A4
:1010B00013078008F337078093F787083EC20100C3
:1010C0000100B7170040930570052380B70413068D
:1010D00080FA2380C7040100010083C6B70493F699
:1010E000F60DA385D704238007049246F3A6068055
:1010F0000100010093760502D5CEF336078093F602
:10110000860836C4010001002380B7042380C70489
:1011100001000100B70614007D89558D88C70100C4
:1011200001000100010023800704A246F3A6068007
:101130000100010073370780137787083AC6010062
:1011400001002380B7042380C704010001000100CF
:1011500001003727004093061005A303D7802380A2
:101160000704B247F3A70780010001009307800836
:10117000F3B7078093F787083ECE01000100B71749
:101180000040130770052380E704130780FA2380CB
:10119000E7040100010003C7B70413670708A3852C
:1011A000E70423800704F247F3A70780010001004A
:1011B0000561828093760504BDC6F336078093F6F9
:1011C000860836C8010001002380B7042380C704C5
:1011D00001000100B7061400938606047D89558D31
:1011E00088C7010001000100010023800704C246F6
:1011F000F3A6068001000100733707801377870884
:101200003ACA010001002380B7042380C70401000B
:1012100001003727004093062005A303D7802380D1
:101220000704D24781B773370780137787083ACC12
:10123000010001002380B7042380C70401000100DE
:1012400098471367070C98C723800704E24719BF24
:101250000111814601468145114506CE97000000E7
:10126000E780A05A93078008F3B7078093F78708B1
:101270003EC601000100B717004013077005238028
:10128000E704130780FA2380E7040100010003C785
:101290006704136717002383E70423800704B2471A
:1012A000F3A7078001000100F2400561828041112F
:1012B000814601468145114597000000E780E054D2
:1012C00013078008F337078093F787083EC40100AF
:1012D0000100B7170040130670052380C70493066A
:1012E00080FA2380D70401000100FD552396B70240
:1012F00023800704A245F3A5058001000100733790
:101300000780137787083AC6010001002380C704CD
:101310002380D7040100010003C767041367170087
:101320002383E70423800704B247F3A70780010063
:10133000010001A0B1473305F50201007D1575FDDF
:101340008280411122C426C206C6AA8401446317C2
:101350009400B24022449244410182800504130566
:10136000803E420497000000E78000FD4180C5B741
:101370009305000273A04580824573901534924016
:101380002242B2424243D2436244F2440255925551
:101390002256B2564257D2576258F25806499649D9
:1013A000264AB64A464BD64B664CF64C065D965DD1
:1013B000265EB65E465FD65F09617300203041113C
:1013C000B7170040985F3AC6945F3247E39CE6FE49
:1013D000324541018280B71700401307000323887C
:1013E000E7028547171700002322F76073002030BB
:1013F000411122C406C637040020976000E0E78050
:101400002075975000E0E78040A11C408297F5B717
:1014100037370040834747009146BD8B639ED70214
:10142000B73600401306F00F973500009385053955
:101430009737000083D7874803C7A6001377F70FB5
:101440001DE3B7E70400BC4F0946894517150000A6
:10145000034585FA829731A099466394D700834764
:1014600057007300203003C786001377F70FE3653A
:10147000F6FC13851700AE97173800002310A84418
:101480002380E70075B7B787004003C76700058B67
:1014900015C729472381E70209472383E7022385EC
:1014A000E7022387E7022389E702A38107001747A2
:1014B0000000A303078605472383E700B7870040A2
:1014C00003C76700098B6309071003C777009306FA
:1014D000000313770703630DD7081748000003487C
:1014E0003895174600001306E6930547B306060134
:1014F0002380E60083C57700174700001307079392
:10150000429793F5F50F2300B70003C58700974571
:10151000000093856591C2951375F50F2380A50092
:101520000347070089451377F703630CB70C63E79C
:10153000E50A6306071A8545630CB7129747000052
:1015400083C7178F3307F600034707001377F70F9A
:1015500019CB850793F7F70F0D476363F71A174702
:101560000000A307F78CB787004009472383E700F3
:10157000B787004083C77700E207E18763DE07048F
:101580009747000083C7D78A17470000130787894A
:101590003E9785462300D7001747000013070789A9
:1015A0003E97930600032300D70017470000130758
:1015B000A7873E97A14685072300D70093F7F70F2B
:1015C0000D476364F71417470000A303F786B78736
:1015D000004009472383E700730020309306100280
:1015E0006300D70E930620026305D7069306000218
:1015F000E316D7F403C727021377C70F1367270033
:10160000D5A803C767001377070465CB03C7A702F4
:101610001738000013088862173500001305C559F4
:10162000134707082385E70203C7A7021377370F7D
:10163000136787002385E702814713070004B3057A
:10164000F5008C41B306F80091078CC2E399E7FEE0
:10165000F5B503C7A702134707042385E70203C7AD
:10166000A7021377C70F136727002385E702F9B591
:1016700003C767001377070449C303C76702173816
:1016800000001308684F173500001305A5461347DF
:1016900007082383E70203C767021377370F13672F
:1016A00087002383E702814713070004B305F50091
:1016B0008C41B306F80091078CC2E399E7FEBDBDEB
:1016C00003C76702134707042383E70203C76702C0
:1016D0001377C70F136727002383E70285B503C776
:1016E00067001377070411CB03C727021377370F5F
:1016F000136787002381E70291B5238006003DBD73
:1017000097370000A3860772B9BD97370000A38101
:10171000077275BD2303048015472303E48001008D
:101720002302A480828083076480E3CE07FE230324
:101730000480828083076480E3CE07FE03454480F3
:10174000828083076480E3CE07FE2302A480828028
:10175000411126C44AC24EC006C61377F50BAD47E9
:10176000AA892E899544630CF7001945970000005B
:10177000E78080FA97000000E78020FB8D444E85CB
:1017800097000000E78040F9FD59FD14639834018B
:10179000B240A24412498249410182801355090195
:1017A0001375F50F97000000E780E0F92209F1BFFB
:1017B000011126CC06CEB704080097000000E78090
:1017C000C0F6154597000000E78000F5970000007F
:1017D000E78080F697000000E78000F62AC69700B1
:1017E0000000E78080F432459377150089EB13659C
:1017F00015001375F50FF240E24405618280FD1477
:10180000E9F00145CDBF397126DC4ADA4ED852D60F
:1018100056D45AD25ED006DE62CE66CCB7E700E080
:101820007D5783AA070022C603AA470023A0E71812
:1018300023A2E718B7170040130770052380E704B9
:10184000130780FA2380E70483C74704930B75FFCF
:10185000B684E20793FBFB0F8546AA892E8B32895B
:1018600037240040E187015763FA76016308D50009
:101870008946130700026313D5000157D98F93F7E8
:10188000F70FB71C00402382FC0411472303E480B8
:101890001305F00F97000000E78000E8094C97005F
:1018A0000000E78080E863657C15B7050700DA95DE
:1018B00037870700795563FEE504B3879500636AAF
:1018C000F704370B0800A94733EB65016395F90866
:1018D00081E8814497000000E78020E5268515A86F
:1018E000DA85094597000000E780C0E60509034551
:1018F000F9FFFD14050B97000000E780C0E481C4E8
:101900009377FB0FE5F797000000E780A0EA69F105
:101910007D55B7170040130770052380E7041307B0
:1019200080FA2380E70403C74704418B2382E7043E
:10193000F250B7E700E023A0571123A24711E25469
:1019400032445259C259325AA25A125B825B724CCB
:10195000E24C21618280A547639BF90685691309E2
:10196000F00FB3069900B3742B01B6941349F9FF35
:10197000B3749900856B33796901416B9387F9FFE3
:10198000B3F7270199E363FC340193D94900C147B8
:10199000E3E637FF3DBF0569C1697D19D9B7130576
:1019A000800D6388690113050002638479011305C2
:1019B0001008CA8597000000E780C0D99700000092
:1019C000E78040DF31D54E99B38434416DBFDA856D
:1019D0002D4597000000E780E0D7CA94E30B99EE0D
:1019E000050997000000E78020D5A30FA9FEFDB7E9
:1019F0009387F9FF93F7F70F636DFC0C83C71C0403
:101A0000130730086315F706370708006361EB0614
:101A1000B3079B00B706100063FBD704334BEB0002
:101A200089476399F9068980D549E38404EADA8510
:101A3000094597000000E780E0D111090327C9FF9D
:101A400091472320E48003076480E34E07FE2303CD
:101A50003481FD17EDFBFD14110B81C49377FB0F4F
:101A6000E9FF97000000E780E0D461F155B5B717B2
:101A7000004003C75704B70708001377070219E3AC
:101A8000B78707007955E376FBE833079B00E3F956
:101A9000E7F841B58547E380F9F0DA852D459700F1
:101AA0000000E78020CB9389F4FFE38404E29700F1
:101AB0000000E78060C893F7390091EB832604802B
:101AC0000327090093074900E396E6E03E89CE84A8
:101AD000D9BFB5476399F9001305900B9700000033
:101AE000E78080C3FDB3B1471305B00AE388F9FE70
:101AF00099476397F904B7050800B365BB002D4506
:101B000097000000E78000C581448D4BA1499700F4
:101B10000000E78060C2639674018327048023205D
:101B2000F9008504E39534FF8327048013172B0104
:101B3000635507002312F90069BB2322F90051BB4A
:101B40009D47639FF90281451305B004970000008B
:101B5000E78040C0BD442320090023220900FD592D
:101B600097000000E78040BD93F77400CA9703C751
:101B70000700FD14398D2380A700E39334FF91BB48
:101B8000A1476397F90697000000E780A0C281444F
:101B9000630D0B008D479304C0036308FB0093049F
:101BA000000563048B01930440041375C507E30229
:101BB00095D2194597000000E78000B69700000015
:101BC000E780A0B6054597000000E780E0B42685D1
:101BD00097000000E78020B7094597000000E780E4
:101BE00080B697000000E780E0BCE31405CE0DB39B
:101BF0009147639FF9001305600697000000E78096
:101C0000A0B197000000E78040B213059009F9B534
:101C1000E38109CCF1547DB9BD6601471736000058
:101C20001306863E938606A685458347060093F7EE
:101C3000F70F91C382800507E3F9E6FE97370000AE
:101C40002384B73CDDB77D16620661869317860153
:101C5000E18763D40700014582809317260033078C
:101C6000F500AE9718439C4363E7E7007D16E37FDA
:101C7000F7FC7D55828005458280FD15E205E185F2
:101C800013978501618793F7F50F63480700FD15EA
:101C9000139725002A97584365D7138517006205C7
:101CA000618582803308B5021C4283A80600B335E3
:101CB000B502C29733B50701AE984695854863676C
:101CC000B5006394A50063E3070181480C43C69502
:101CD0000CC388C21CC28280814713978701618729
:101CE0006343B7008280139727002A9723200700B9
:101CF0008507E5B78147014793968701E18663C56C
:101D0000B60013351700828093962700AA96944256
:101D10008507558FD5B793D755408A07AA979C4317
:101D200005453315B5007D8D828017F3FFDFE7028F
:101D3000833D2A8497000000E78060F405C593176F
:101D400025003E940327C4FF814711EB7D1516053E
:101D50003E954205418517F3FFDF6700033D05838C
:101D60008507E5B70145C5BF81471397870161879F
:101D70006343C700828013972700B386E50094422F
:101D80002A97850714C3D5B77D1662066186014779
:101D900093178601E18763D507001335170082800A
:101DA00093172600B306F500AE9794429C437D1628
:101DB000B58F5D8FF1BF8A05AA9501476363B500B2
:101DC000828083A6C5FFF11593D71600D98F9CC1D9
:101DD0001397F601E5B72A8301480147014563439C
:101DE000D7008280B387050183A80700B3070601E7
:101DF0009C43C697AA976384F80033B5170105077B
:101E0000B3080301620723A0F80061871108C1BF6E
:101E10002A8301478147014563C3D7008280338805
:101E2000E50083280800330EE600032E0E003388F9
:101E3000A8403308C8416384080133B50801850709
:101E4000B308E300E20723A00801E1871107E9B71F
:101E500017F3FFDFE702232B0111B286B2842E862F
:101E6000AA850A8597000000E780C0FA2A84A68523
:101E70000A8597000000E78020E8333480000604DC
:101E800013351500018D056117F3FFDF6700E329A6
:101E900017F3FFDFE702A3244111AA89AE8A328B30
:101EA000B68402C202C402C60144131C8401135C3E
:101EB0008C4163499C02939B1400FD1B0549138CC4
:101EC000F4FFF15C330489016204618463407407A8
:101ED00092478E04CE9423AEF4FE410117F3FFDF48
:101EE0006700632313192400B30B2B01014A9317D6
:101EF0002A00D69783A50B00884378003400500051
:101F000097000000E78040DA050A93178A01E1870D
:101F1000F11BE35EFCFC92474E9905042320F90077
:101F2000A2473EC2B24702C63EC441B7131A890156
:101F3000135A8A41131D240093178A01E18763CF46
:101F4000970092470A044E941CC0A24705091379D2
:101F5000F90F3EC2B24702C63EC4ADB7B3079A03FB
:101F600013152A0056950841780034005000050AE0
:101F7000EA97DA978C4397000000E780E0D26DBFC4
:101F8000197106C212C416C61AC81ECA22CC26CEA1
:101F90002AD02ED232D436D63AD83EDA42DC46DEC9
:101FA000CAC0CEC2D2C4D6C6DAC8DECAE2CCE6CE39
:101FB000EAD0EED2F2D4F6D6FAD8FEDA97150000BF
:101FC000938545A28841E700050092402242B24233
:101FD0004243D2436244F244025592552256B256CD
:101FE0004257D2576258F25806499649264AB64A8D
:101FF000464BD64B664CF64C065D965D265EB65E4D
:10200000465FD65F096173002030000097210020F1
:10201000938141FF174100201301C17E17F5FFFF97
:10202000130585FE970500209385C5FD1716002032
:102030001306C6FD63FAC5008322050023A05500E0
:1020400011059105E3EAC5FE17150200130585D0B9
:1020500097150020938585FB171600201306067C34
:1020600063FAC5008322050023A0550011059105E0
:10207000E3EAC5FE171500201305457A97450020B1
:10208000938545446377B500232005001105E36D72
:10209000B5FEFD42739002BC8D4273904280B72220
:1020A000000093828288739002309702002093820E
:1020B00062F593E23200739052309752000093829F
:1020C0006292739012346FB0B47373002030397120
:1020D00001436EC619A0397141536AC866CA62CC01
:1020E0005ECE19A0397101535AD056D252D44ED671
:1020F0004AD826DA22DC06DE3301614082824111B1
:102100004AC026C222C406C68282B24D4101024D97
:10211000924C224CB24B4101024B924A224AB249A4
:102120004101024992442244B240410182803D4330
:102130002A876373C3029377F700BDEFADE593760B
:1021400006FF3D8ABA960CC34CC30CC74CC7410767
:10215000E36BD7FE11E28280B306C3408A06970282
:10216000000096966780A6002307B700A306B70075
:102170002306B700A305B7002305B700A304B700E3
:102180002304B700A303B7002303B700A302B700DB
:102190002302B700A301B7002301B700A300B700D3
:1021A0002300B700828093F5F50F93968500D58DB7
:1021B00093960501D58D61B793962700970200008D
:1021C00096968682E78086FA9680C1171D8F3E9686
:1021D000E374C3F8A5B73367B500FD530D8B79E7FA
:1021E000B7877F7F9387F7F710419441B372F6006A
:1021F0003363F600BE92B3E262006397720C631819
:10220000D6065041D441B372F6003363F600BE9255
:10221000B3E262006398720A631BD60410459445CA
:10222000B372F6003363F600BE92B3E262006391CC
:10223000720A631ED6025045D445B372F60033636A
:10224000F600BE92B3E26200639A72086311D6028E
:1022500010499449B372F6003363F600BE92B3E2BC
:102260006200639372085105D105E30FD6F6131788
:10227000060193970601631CF7001357060193D7D5
:1022800006013305F7409375F50F91E9828041838C
:10229000C1833305F7409375F50F91E18280137781
:1022A000F70F93F7F70F3305F740828003460500D9
:1022B00083C60500050585056313D60065FA330559
:1022C000D640828011059105E312D6FE0145828039
:1022D0002105A105E31CD6FC014582803105B1052D
:1022E000E316D6FC014582804105C105E310D6FC0A
:1022F00001458280B717004003C777051377E70FC2
:10230000A38BE704130700F8A38DE7043D47238C54
:10231000E70413075003A38CE70403C7A70513774B
:10232000D70F238DE7048280B717004003C7E70269
:102330000D8941111377C70F498F93068008F3B6B3
:10234000068093F6860836C60100010093067005E4
:102350002380D704930680FA2380D704010001006C
:102360002387E70223800704B247F3A70780010011
:1023700001004101828041112A83014E930E407E6B
:10238000130F0019930F400663E56E1293080019AE
:1023900013034006B3781503854E0D4FA14F3373D9
:1023A00065020D891335150063EFBE121308F6FFA1
:1023B000794672984208135808013307C70213D6AA
:1023C0001700BE0732976146B3F6C6021306807047
:1023D000B386C6023697A166F58F42075D8FB716A2
:1023E000004083C7F60293F70708A303F1000346F2
:1023F000710083C7F60293F70708E394C7FE83478B
:102400007100B716004093F7F70F63880712930720
:102410008008F3B7078093F787083EC401000100E6
:10242000B7170040930670052380D704930680FAFF
:102430002380D7040100010023AA070383C61703E2
:1024400093E60608A388D70223800704A247F3A7D0
:102450000780010001001166B71700407D16D45BAC
:10246000C85F93854703A98EF18EF5FA930680081D
:10247000F3B6068093F6860836C60100010093067F
:1024800070052380D704930680FA2380D7040100C7
:10249000010098C103C7170313670704A388E70265
:1024A00023800704B247F3A7078001000100410120
:1024B00082807D133368E3039308E016630E0800FF
:1024C0003368F3039308D016630808009378330049
:1024D00093B818009388D81633081E01131E0801FC
:1024E000135E0E0155B56393E50305486386080046
:1024F0000148630303002A8871087298FD15131EB2
:102500000801C205135E0E01C18179BD13F81500E3
:1025100063F4BF007908D5B713381800E5BF83C747
:10252000F60293F70708A303F1000346710083C77F
:10253000F60293F70708E394C7FE8347710093F709
:10254000F70FF1DFE9B531714AD966CB06DF22DD3D
:1025500026DB4ED752D556D35AD15ECF62CD6AC94B
:102560006EC7AA8C02D897100000E78020B12A8994
:1025700093078008F3B7078093F787083EDA0100D6
:102580000100B7170040130770052380E704130705
:1025900080FA2380E7040100010003C7F7021377E4
:1025A000770FA387E70203C7F70213678700A387A4
:1025B000E70223800704D257F3A707800100010038
:1025C000054597000000E78060D6130780C13347B8
:1025D000E902116A93070AE893065002BD69930B5A
:1025E000A004814A014B13048008930470057D1AEE
:1025F000B347F9023307D7023EC0FD873ECC93872D
:1026000009A69309803E3347F7023AC27D873AC450
:10261000334739038549B399990193D93940B306B2
:10262000D702B30B7703B3C6F602B3CBFB0236C6B1
:10263000FD8636C893D6FB4136CEB7460F0093864B
:1026400006243349D9028566938606FAB396960125
:10265000B389E902130760553309D90293060010C4
:10266000B389E9023349D902B3C9F9029316390093
:1026700036CA37190040FD8636D0930D090493D72A
:10268000F9413ED2F336048093F6860836DC010029
:102690000100930770052380FD00930680FA2380D4
:1026A000DD00010001008346390593F6860FA3097A
:1026B000D9048346390593E61600A309D90423807B
:1026C0000D00E256F3A6068001000100130C80FA0B
:1026D000116DF336048093F6860836DE01000100A2
:1026E000930770052380FD0023808D010100010008
:1026F00083463905216693E60602A309D904835669
:102700000905B3E6A6012318D90483560905D18E1D
:102710002318D90423800D00F256F3A60680010089
:1027200001008346390593F606026381061A0346C3
:102730003905218A6DDE081897100000E78000989F
:102740007336048013768608B2C20100010023802C
:102750009D0023808D0101000100B717004003C6D2
:1027600037051376F60DA389C70403C6370513662C
:102770000602A389C704835609052166B3E6A601AC
:102780002318D90483560905D18E2318D904238030
:102790000D009646F3A60680010001008346390528
:1027A00093F60602638B061483463905A18AEDFE73
:1027B00097000020E780208EAA8636D4970000205C
:1027C000E780608DA256E30AD5FE8356090542557F
:1027D000B3E6A6012318D90497100000E780C08F44
:1027E00083463905A18AEDDE03560905834629058E
:1027F00082473376CA00B306DA0293D5F641B29621
:10280000B388F640E24733B8C6002E983308F84044
:10281000A247B3B616013308D84063C70701631D4A
:10282000F800924763FA1701C247634FF80E6395A9
:102830000701B24763EAF80E894663E9660FF2467C
:102840009315180013D3F8015E8613951800B3652D
:10285000B30042D646D497C00100E78080153258B5
:10286000050B137BFB0F63470001631A0838A2585E
:102870006387083813081500B336A800B69513D639
:10288000F5013298B336C800AE9613581800FE060C
:10289000B3E606017336048013768608B2C60100DB
:1028A000010023809D0023808D010100010003565B
:1028B000C902B296C206C1822316D90223800D0036
:1028C000B646F3A606800100010021B5F336048068
:1028D00093F68608B6C00100010023809D00238086
:1028E0008D01010001008346390593E60602A30924
:1028F000D90423800D0086460DB5F336048093F687
:102900008608B6C40100010023809D0023808D014C
:10291000010001008346390593E60602A309D904A4
:1029200023800D00A646BDB5E30B0BF0F336048003
:1029300093F68608B6C801000100930680FA23804A
:102940009D002380DD00010001008346390593F5D9
:10295000FC0F93F6860FA309D90483463905CD8E63
:10296000A309D90423800D00C646F3A60680010002
:102970000100130580FA03463905930639051D8ABF
:10298000631C96297336048013768608B2CC010046
:102990000100130680FA23809D002380CD000100F2
:1029A000010003C606001376F60D2380C60003C699
:1029B0000600136606022380C600835609051166C9
:1029C000D18E2318D904835609052166D18E231888
:1029D000D90423800D00E646F3A60680010001001D
:1029E000130680FA8346390593F6060263800626AD
:1029F00083463905130C3905A18AFDDA08189700BA
:102A00000000E780A06BF336048093F68608B6D00A
:102A100001000100930680FA23809D002380DD00E1
:102A20000100010083460C00116693F6F60D2300A9
:102A3000DC0083460C0093E606022300DC0083568C
:102A40000905D18E2318D904835609052166D18E34
:102A50002318D90423800D008656F3A606800100B2
:102A60000100130680FA8346390593F60602638A4D
:102A7000062083463905A18AEDFE97F0FF1FE78007
:102A800080612A8C97F0FF1FE780E060E30C85FFF0
:102A90008356090511664255D18E2318D904970033
:102AA0000000E78060638346390513063905A18A73
:102AB000FDDAF336048093F68608B6D401000100EF
:102AC000930680FA23809D002380DD000100010031
:102AD0008346060093F6F60D2300D60023800D00F2
:102AE000A656F3A606800100010083560905034699
:102AF0002905D247B376DA003306CA021305800CE3
:102B00009355F6413696330DF6408257333CD60046
:102B10002E9C3336A601330CFC40330CCC403308DA
:102B2000850392564E86B335A5033305A503C2959A
:102B300097C00100E780E0E763468001631E0C1642
:102B4000630C0D16130615003335A6002E9593560B
:102B5000F5013696B335D600AA959396F501058210
:102B60008585D18E6346B000639D051A638B061A76
:102B70000356C90215823305D6003336C500B29517
:102B80006348B000639105241306F00F637DA6220D
:102B9000894663F3561593078008F3B7078093F7C8
:102BA0008708BED601000100371700409307700563
:102BB0002300F704930780FA2300F70401000100C3
:102BC0008356C70289678117D58FC207C183231631
:102BD000F70223000704B657F3A70780010001009E
:102BE000FA506A54DA544A59BA592A5A9A5A0A5B1C
:102BF000FA4B6A4CDA4C4A4DBA4D2961828013086F
:102C0000F5FF3335A800FD152E951356F5013298C2
:102C1000B336C800AA9695B9F336048093F68608B1
:102C2000B6CA0100010023809D002380AD00010091
:102C3000010083463905CD8EA309D90423800D00F8
:102C4000D646F3A606800100010035B3F3360480B2
:102C500093F68608B6CE0100010023809D002380F4
:102C6000CD00010001008346390593E60602A30961
:102C7000D90423800D00F646F3A60680010001006A
:102C800095B3F336048093F68608B6D201000100AE
:102C900023809D002380CD0001000100834639057B
:102CA00093E60602A309D90423800D009656F3A6E5
:102CB00006800100010045BB9306F5FF33B5A60071
:102CC000FD152E959355F501AE96B3B5B600AA95B0
:102CD0001396F501858269B5F336048093F686086C
:102CE000B6D801000100930680FA23809D0023805E
:102CF000DD00010001008356C9020566011693F646
:102D0000F60FD18EC206C1822316D90223800D0090
:102D1000C656F3A6068001000100850A93FAFA0F51
:102D200095B233E6B60045C20356C9023305D0401A
:102D30003338A000B305B040B38505411582634523
:102D4000B000D1E16371A608894663F05605930788
:102D50008008F3B7078093F78708BEDA0100010007
:102D6000B7170040130770052380E704130780FAA4
:102D70002380E7040100010003D7C7027D8B23965F
:102D8000E70223800704D65781BDF336048093F60B
:102D90008608B6DC01000100930680FA23809D00BE
:102DA0002380DD00010001008356C902056601167B
:102DB00093F6F60FD18EC206C1822316D902238064
:102DC0000D00E656B9B793078008F3B7078093F76D
:102DD0008708BEDE01000100371700409307700529
:102DE0002300F704930780FA2300F7040100010091
:102DF0000356C70293975600B297C207C1832316A2
:102E0000F70223000704F657C1BB914763EEB702F0
:102E100017E70100130747C98A05BA959C41BA977D
:102E20008287B717004003A7470B1345F5FF698F4B
:102E300023AAE70A03A7070B698F23A8E70A03A7BA
:102E4000070A798D23A0A70A8280B717004083A6BE
:102E5000470B1347F5FFF98E23AAD70A83A6070B62
:102E6000558D23A8A70A83A6070A758F23A0E70A12
:102E70008280B717004003A7470B498F23AAE70AB0
:102E800003A7070B1345F5FF45BFB717004083A6FF
:102E9000470B1347F5FF758F23AAE70A03A7070A15
:102EA000598D4DB7B717004003A7470B498FEDB7B2
:102EB000914763EEB70217E70100130727C08A05A1
:102EC000BA959C41BA978287B717004003A7470D70
:102ED0001345F5FF698F23AAE70C03A7070D698F38
:102EE00023A8E70C03A7070C798D23A0A70C8280E9
:102EF000B717004083A6470D1347F5FFF98E23AAA5
:102F0000D70C83A6070D558D23A8A70C83A6070C05
:102F1000758F23A0E70C8280B717004003A7470DE9
:102F2000498F23AAE70C03A7070D1345F5FF45BFFB
:102F3000B717004083A6470D1347F5FF758F23AAE7
:102F4000E70C03A7070C598D4DB7B717004003A72F
:102F5000470D498FEDB7797122D43714004026D23E
:102F60004AD0035924028354040206D64209C204FB
:102F70004ECE52CC56CA13590901C1802DE11379A6
:102F8000F9F793F4F49F4209C20413590901C1806F
:102F900093078008F3B7078093F787083EC40100C2
:102FA0000100930770052300F404930780FA2300BF
:102FB000F4040100010023112403231094022300D0
:102FC0000404A247F3A7078001000100B250225475
:102FD00092540259F249624AD24A45618280B7F559
:102FE000070081463000B105194597000020E780B1
:102FF0008081A24713972701E34A07FC1369090858
:1030000093E4044093098008F3B7098093F7870895
:103010003EC001000100930A700523005405130A05
:1030200080FA23004405010001002311240323102A
:103030009402230004048247F3A7078001000100E3
:10304000294597F0FF1FE780E02EF3B9098093F937
:1030500089084EC2010001002300540523004405E5
:10306000010001008357040293E707202310F402B4
:10307000230004049247B9B7B717004088474205B8
:1030800041819377050491EB9377F5013755E8017A
:10309000130505803345F50282809377050C1307ED
:1030A00000046397E7009377F50137459C1CCDB783
:1030B0002165130505D0828037E700E01C435443A7
:1030C000A183E206D58F1CC1FD572320F7182322C8
:1030D000F718828013178500B7E700E023A0E710F8
:1030E000618123A2A7108280B7F700E08847CC4710
:1030F0008280814737370040A14663C4C7003285CC
:1031000082800345B740E38EA6FE3385F500034574
:10311000050085072304A740CDB7970700209387B4
:10312000E7EE9C43173700201307C7393E95636EBF
:10313000E500173700201307E74C6368A70017075F
:1031400000202325A7EC3E858280FD57EDBF8280BD
:10315000411122C406C62A8497000000E78000F2CD
:103160002947B307E502B2408D83B3D787022244D3
:103170009507B3D7E70237370040C207C18323164C
:10318000F70041018280411137150E0006C69700F5
:103190000000E78020FCB7370040130770F8238158
:1031A000E7000D47A381E70013070004A380E700B1
:1031B00005472387E700B24041018280373700404E
:1031C000834727001A0593F7F703C98F93F7F70F83
:1031D0002301F7008280B737004003C7170019C9E1
:1031E000D98DA380B70003C707001367870023802A
:1031F000E700828093C5F5FFF98DA380B700828038
:10320000AE872A87B736004021463738004089E725
:10321000170300006700E3F383C8B600E30916FF55
:1032200005078348F7FFFD17C20723041801C18370
:10323000F9BF411122C406C62A8497000000E78026
:10324000E0E32947B307E502B2408D83B3D7870295
:1032500022449507B3D7E70237370040C207C1833E
:103260002316F74041018280716541111305052045
:1032700006C697000000E78000FCB7370040130740
:1032800070F82381E7400D47A381E740130700044E
:10329000A380E74005472387E740B2404101828091
:1032A000CC41411106C6328503C6150083C5050011
:1032B00022064D8E42068D654186138875A2630CE9
:1032C0000611634BC804138845A26300060D634AC8
:1032D000C800938535A26301B608239006002946ED
:1032E0004DA0138855A26305060D938565A2E316CC
:1032F000B6FE8D451D4663E6E5081146198E63F35B
:10330000C7003E86B7E704002390C600FC4797D568
:1033100001009385E57C9DA0138895A263030611A7
:10332000634E060D1388A5A263000613938505A5B9
:10333000E315B6FA99451D4663E5E504198E63F376
:10334000C7003E86B7E704002390C600FC479705F8
:1033500000209385E5D51DA09D451D4663E3E5024C
:103360002146198E63F3C7003E86B7E70400FC4789
:103370002390C600970500209385C54ABA95829789
:103380000146B240328541018280AD451D46E3EAE7
:10339000E5FE3146198E63F3C7003E86B7E70400A9
:1033A0002390C600FC4797D501009385E575F9B7D2
:1033B000B1451D46E3E7E5FC3546198E63F3C700CA
:1033C0003E86B7E704002390C600FC4797D501006E
:1033D0009385857465B78D451D46E3E4E5FA11468E
:1033E000198E63F3C7003E86B7E704002390C6003A
:1033F000FC4797D501009385656F49B78D451D46FC
:10340000E3E1E5F81146198E63F3C7003E86B7E79E
:1034100004002390C600FC4797D501009385857171
:10342000B1BFA5451D46E3EEE5F42946198E63F3C9
:10343000C7003E86B7E704002390C600FC4797D537
:1034400001009385656B1DBFB5451D46E3EBE5F2B5
:103450003946198E63F3C7003E86B7E70400239010
:10346000C600FC4797D501009385856601BFB7E785
:10347000040003A3071397060020938666C2414603
:10348000A545170500201305A5B802832D455DE766
:1034900003C505000947631FE50803A8450041115E
:1034A00006C6034718003285034608002207416814
:1034B000518F930828FE6307170563E9E800051894
:1034C0006303070323900600294591A8130648FECD
:1034D000630AC7041518E31707FF15463E87637B89
:1034E000F600154701A8130600023E876374F60034
:1034F00013070002B7E704002390E600FC47131609
:10350000070111A83E8691C30546B7E70400FC47B2
:103510002390C6004206CC45418282970145B240C5
:1035200041018280130600083E87E375F6FC13070D
:103530000008C9B723900600054582808280416754
:1035400079176304E504411122C406C685472A841D
:10355000639FF500B7E7040022852244B24003A32D
:1035600087139705002093852546410102838947EB
:103570006399F500B7E7040083A7070B8545829799
:1035800071D9B2402244410182808280797126D271
:1035900052CCAE842A8A97D501009385A55B17D5B6
:1035A00001001305A55D06D63AC622D44AD036845A
:1035B00032894ECE97C00100E780E08AA28517D5F8
:1035C00001001305A55C97C00100E780C08929456B
:1035D00097C00100E780008E83C7840093F707023D
:1035E000F9E383C904008947054532476396F90822
:1035F000D44083C7160083C60600A207D58FC166D4
:10360000138616FE638CC7028D16638FD7068D66F0
:103610009386269029456391D706B7E70400A286D2
:10362000225403A34714B250F2494A86A685025990
:1036300092545285624A8547456102832D450DEFBC
:1036400093070002354563E98702B7E70400FC47AA
:10365000C84413060002CA85829781499707002053
:10366000938747379C43014581CB9C4391C74E8547
:103670002286CA8582970145B2502254925402593B
:10368000F249624A456182802D457DF79307700FAC
:103690003545E3E387FEB7E70400FC47C8442286CC
:1036A000CA85829765BF2145C1BF411122C437E455
:1036B00004008327841326C2AA84416506C69705A1
:1036C0000020938565307D1582978327C40A1705EE
:1036D0000000130505E78588829795C0032304132E
:1036E0002244B2409244970600209386E6AD4146BC
:1036F000C545170500201305259C41010283B240F2
:103700002244924401454101828019C59707002057
:1037100023A2A72C01458280454582801147636A18
:10372000A70A97D601009386A6410A053695184147
:10373000411106C63697AE87B2850287130700028D
:103740006145639DE700B7E70400FC4713060002EC
:10375000170500201305850D82970145B2404101F0
:10376000828005476145E39BE7FEB7E70400FC471D
:103770000546170500201305650DF9BF1307700FE7
:103780006145E39DE7FCB7E70400FC471306700FB3
:10379000170500201305C50BC1B7130700086145C5
:1037A000E39EE7FAB7E70400FC4713060008170595
:1037B0000020130565194DB715476145E390E7FAF9
:1037C000B7E70400FC471546170500201305052040
:1037D00061B709458280411126C2B7E4040083A77E
:1037E000C41322C44AC006C62E84970500209385C0
:1037F000A51D2A898297058905C59707002093870B
:10380000A78B83D7A70BA28503A3440D2310F40035
:103810002244B24092444A85024901464101028352
:10382000B2402244924402494945410182809707AF
:1038300000202383071A9707002023A1071AB71730
:10384000004003A7070CB706C0FFFD16758F23A025
:10385000E70C03A7070DB7064000558F23A8E70C18
:1038600003A7070C3D9B23A0E70C03A7070D1367D5
:10387000070123A8E70C8280B717004003A5470C77
:1038800083A7470C598113451500C18B058999E31E
:10389000136525009707002083C707146380A702DC
:1038A00097070020238AA71211C997070020938742
:1038B000E71203A30700630303000283828011451C
:1038C00017F3FFFF670063C8411193962500AA858F
:1038D0002D4506C697F0FF1FE780E0F2B240014594
:1038E00041018280011122CC06CE3714004026CA45
:1038F0004AC84EC652C483447405034AB40583497A
:1039000084050349940597F0FFFFE780E09E834715
:10391000A40593F4F40F137AFA0F93E71700230D1D
:10392000F40493F9F90F1379F90FB717004003C79F
:10393000A705058B6DFF03D5C705A38D4705238C10
:103940003705A38C2705A38B9704F2406244D24429
:103950004249B249224A056182804111939705018B
:1039600022C406C626C2C1872E8463DC0700B7E4E2
:103970000400FC54829719C1BC5482972165218DA3
:1039800015A893F7150013C515008DE793F72500CB
:103990009DC797000000E78060EEB7E70400BC4FCA
:1039A0001306000A8945170500200345A5038297E1
:1039B00013452400B24022449244410182809397EF
:1039C000250163D80702B7E4040083A7C41E8297C9
:1039D00097000000E780E0EEBC4C37560700130666
:1039E00006308965170500200345C5FF82970965E4
:1039F00079B7939715010145E3DE07FA17D5010062
:103A00001305C52097B00100E780C05DB7E704004B
:103A1000BC4F13060064916517050020034585FC23
:103A200082971165A9BF2D71232A9110FD74E98C2D
:103A3000232C811023282111232631112A84AE89B9
:103A40003289930600100A86A6852D45232E111073
:103A500097F0FF1FE78020DB13154401B7E7040050
:103A6000FC4751810A0513962900CA850A95829759
:103A7000A68585660146254597F0FF1FE780A0D8FB
:103A80000A86A68593060010294597F0FF1FE78058
:103A900080D78320C111032481118324411103297C
:103AA00001118329C11015618280B7F7070003C790
:103AB0000701411106C622C426C24AC0A547631D9C
:103AC000F70097000000E78040F6B240224492449D
:103AD000024901454101828013942500AA8432895C
:103AE000A286AA850146254597F0FF1FE780A0D151
:103AF000A2864A86A685294597F0FF1FE780A0D0B9
:103B0000E9B71D71A2CC37E404005C5C485886CE4E
:103B1000494697D501009385E50A829711E917D5A3
:103B200001001305650B97B00100E780A04B01A0D1
:103B3000B7F600E0795798CAFD57DCCA0567B7E7C2
:103B400000E023A0E7101306F00290C223A0E718BC
:103B500001000100370700201847130600048145C3
:103B60009706002023AEE6E64157A38AE7403C448F
:103B700008088297971700209387C7833EC88567F8
:103B800013870740231AE1001D673ACC3707010568
:103B9000130707103ACE938757D11307B00F23109E
:103BA000E1022312F102054797F7FFFF93870754BD
:103BB0002301E1023ED817070000130727D197071A
:103BC0000000938767D2B7F50700BAC23EDC17073B
:103BD00000001307C7ED97070000938787CE814643
:103BE0003000E1051945BAC43EDE97F0FF1FE780BB
:103BF00080C118088147994630003E96034606006A
:103C000085070507A30BC700E398D7FEC24791C7F6
:103C10000357410185676373F70001A0B7E704000C
:103C200083A7470A08088297AA8511C917D50100FA
:103C30001305C5FB97B00100E780E02201A0F64024
:103C4000664425618280411126C2B7E4040083A73F
:103C5000040806C622C417050000130545D0829744
:103C600017040020130404D82300A40097000000C8
:103C7000E780800297000000E780A0BB03450400B6
:103C8000224403A38405B24092441306003289659E
:103C900041010283797106D622D413078008F337D5
:103CA000078093F787083EC201000100B717004064
:103CB000930570052380B704130680FA2380C70498
:103CC0000100010083C6F70293F6A60FA387D7026F
:103CD000238007049246F3A6068001000100733793
:103CE0000780137787083AC4010001002380B704D6
:103CF0002380C7040100010003C7F70213672700F0
:103D0000A387E70223800704A247F3A707800100E7
:103D10000100054597E0FFFFE78040619700000044
:103D2000E78020BA0147814681470546854513054E
:103D3000407E97E0FFFFE780406437E404003C44A6
:103D40006800514681458297B707C0A83EC8B7872B
:103D5000E803938707D03ECA97E7FF1F938727663C
:103D60003EC67C5868008297B250225445618280DA
:103D7000411197D501009385655117D501001305B1
:103D8000E5DF06C697B00100E780E00D17D501001A
:103D90001305856A97B00100E780E00CB240294521
:103DA000410117B301006700E310411197D50100ED
:103DB0009385054F17D50100130545DC06C697B05E
:103DC0000100E780400A17D501001305A56597B0EB
:103DD0000100E7804009B2402945410117B30100C5
:103DE0006700430D411122C406C6834705002A849B
:103DF0009DC797D501009385655017D50100130520
:103E0000E5D797B00100E78000064C4017D50100C8
:103E10001305C57097B00100E780E0043DA058414C
:103E20000DEF97D501009385654D17D5010013055A
:103E3000E5D497B00100E780000317D50100130512
:103E4000656F97B00100E78000022244B240294527
:103E5000410117B301006700E305A1679386D7030B
:103E60006313D70297D501009385454917D5010003
:103E70001305C5D097B00100E780E0FE17D501001B
:103E80001305456C7DBFED0797D501009385054768
:103E900017D50100130585CE631BF70097B001000D
:103EA000E78060FC17D501001305056B59BF97B07B
:103EB0000100E78040FB4C4017D501001305C56B9E
:103EC00091BF411197D501009385C53E17D50100DB
:103ED0001305C5CA06C697B00100E780C0F8B24016
:103EE0002945410117B301006700C3FC797122D451
:103EF00026D24AD02E842A898145B2844800714650
:103F000006D697E0FFFFE780C02297F7FF1F938751
:103F1000674CDC4783D70700231421012313F100EA
:103F200097500000E78020169547A305F1009307FE
:103F3000401F3EC6FD572305A100230AF1009750FC
:103F40000000E78080282686A28548009750000060
:103F5000E7804016B2502254925402594561828043
:103F600097270020239B079497270020238407840A
:103F7000B7E70400BC47411106C641468145170515
:103F8000002013056531829797200000E780A0602C
:103F900097200000E780A041014597600000E7807E
:103FA000C0A117070020034727319307F00A6315C4
:103FB000F7029307F0F88945170500201305C52F70
:103FC00017070020230AF72E97070020A386072E45
:103FD00097600000E78000C997600000E78060F507
:103FE0008145370504009707002023A5072A970776
:103FF0000020239F072897070020238C0728970776
:104000000020239D072097070020239B071E97076A
:104010000020239E07269707002023970728973024
:104020000000E780E056014597600000E78080CC03
:1040300097D501009385852A17D50100130505B48E
:1040400097B00100E78020E217D50100130505595C
:1040500097B00100E78020E1B2402945410117B344
:104060000100670023E5411122C406C626C293F76A
:1040700015002E84638F0710814617F6FF1F130665
:10408000A6328545170500200355451797C0000047
:10409000E780204F15C997D501009385E52417D5F2
:1040A00001001305A5AD97B00100E780C0DB17D56F
:1040B0000100130525C697B00100E780C0DA294545
:1040C00097B00100E78000DF97D501009385C521F7
:1040D00017D50100130585AA97B00100E780A0D885
:1040E00017D50100130545C497B00100E780A0D79C
:1040F000294597B00100E780E0DB17F5FF1F1305A6
:10410000652D5C4505472390E70097400100E78057
:10411000A0FF97D501009385251D17D50100130534
:10412000E5A597B00100E78000D417D5010013057D
:10413000E5C097B00100E78000D3294597B00100A2
:10414000E78040D7930710F8170700202306F716DB
:104150009707002083D7470A17070020A30EF714FC
:104160001705002013054515A18391451707002069
:104170002305F71497070020A38107149760000018
:10418000E78040AE13451400B240224492444101FE
:10419000828093F72500E1C3170700200357470FDC
:1041A00045CB970600209386E60E944297D70100F0
:1041B0009387C744170600200346A60D81451705BF
:1041C00000201305650D97700000E780E05AAA846F
:1041D00041C197D501009385E51917D50100130555
:1041E000E59997B00100E78000C8A68517D50100C2
:1041F000130545B697B00100E780E0C6294597B0A2
:104200000100E78020CB970700202393070893073E
:1042100010F8170700202301F70A9707002083D71B
:10422000A7FD17070020A309F708A183170700209F
:104230002305F70891458D47170500201305C5078D
:1042400017070020A30BF70697600000E78080A106
:104250001345240015BF93F74500D1C397D501003E
:104260009385451117D501001305459197B00100BD
:10427000E78060BF17D50100130585AF97B0010037
:10428000E78060BE294597B00100E780A0C2930790
:1042900020F8170700202301F7029707002083D793
:1042A000E7F717070020A309F700A18317070020ED
:1042B0002305F700854717070020A300F700975054
:1042C0000000E78080F0170500201305E5FE91450A
:1042D00097600000E78000991345440075B593F797
:1042E0008500A9C797D501009385C50817D501009A
:1042F0001305C58897B00100E780E0B617D5010027
:10430000130545A897B00100E780E0B5294597B0AF
:104310000100E78020BA97070020239B07F69770DB
:104320000000E780405513458400B9BD93F70501AF
:10433000D1C3854517050020035545EE9760010060
:10434000E780600797D501009385C50217D5010066
:104350001305C58297B00100E780E0B017D50100D2
:10436000130585A397B00100E780E0AF294597B01A
:104370000100E78020B4930730F817070020230DD1
:10438000F7F29707002083D767E917070020A305F6
:10439000F7F217050020130525F2A1838D451707B5
:1043A0000020230CF7F097600000E780A08B1345F6
:1043B0000401D9BB93F70502D1C797D501009385B6
:1043C00065FB17C501001305657B97B00100E78009
:1043D00080A917D501001305659E97B00100E780FD
:1043E00080A8294597B00100E780C0AC930740F84A
:1043F000170700202302F7EC9707002083D747E038
:1044000017070020A30AF7EAA18317070020230655
:10441000F7EA854717070020A301F7EA970700206E
:10442000239007DE97500000E78020DA1705002070
:10443000130585E8914597600000E780A082134549
:10444000040299B393F70504FDC397D50100938542
:1044500065F217C501001305657297B00100E7808A
:1044600080A017D501001305E59697B00100E780FD
:10447000809F294597B00100E780C0A397070020DF
:1044800083C787E31307700A6386E7061307800A6A
:10449000638CE7081307600A6393E704930760F8E7
:1044A00017070020230AF7E09707002083D727DEAD
:1044B00017070020A302F7E0A18317070020230EAF
:1044C000F7DE854717070020A30DF7DEB145170576
:1044D0000020130565DE97500000E780A078975014
:1044E0000000E78080CE1345040497070020239046
:1044F00007DA59B9930770F817070020230EF7DA87
:104500009707002083D7A7D817070020A306F7DA5C
:10451000A183170700202302F7DA85471707002039
:10452000A30EF7D8994565B7930780F8F1B793F7CD
:1045300005080145E38A07C497D50100938585E303
:1045400017C501001305856397B00100E780A091AE
:1045500017D501001305858997B00100E780A09069
:10456000294597B00100E780E0949307A0F817076A
:1045700000202303F7D49707002083D7E7D217073B
:104580000020A30BF7D2A183170700202307F7D23F
:10459000854717070020A302F7D29707002023952D
:1045A00007D097500000E78040C217050020130590
:1045B000A5D0914597500000E780C06A13450408D4
:1045C000E1B6411122C497D50100938565D42A84B0
:1045D00017C501001305855A06C697B00100E7808C
:1045E00080884C4017D501001305C5F097B0010035
:1045F000E7806087294597B00100E780A08B0347DB
:1046000004009307F00F631FF70297D5010093850D
:1046100025D017C501001305655697B00100E78046
:1046200080844C4017D501001305C5ED97B00100FB
:10463000E78060832244B2402945410117B301005D
:1046400067004387B240224441018280B1C14111D9
:1046500022C417C50100130565522E8497D50100A9
:10466000938505C606C697A00100E780C07FA28596
:1046700017D50100130545F497A00100E780A07E3F
:104680002244B2402945410117B3010067008382EB
:104690008280411122C426C22E84AA8497D50100AB
:1046A0009385C5C217C501001305454D06C697A0E1
:1046B0000100E780407B17D501001305A5F097A006
:1046C0000100E780407A294597A00100E780807EBD
:1046D00097D50100938585BF97070020239097B257
:1046E00017C50100130585498544970700202395C8
:1046F00087B097070020239297B097170020239E3A
:10470000871A97A00100E78000769715002083D5CF
:10471000C51A17D50100130565EB97A00100E780C6
:104720008074294597A00100E780C0789717002082
:104730002382970897200000E78060C72285975062
:104740000000E7808027054597500000E780805AE9
:1047500097F7FF1F938707C8DC4703D70700C16798
:10476000FD176312F7022244B7E70400B2409244F7
:1047700003A3870517F5FF1F034545271306000A06
:10478000854541010283B240224492444101828026
:10479000011122CC37E404005C5C06CE354697D587
:1047A00001009385A5CA17E50100130565AF82973F
:1047B00011E917C501001305254297B00100E780F4
:1047C000608201A097F7FF1F938707233EC4B7F5C8
:1047D0000700856793870780814617F6FF1F13063A
:1047E0002621E10519453EC697E0FF1FE780A0019D
:1047F0007C44194697F5FF1F9385851F17050020F8
:10480000130505A28297340017F6FF1F1306461EF4
:1048100097D501009385451117D501001305451261
:1048200097700000E78040CA2A841DCD97D501000B
:10483000938545B117C501001305453497A00100C4
:10484000E7806062A28517D50100130525C197A0F6
:104850000100E7804061294597A00100E78080655D
:10486000F24062440561828097E00000E780A02C5E
:1048700017D50100130585B597600000E78080BE5D
:1048800097B00000E780E08097600100E78060E576
:1048900017F5FF1F130585B097600100E78000CE74
:1048A00017D50100130585B397600100E780E0E5A7
:1048B0002A8497600000E780C02497100100E780F9
:1048C00040BD97800100E780605697700000E78048
:1048D000007D97700000E780C09A97300100E78064
:1048E000A07E97D501009385E5A517C501001305A6
:1048F000E52819C897A00100E780E056A28517D5E2
:1049000001001305E5B7A1B797A00100E780A05506
:1049100017D50100130505B997A00100E780A05441
:10492000294597A00100E780E05897300100E78013
:10493000805A97F00000E780407955C985453705D2
:10494000040097300000E780A0C497D5010093854C
:10495000659F17C501001305652297A00100E78038
:10496000805017D50100130565B597A00100E780B9
:10497000804F294597A00100E780C05397F7FF1F9C
:104980009387079583D70700171700202317F7F29F
:10499000854717170020230FF7E097200000E780D6
:1049A00000BA97200000E78080A01715002003556B
:1049B000C5F097500000E780400005459750000083
:1049C000E780403397D501009385C59717C501004F
:1049D0001305C51A97A00100E780E04817D501002C
:1049E000130505B097A00100E780E047ADB597D566
:1049F00001009385259517C501001305251897A07B
:104A00000100E780404617D50100130525BD97A09A
:104A10000100E7804045294597A00100E7808049D3
:104A2000014569BF411122C437E404008327041AF9
:104A300006C6829797500000E780E0FB83270408B2
:104A400017F5FFFF13056562829797F7FF1F238F06
:104A5000A7F817F5FF1F1305E59797500000E780AB
:104A600060A92244B240410117030000670083D2CD
:104A7000411106C622C426C299C1AA8415ED97D554
:104A800001009385258D17C501001305250F97A0FB
:104A90000100E780403D17C501001305E52597A0FB
:104AA0000100E780403C2244B24092442945410144
:104AB00017A301006700034037E404007C4441462B
:104AC00017F5FF1F1305457D829717F5FF1F130587
:104AD000A57C97200000E780A09F97200000E7803A
:104AE000008D03238405224497F7FF1F2392977AB2
:104AF000B240924417F5FF1F034545EF1306000A25
:104B0000894541010283B7E70400FC471171A2DD2A
:104B1000CAD986DFA6DBCED72E8432892E86AA8517
:104B200017F5FF1F13054579829717F7FF1F130726
:104B3000A77883470700930680029387E70793F7D8
:104B4000F70FE3ECF610BA898A0717C701001307BD
:104B5000270CBA979C43BA9782878D4797D5010057
:104B60009385858217C5010013054501630FF40085
:104B700097A00100E780202F17C501001305853D90
:104B800097A00100E780202EBDA497A00100E78038
:104B9000802D17C501001305653D97A00100E78032
:104BA000802C294597A00100E780C030930720F8AA
:104BB000114697F5FF1F938525704A8517F7FF1F4C
:104BC000230CF76E97F7FF1FA389076E97F0FFFF7F
:104BD000E78000322A841DC997C501009385C57AF4
:104BE00017C50100130585F997A00100E780A027EC
:104BF000A28517C501001305253B97A00100E7809A
:104C00008026294597A00100E780C02A97C50100AA
:104C10009385857717C50100130545F697A0010018
:104C2000E780602417C501001305453997A00100EE
:104C3000E7806023294597A00100E780A027416510
:104C4000930730FA054697F5FF1F9385E5667D15B6
:104C500017F7FF1F2302F76697F0FFFFE780402951
:104C60002A841DC997C501009385057217C50100E7
:104C70001305C5F097A00100E780E01EA28517C5C7
:104C800001001305653297A00100E780C01D29458A
:104C900097A00100E7800022B7E70400BC4F05663B
:104CA000130606C8A14517F5FF1F034525D48297B3
:104CB000FE506E54DE544E59BE59116182809147A8
:104CC0006303F40297C501009385056C17C50100C5
:104CD0001305C5EA97A00100E780E01817C5010099
:104CE0001305053171BDB7E70400FC4F914517F579
:104CF000FF1F0345A5CF829797C501009385C5681F
:104D000017C50100130585E797A00100E780A015EE
:104D100017C501001305852F97A00100E780A01497
:104D2000294597A00100E780E01897400000E78040
:104D3000C049914535A485476303F40297C5010036
:104D40009385856417C50100130545E397A001000D
:104D5000E780601117C501001305C52C15B597F73D
:104D6000FF1F239D274BB7E704000566BC4F1306C2
:104D700006C8C1450DBF8D476303F40297C5010006
:104D80009385856017C50100130545DF97A00100D5
:104D9000E780600D17C501001305852AD5B3930779
:104DA00040F8114697F5FF1F938505514A8517F77F
:104DB000FF1F2303F75097F7FF1FA380075097F0BB
:104DC000FFFFE780E0122A84E30405EE97C50100A7
:104DD0009385855B17C50100130545DA97A001008F
:104DE000E7806008A28517C501001305E51B97A0A1
:104DF0000100E7804007294597A00100E780800B6C
:104E000045BD9147E31CF4F6B7E70400FC4F93055A
:104E1000000217F5FF1F034565BD829797C5010086
:104E20009385855617C50100130545D597A0010048
:104E3000E780600317C5010013050522F1BD89470E
:104E400063E3870297C501009385055417C50100E8
:104E50001305C5D297A00100E780E00017C5010047
:104E60001305C52031BB97F4FF1F83C4044597F792
:104E7000FF1F83C7774497C501009385E550A204BF
:104E800017C50100130585CFDD8C97A00100E780D1
:104E900080FDA28517C501001305851E97A001009E
:104EA000E78060FCC204294597A00100E7808000EC
:104EB000C1849305D4FF93960401C1824A8693F579
:104EC000F50F17F5FF1F1305553F97200000E780EA
:104ED000E06FE35F90DC930750F817F7FF1F230D97
:104EE000F73C83C73900228697F5FF1F9385C53CA1
:104EF00085074A8517F7FF1FA301F73C97F0FFFFCF
:104F0000E78000FF2A84E30505DA97C50100938551
:104F1000A54717C50100130565C697A00100E780E6
:104F200080F4A28517C5010013050568C9B5894736
:104F300063E3870297C501009385054517C5010006
:104F40001305C5C397A00100E780E0F117C5010074
:104F50001305C51435B197400000E7800027A285EE
:104F600017F5FF1F1305453597500000E78080CFE8
:104F700081B38D476303F40297C501009385C54053
:104F800017C50100130585BF97A00100E780A0EDBC
:104F900017C5010013054512E5B6B76602000146C4
:104FA000B7750200054597E0FF1FE780C0859307AE
:104FB00060F817F7FF1F2301F73097F7FF1FA38E45
:104FC000072E9307000617F7FF1F2309F72E8947BF
:104FD00017F7FF1FA304F72E97F7FF1F2381072E54
:104FE00097F7FF1FA38D072CC14717F7FF1F230952
:104FF000F72C930720F917F7FF1FA303F72C31466F
:1050000097F7FF1FA38FA72A97F5FF1F9385C52A40
:105010004A8597F7FF1F2386072A97F0FFFFE7804F
:1050200020ED2A84E30605C897C501009385C535A0
:1050300017C50100130585B497A00100E780A0E221
:10504000A28517C501001305A50855B3B147630331
:10505000F40297C501009385253317C50100130598
:10506000E5B197A00100E78000E017C50100130536
:10507000E50739B6B7E70400FC4F9305000417F5C0
:10508000FF1F0345A596829797400000E780E01335
:10509000B145F9B5914763E3870297C50100938550
:1050A000A52E17C50100130565AD97A00100E78087
:1050B00080DB17C5010013052505D9B497F4FF1F40
:1050C00083C4C41F97F7FF1F83C7371FA204DD8C5B
:1050D0008E04B77702006D14BE942286A68517C58C
:1050E00001001305A50397A00100E780C0D7B7E72B
:1050F0000400FC47228697F5FF1F9385351C280086
:10510000829793160401C1823000A685094597D085
:10511000FF1FE780406F2A8409C917C501001305E6
:10512000A50197A00100E780E0EB930770F819460E
:1051300097F5FF1F938545184A8517F7FF1F230D25
:10514000F71697F7FF1FA38B871697F0FFFFE780EF
:1051500020DA2A84E30E05B497C501009385C522A1
:1051600017C50100130585A197A00100E780A0CF16
:10517000A28517C50100130525FD95B99947630B55
:10518000F41297C501009385252017C5010013056A
:10519000E59E97A00100E78000CD17C5010013052B
:1051A00025FCF9BA914763E3870297C5010093850F
:1051B000A51D17C501001305659C97A00100E78098
:1051C00080CA17C50100130525FB5DBA97F4FF1FC0
:1051D00083C4C40E97F7FF1F83C7370EA204DD8C6C
:1051E0008E04B77702006D14BE942286A68517C57B
:1051F00001001305A5F997A00100E780C0C6B7E735
:105200000400FC47228697F5FF1F9385350B280085
:10521000829793160401C1823000A6850D4597D070
:10522000FF1FE780405E2A8409C917C501001305E6
:10523000A5F797A00100E780E0DA930780F8194608
:1052400097F5FF1F938545074A8517F7FF1F23052D
:10525000F70697F7FF1FA383870697F0FFFFE78006
:1052600020C92A84E30605A497C501009385C511CA
:1052700017C501001305859097A00100E780A0BE27
:10528000A28517C50100130565F395B69947630319
:10529000F40297C501009385250F17C5010013057A
:1052A000E58D97A00100E78000BC17C5010013053C
:1052B00065F2F9B0B7E70400FC4F9305000417E569
:1052C000FF1F0345A572829797400000E780E0EF3B
:1052D000994579B18D476303F40297C50100938521
:1052E000A50A17C501001305658997A00100E7808D
:1052F00080B717C50100130565EF59B017C5010048
:105300001305C5EF97A00100E780C0CD1305C012BB
:1053100097D0FF1FE780E002014597E0FFFFE7809D
:10532000E0D90D4597100000E780E0A3294597D00C
:10533000FF1FE780000197D0FF1FE78060F18DBA63
:1053400099476303F40297C501009385E50317C5E8
:1053500001001305A58297A00100E780C0B017C522
:105360000100130565EA29B817F7FF1F034717F572
:1053700097F7FF1F83C787F422075D8F9166BA9660
:10538000C2061166C1821306F6EF8D476365D60229
:1053900097E7FF1F938707049C4B17F6FF1F0346F1
:1053A000D6F19386C7002DC203D6070069CA8907C4
:1053B000E39CD7FE89471307A0F8114697F5FF1F16
:1053C000938585EF4A8597F6FF1F2387E6EE17F74B
:1053D000FF1FA304F7EE97F0FFFFE78060B12A8478
:1053E000E308058C97C50100938505FA17B5010000
:1053F0001305C57897A00100E780E0A6A28517C530
:1054000001001305A5E1E5B203D60700630EE60A25
:105410008907E39BF6FE8D4779BF91476304F40249
:1054200097C50100938545F617B50100130505756D
:1054300097A00100E78020A317C50100130585DFB1
:105440006FF00FF4B7E70400FC4F9305000817E571
:10545000FF1F0345A5598297C9B897C501009385D9
:10546000A5F217B501001305657197A00100E7804B
:10547000809F17C50100130565DD6FF06FF0239065
:10548000E70017E5FF1F1305E5F497300100E780FB
:1054900000CA97C50100938525EF17B501001305D4
:1054A000E56D97A00100E780009C17C5010013057A
:1054B000E5DA97A00100E780009B294597A001004D
:1054C000E780409F8147C5BD2390070017E5FF1F78
:1054D000130545F097300100E78060C597C50100CE
:1054E000938585EA17B501001305456997A001006A
:1054F000E780609717C501001305C5D75DBF41114F
:1055000022C406C626C24AC0834705002A84A1C316
:1055100097C50100938505E117B5010013050566E0
:1055200097A00100E78020944C4017C501001305A7
:10553000E50D97A00100E78000932244B240924419
:1055400002492945410117A301006700A39658416C
:10555000B707CF009387777D631CF7080445638501
:1055600004120359C500630109120354E50097C5ED
:105570000100938525DB17B501001305256097A071
:105580000100E780408E03C60400A286CA8517C5C5
:1055900001001305250997A00100E780C08C29456B
:1055A00097A00100E78000914A86A6852285972072
:1055B0000000E78020DA83C7140003C70400A207B5
:1055C000D98F13978700A183D98FC2073167C18311
:1055D0001307C755638AE70A22862244B240CA8568
:1055E000268502499244410117F3FFFF6700E3510A
:1055F000B707CC009387777D6310F70697C5010046
:10560000938545D217B501001305455797A00100B2
:10561000E78060851C448355C4008356E40003C6BC
:10562000070017C501001305E5FF97A00100E780FB
:105630008083294597A00100E780C0870356C400F6
:105640000C440355E4002244B24092440249410113
:1056500017230000670003D0B707CE009387777D3C
:105660006304F70297C501009385C5CB17B5010008
:105670001305C55097900100E780E07E4C4017C5A8
:105680000100130565EF75B5B2402244924402490A
:1056900041018280B7E70400FC4741112E8606C60F
:1056A00022C426C24AC02E842A89AA8517F5FF1F64
:1056B000130585C0829797C501009385A5CE17B5C0
:1056C00001001305A54B97900100E780C07997F57D
:1056D000FF1F83C565BE17B501001305A57297901E
:1056E0000100E7804078294597900100E780807CA1
:1056F00097F4FF1F938444BC83C7040041479387FA
:10570000070693F7F70F636AF75C17B701001307F3
:10571000675A8A07BA979C43BA9782879D4763075F
:10572000F40297C501009385E5C717B5010013057D
:10573000E54497900100E780007317B50100130559
:10574000E56C97900100E7800072ADAC97F7FF1F02
:1057500083C797B6DDCB17F7FF1F034717B697F739
:10576000FF1F83C787B522075D8F97F7FF1F83C78A
:10577000E7B4C2075D8F97F7FF1F83C737B4E2070F
:10578000D98F17F7FF1F2327F7B083C7640097C58A
:105790000100938525C117B501001305253E17F7B4
:1057A000FF1F2308F7AE97900100E780C06B97F7C3
:1057B000FF1F938727AE8C4317F6FF1F034666AD86
:1057C00017B501001305456697900100E780A069B1
:1057D000294597900100E780E06D97F7FF1FA38DA3
:1057E00007AC2244B24092440249930700F817F7ED
:1057F000FF1F2303F7AC9D4517F5FF1F1305C5AB2E
:105800004101174300006700E34597600000E7800F
:10581000001697F7FF1F2382A7AA9357850017F753
:10582000FF1FA30CF7A8935705012A8417F7FF1F42
:105830002306F7A893578501014517F7FF1FA30F0C
:10584000F7A697600000E780401397F7FF1F2388B3
:10585000A7A697C501009385E5B417B50100130508
:10586000E53197900100E780006017F6FF1F0346BF
:1058700006A5A28517B501001305855CB1B7CD4714
:105880006303F40297C501009385C5B117B5010004
:105890001305C52E97900100E780E05C17B5010065
:1058A0001305855B79BD37E404007C44414697F5D8
:1058B000FF1F938575A017F5FF1F1305E59D8297C0
:1058C00017F5FF1F1305459D97100000E78040C0A6
:1058D00097100000E780A0AD97F7FF1F83C7E79EF2
:1058E00017F7FF1F0347579EA20703238405D98F8D
:1058F00017F7FF1F231EF7981306000A8945224455
:10590000B2409244024917E5FF1F0345250E4101AD
:1059100002838D476303F40297C50100938585A830
:1059200017B501001305852597900100E780A05366
:1059300017B501001305056229B517F4FF1F0344CD
:10594000C49797F7FF1F83C7379797C501009385C3
:1059500065A5220417B50100130545225D8C9790BB
:105960000100E7804050A28517B50100130545509E
:1059700097900100E780204F294597900100E7802C
:1059800060530D4697F5FF1F93850593228597E099
:10599000FFFFE780E055AA8421C197C501009385E8
:1059A00065A017B501001305651D97900100E780FC
:1059B000804BA68517B501001305C54C97900100D3
:1059C000E780604A2244B24092440249294541019D
:1059D000179301006700034E97F7FF1F23908784FA
:1059E000B7E70400116603A38705130606E891458F
:1059F00039B78D476303F40297C501009385859AF3
:105A000017B501001305851797900100E780A045A1
:105A100017B501001305C5622DB317F4FF1F03442A
:105A2000C48997F7FF1F83C7378997C501009385FE
:105A30006597220417B50100130545145D8C9790F6
:105A40000100E7804042A28517B501001305C54457
:105A500097900100E7802041294597900100E78059
:105A600060450D4697F5FF1F93850585228597E0D4
:105A7000FFFFE780E047AA841DC197C50100938519
:105A8000659217B501001305650F97900100E78037
:105A9000803DA68517B501001305454105B797E779
:105AA000FF1F239F8774B7E70400116603A38705D0
:105AB000130606E89305000299B5894763E3870258
:105AC00097C501009385058E17B501001305050BD9
:105AD00097900100E780203917B50100130505599B
:105AE0008DB197E4FF1F83C4447D97E7FF1F83C7F1
:105AF000B77C97C501009385E58AA20417B501001C
:105B00001305C507DD8C97900100E780C035A68599
:105B100017B501001305053B97900100E780A034FD
:105B2000294597900100E780E038228697E5FF1F1E
:105B300093858578268597E0FFFFE780603B2A8480
:105B4000630E051A97C501009385C58517B5010039
:105B50001305C50297900100E780E030A28517B5D4
:105B600001001305653799BD854763F9871883459B
:105B700019002244B24092440249B335B00097E77D
:105B8000FF1F2387B76A17B50100130525364101AA
:105B9000179301006700232DA2852244B24092444E
:105BA0004A85024941011703000067000322994713
:105BB0006303F40297B501009385C57E17B5010014
:105BC0001305C5FB97900100E780E02917B5010098
:105BD00013058563BDB617E4FF1F0344046E97E702
:105BE000FF1F83C7776D97B501009385A57B2204BE
:105BF00017B50100130585F85D8C97900100E780CB
:105C00008026A28517B501001305C52F97900100C6
:105C1000E7806025294597900100E780A029194673
:105C200097E5FF1F93854569228597E0FFFFE78091
:105C3000202CAA841DC197B501009385A57617B5C0
:105C400001001305A5F397900100E780C021A68508
:105C500017B501001305052C95B397E7FF1F239592
:105C60008764B7E70400116603A38705130606E8F7
:105C70009305000869B1854797B501009385857242
:105C800017B50100130585EF630BF4009790010031
:105C9000E780601D17B50100130505295DB49790D5
:105CA0000100E780401C17B5010013056529979096
:105CB0000100E780401B294597900100E780801F85
:105CC0002244B2409244024997E7FF1F2392075CA7
:105CD000410117630000670003BA97B5010093857F
:105CE000656C17B50100130565E997900100E78021
:105CF000801717B5010013056555A1B4B2402244C1
:105D00009244024941018280411106C622C497E0B3
:105D1000FFFFE780E01D9377F50FA1C32A8497B5B5
:105D200001009385A56917B50100130525E5979036
:105D30000100E78040139375F40F17C501001305A8
:105D4000A58697900100E78000122244B2402945C1
:105D50004101179301006700E315B240224441015D
:105D60008280411122C491462A8417E6FF1F130640
:105D7000E6629D652D4506C697D0FF1FE780A0A867
:105D8000B7F7070003C70701A5476313F70001A092
:105D90009306001001469D65254597D0FF1FE780BB
:105DA00080A697E7FF1F238B875E2244B24091466F
:105DB00017E6FF1F1306865E9D652945410117D32F
:105DC000FF1F670043A41171CED7B7E9040083A772
:105DD000C904CAD917E9FF1F1309094EA2DD2E868F
:105DE00086DFA6DB2E84AA854A85829797E7FF1F68
:105DF00083C7874C1307700A6385E710636DF7004C
:105E00001307600A6385E704FE506E54DE544E5952
:105E1000BE59116182801307800A6385E716130754
:105E2000900AE393E7FE8D476306F41C97C50100D3
:105E30009385C58A17B50100130545D497900100D5
:105E4000E780600217C501001305858625A08D47F0
:105E5000630CF40297C501009385458817B50100CE
:105E60001305C5D197900100E780E0FF17B5010049
:105E70001305457D97900100E780E0FE2945979046
:105E80000100E780200349B7854717B501001305D6
:105E9000257D17E7FF1F230DF73897900100E78056
:105EA0006014B7750200B76602000146054597D039
:105EB000FF1FE7804095930760F817E7FF1F230D4A
:105EC000F73E97E7FF1FA38A073E9307002617E7D1
:105ED000FF1F2325F73EE5779387072117E7FF1F6D
:105EE0002310F73EB14597E7FF1F238C073C97E748
:105EF000FF1FA388A73C4A8597000000E780401653
:105F000021B7914763E3870297B501009385057D2B
:105F100017B50100130585C697900100E780A0F42E
:105F200017B501001305C575B1B797E4FF1F83C40A
:105F3000E43897E7FF1F83C75738A204DD8C83A797
:105F4000C9046D14228697E5FF1F93853537280015
:105F500082978E0493160401B7750200C182300047
:105F6000A695094597D0FF1FE780E089930770F851
:105F700017E7FF1F2302F734994597E7FF1FA38F09
:105F8000A73295BF914763E3870297B501009385D8
:105F9000E57417B50100130565BE97900100E78011
:105FA00080EC17B501001305256FE9B597E4FF1FD5
:105FB00083C4C43097E7FF1F83C73730A204DD8C4A
:105FC00083A7C9046D14228697E5FF1F9385152FBB
:105FD000280082978E0493160401B7750200C182CF
:105FE0003000A6950D4597D0FF1FE780C08193072D
:105FF00080F8BDBF17B501001305C56C979001006F
:10600000E78040FE930790F82304F10083471900CE
:106010008D452800A304F100834729002305F100E2
:1060200097000000E780C0031305C01297C0FF1F50
:10603000E7802031014597D0FFFFE78020080D451C
:1060400097000000E78020D2294597C0FF1FE78016
:10605000402F97C0FF1FE780A01F7DB397E7FF1F6A
:106060009387C73403A30700630303000283174326
:106070000000670023BF8280011126CA06CE22CC11
:106080000344550083474500AA8422045D8C2EC634
:1060900017B5010013054567A28597900100E780B9
:1060A00080DC228562443246F240A685D2440561F6
:1060B00017030000670083C5011122CC2A8417B59D
:1060C00001001305656306CE2EC697900100E78098
:1060D00060F122856244B245F24005611713000069
:1060E0006700E3368D4763FBB70A011126CA06CE67
:1060F00022CC0344350097E4FF1F83C4742B97B56B
:1061000001009385A561B337800017E7FF1FA30146
:10611000F72A09C497B501009385056117B50100F9
:106120001305056197900100E780E0D397E7FF1F13
:1061300083C717286386970097000000E780402BED
:1061400097E7FF1F83C7D7268DC785472306F10032
:10615000B7E7040083A74717700085451305503043
:10616000829717B501001305A55D97900100E780A0
:1061700060E79967938757EE2316F100680085471B
:106180009145A30781002307F10097000000E780F5
:1061900020EDF2406244D2440561828082808947CA
:1061A00063F7B708011122CC06CE26CA8344250026
:1061B00085472A84639DF404914763F5B70403453A
:1061C00045008347340022055D8D97D7FF1F239438
:1061D000A72297000000E780E0439967938767EE66
:1061E0002314F1008347340023059100A305F10037
:1061F00083474400954528002306F10097000000DE
:10620000E78000E6F2406244D24405618280FDF8F6
:106210009967938767EE2314F10097D7FF1F83D701
:10622000871DA305F10023050100A183E1B782804A
:106230000111996722CCD51717F4FF1F1304845757
:106240002314F1008347040026CA97F4FF1F9384A8
:10625000C4662305F10083D7040028009545A305F3
:10626000F100A18306CE2306F10097000000E7802D
:1062700020DF03D604008345040017B50100130591
:10628000A54D97900100E78000BEF2406244D244E1
:10629000056182809D677971D9172316F10097F700
:1062A000FF1F83C7275106D62307F100A9C3B7E70D
:1062B0000400FC47414697E5FF1F9385E5FD130564
:1062C000F10082976800CD4597000000E78040D933
:1062D00097F5FF1F83C5054E17B501001305C54A85
:1062E00097900100E78020B8B25045618280B7E7FF
:1062F0000400BC47414681451305F1008297D9B798
:1063000045C5411106C622C4930750FA2300F50083
:106310009307A005A300F50089472301F5009147E5
:10632000A301F50093078002A302F50097F7FF1F72
:106330009387474883C70700230205002A84230365
:10634000F50097E7FF1F9387B70683C7070041460D
:1063500097E5FF1F938545F4A303F50097F7FF1F0B
:1063600083D7A7552304F500A183A304F50097D78D
:10637000FF1F83D747082305F500A183A305F50078
:10638000B7E70400FC47310582972285F145970065
:106390000000E7802024230EA4002181A30EA40086
:1063A000B24022444101828082805D710A8586C6A6
:1063B000A2C497000000E780E0F437E404007C44C6
:1063C0008A850810794682973C441305E103094603
:1063D00081458297101093050002014597D0FFFF79
:1063E000E7800034B640264461618280B7C7A55A71
:1063F00001119387C7333EC497E7FF1F83C757FB3D
:106400003EC6B7F7070003C7070106CE22CCA54753
:106410006313F70001A01164930504F093060010C4
:106420000146254597C0FF1FE780E03D30009305FA
:1064300004F0A146294597C0FF1FE780C03C97E5BF
:10644000FF1F83C5F5F617B501001305A544979006
:106450000100E78040A1F2406244056182800111A1
:106460009165A1463000938505F02D4506CE97C075
:10647000FF1FE78040392247B7C7A55A9387C73324
:106480006314F702B24517B501001305E533B335C0
:10649000B00097E7FF1FA38DB7F097900100E7804A
:1064A000809CF24005618280814517B5010013058B
:1064B000E53397E7FF1FA38D07EE97900100E78074
:1064C000809A97000000E780A0F2E1BFB7C7A55A05
:1064D00079719387F7353EC6B7E70400FC47AA8574
:1064E00006D622D4414608088297B7F7070003C7AB
:1064F0000701A5476313F70001A01164930504E8A1
:10650000930600100146254597C0FF1FE780A02F86
:106510007000930504E8D146294597C0FF1FE78026
:10652000802E17B501001305A53A97900100E7806A
:1065300060ABB25022544561828079719165D14639
:106540007000938505E82D4506D697C0FF1FE780AC
:10655000802B3247B7C7A55A9387F73517B5010087
:106560001305C5306310F702B7E70400FC4717E5D1
:10657000FF1F130565D241460C08829717B501002D
:106580001305C52C97900100E780C0A5B250456166
:106590008280B7F7070003C70701A5476313F70019
:1065A00001A091654111930600100146938505E80D
:1065B000254506C697C0FF1FE780E024B24017B507
:1065C00001001305A51E410117930100670083A177
:1065D000C16769768146FD17050613970601418359
:1065E0006364B7003E8582803307D5000347070008
:1065F000B98F214713F81700858363050800B18F11
:10660000C207C1837D171377F70F6DF78506F1B7C2
:10661000B7C7A55A01119387E7343EC42AC6B7F716
:10662000070003C7070106CE22CC26CAA54763137D
:10663000F70001A091642A84938504EE930600106C
:106640000146254597C0FF1FE780E01B3000A146AB
:10665000938504EE294597C0FF1FE780C01AA285E5
:1066600017B501001305052597800100E780A07F7D
:1066700097000000E780A0D3F2406244D244056155
:10668000828001119165A1463000938505EE2D456C
:1066900006CE97C0FF1FE78000172247B7C7A55A4D
:1066A0009387E7346318F702B24517B50100130565
:1066B000E51597D7FF1F2390B7D4C205C1819780F6
:1066C0000100E780407A97000000E78040CEF2406A
:1066D00005618280D147D14517B501001305051525
:1066E00017D7FF1F2319F7D097800100E780A07705
:1066F00017D5FF1F035525D097000000E78080F1D4
:10670000F9B721C1411126C206C622C4AE848DC587
:106710002A8497100000E780E0E397E7FF1F83C714
:1067200027C999CB22852244B240A68592444101D3
:106730001733000067000353B240224492444101E2
:106740008280828001114AC806CE22CC26CA4EC65B
:1067500093F715002E899DCBAD67371700409387BF
:10676000A7AA1CC3B7E70400BC4F13060019854550
:1067700017D5FF1F034505C8829713451900F2403E
:106780006244D2444249B2490561828093F72500B0
:106790006389071817F7FF1F03570712954763F917
:1067A000E70C014417F6FF1F130606019306300598
:1067B00013055004130810049308B0041303900544
:1067C000930764006374F7043A84FD5997F4FF1F3C
:1067D00083C484FE97F7FF1F83C717FEA204DD8CD6
:1067E000AD679387B755638AF41063E3970AA96787
:1067F0009387A755638DF410A28517F5FF1F130526
:10680000A5FB97000000E78000F0E9A0B307860031
:1068100083C50700639AD50483C517006396A50452
:1068200083C527006392050583C53700639ED502A3
:1068300083C54700639A150383C7570063966702B1
:10684000A2890DE897F5FF1F83D50507B38535416C
:10685000C20517F5FF1F130525F6C1814E95970058
:106860000000E78040EA59A005044204418089BF46
:106870003A84FD598547E3EB87F435C4854517F520
:10688000FF1F130565F397000000E780C0E7A1A88C
:10689000B1679387C755638FF402B5679387D75560
:1068A000E39CF4F4A28517F5FF1F1305E5F097307C
:1068B0000000E780203B8947630EF4009305E4FF66
:1068C000C205C18117F5FF1F130525EF97100000C2
:1068D000E78040C8A68517B50100130565019780BC
:1068E0000100E7804058FD57E39EF9F497F7FF1F3A
:1068F000239407FC1345290059B5A28517F5FF1FFE
:10690000130585EB97F0FFFFE7804077E1B7A2859D
:1069100017F5FF1F130545EA97F0FFFFE780007AA0
:1069200055BF93F745000145E38B07E417B5010018
:10693000130545FD97800100E780C06A973000008D
:10694000E780E060134549001DBD411122C437E4D2
:1069500004005C5C06C6354697B50100938505AF1B
:1069600017C501001305C593829711E917B50100FA
:10697000130505FA97800100E780C06601A0832710
:10698000041C82972A84054597C00000E780001AFE
:1069900097700100E780209F97600100E7802074D6
:1069A00097B00000E780802B2285B240224441014D
:1069B00082801567B71700401307575598C3D8430F
:1069C0009D66558FD8C3D843FD76758FD8C3D843FD
:1069D0001367F70FD8C335671307C7CC98C38280F6
:1069E0004111054506C622C426C297C0FFFFE780B5
:1069F000C0561305A00497B0FF1FE780406B757564
:106A000085457D1597C0FFFFE78060407D75854512
:106A10001305F53697C0FFFFE780C04937140040E3
:106A20008327840A8D451305002093E7072023243C
:106A3000F40A97C0FFFFE780803DB7E4040097D0D9
:106A4000FFFFE780A082C85897800100E780805947
:106A500017C501001305C58497800100E7808058A1
:106A60008327840C8545414593E707082324F40CCC
:106A700097C0FFFFE78000448D451305000897C0CD
:106A8000FFFFE780204397C0FFFFE780007037A536
:106A900007001305051297C0FFFFE780A06B0145B3
:106AA00097C0FFFFE780C07195450545894717F7F7
:106AB000FF1F2305F7E097C0FFFFE7800072B7E7ED
:106AC00000E013070006238DE7403707000423A0EA
:106AD000E71097D0FFFFE780000397D0FFFFE78024
:106AE000C01697000000E78080E697000000E7806E
:106AF000409797000000E78000B997100000E780FA
:106B0000A0A697E0FFFFE78020F297000000E78053
:106B1000602D97100000E780609F83A70408170589
:106B20000000130565C2829797D7FF1F2384A78CA7
:106B3000BC4C130600648545829797000000E780EF
:106B400080E797C0FF1FE780A08A01458280B7F7E2
:106B5000070003C70701A547AE866316F7009397A2
:106B6000450191C301A0AA850146254517C3FF1F12
:106B7000670063C94111B2862E86AA852D4506C6D7
:106B800097C0FF1FE78020C8B240014541018280C5
:106B90009307000463E8C7021D71A2CC2A84080889
:106BA00086CE32C697800100E7808020B24610086A
:106BB000A285294597C0FF1FE780E0C4F6406644E0
:106BC000256182803955828097F7FF1FA38607D4FD
:106BD00097F7FF1F238207EA97F7FF1F238E07D23D
:106BE000B7E70400FC5F411106C682978967938767
:106BF00007F4B2403E9597F7FF1F23ADA7D04101A0
:106C00008280930600022547830705006385D7002D
:106C10006383E70082800505C5BF17F5FF1F0345A5
:106C200045CF0DE5411122C417F4FF1F130484CE94
:106C30001C4006C681CBB7E70400FC5F82971C406E
:106C40001D8D7D81B24022444101828005458280B4
:106C50008145B307B5008387070091E789C91723EA
:106C60000000670023F68505C205C181DDB782807B
:106C7000AA871375F50F130705FD1377F70FA546C0
:106C800063E5E600138507FD82801307F5F91377A6
:106C9000F70FE54663E6E600011593178501E187E6
:106CA0001387F7FB1377F70F95467D5563E4E600EE
:106CB000138597FC828035C5011126CA4AC84EC685
:106CC00052C406CE22CCAE8997000000E780A0F324
:106CD0002A898144414A0305090097000000E780A2
:106CE00060F92A840305190097000000E78080F806
:106CF00063470402634505021204B3879900498C77
:106D00002380870085040909E39744FD0545F24087
:106D10006244D2444249B249224A05618280014517
:106D2000FDB7014582808147E5483387F5000307B9
:106D3000070019E305458280B306F50003860600C7
:106D40009376F60F1388F6F91378F80F63E60801C7
:106D500081161396860161869376F70F1388F6F9EC
:106D60001378F80F63E60801138706FE6207618750
:106D70006316C7008507C207C18345BF01458280EE
:106D8000011122CC2A842E8526CA4AC84EC606CEB8
:106D90002E8997800100E780403593140501C1805A
:106DA0009309D0038307040099E301450DA0CA8528
:106DB000228597000000E78040F70DC1B3079400DB
:106DC00083870700639C3701138514002295F240E6
:106DD0006244D2444249B249056182800504D9B770
:106DE00097F7FF1FA38A07B297F7FF1F238607C8ED
:106DF00097F7FF1F238207B297F7FF1F239A07B069
:106E000097F7FF1F238707B097F7FF1F23A407B04B
:106E10008280011106CE22CC26CA4AC84EC69720CF
:106E20000000E78040D905E197F7FF1F238307AEF5
:106E300097F7FF1F23A007AEF2406244D2444249B5
:106E4000B2490561828097000000E78040DD6DF562
:106E500097F4FF1F938484AC130940078D4997F67C
:106E6000FF1F83C666ABE9DA17F7FF1F0347D7AAF0
:106E7000B30727033384F40003552400835504002B
:106E8000636FB500050733773703FD1697F7FF1FCC
:106E90002384D7A897F7FF1FA380E7A8C9B7898DD8
:106EA00091073E95C205C181269597200000E78095
:106EB00080DA59D1835724003E952311A40045B7A9
:106EC0006307054863850548717156CBC16A26D3AF
:106ED0004AD14ECF52CD5AC95EC762C506D722D518
:106EE00066C36AC12E8AAA890149B54B17FBFF1FE9
:106EF000130B0B9DF91A97D4FF1F9384E43917BC29
:106F00000100130CECB593170901C18363E047033B
:106F1000BA502A549A540A59FA496A4ADA4A4A4BE8
:106F2000BA4B2A4C9A4C0A4D4D618280B387290195
:106F3000038707006307770DA94697F7FF1F83D7DD
:106F4000279D6313D73AD5CFDA9717F5FF1F13059F
:106F500025972380070097000000E780C0CA97B5F7
:106F600001009385A5A12A8497000000E780E0DB5B
:106F700049C51305640097000000E780C0C82A8453
:106F800097000000E78080C497B501009385859F36
:106F9000228597000000E78040D915CD83072400A3
:106FA00013F7F7FD01C725476397E702130880022F
:106FB0008147114797B601009386069D17B60100D9
:106FC0001306469D930500080A8597800100E78017
:106FD000A0020A8539A897B501009385259E2285D0
:106FE00097000000E78060D419CD17B501001305A4
:106FF000659D97000000E780E0C597F7FF1F239984
:107000000790050909B797B50100938565A022850A
:1070100097000000E78060D179C58307340013072B
:1070200000026385E7002547639FE70A13053400E4
:1070300097000000E78020BD97B501009385859DEE
:107040002A8497000000E78040CE0DC1930780029C
:107050000147914617B601001306069C93050008E8
:107060000A8597800100E78020F9A5B797B5010050
:107070009385059C228597000000E78000CB0DC515
:1070800017E7FF1F0347077397F6FF1F83D6E682B4
:1070900017B601001306469A930500080A859780E3
:1070A0000100E78060F535B797B501009385059B32
:1070B000228597000000E78040C70DC18147414706
:1070C000B386970083C60600639E06228507E39970
:1070D000E7FE17B501001305E5AD21BF17B50100A7
:1070E0001305859839B797B501009385E5992285F1
:1070F00097000000E78060C36303051E8307340028
:10710000130700026385E7002547639AE71C130510
:10711000340097000000E78000AF97B50100938529
:10712000E5962A8497000000E78020C02DC19305D2
:10713000D003228597800100E78060F811C983069B
:1071400015000547938706FD93F7F70F6377F70060
:1071500017B501001305059469BD93071003639FDC
:10716000F60097E7FF1F2386E77A97000000E78085
:10717000E0A517B5010013056594A5BD97E7FF1FAE
:107180002389077897E7FF1F23A60778DDB797B510
:1071900001009385A58C228597000000E780E0B868
:1071A00031C99305D003228597800100E78020F143
:1071B00011E517B501001305E59125BD8A85050583
:1071C00097000000E78060AF6DD5B7E70400FC478B
:1071D00041468A8526858297268597F0FFFFE780BE
:1071E000202F97F0FFFFE780801C17B501001305E3
:1071F000A59001B597B501009385858322859700F9
:107200000000E78080B279C597B5010093850590AD
:10721000228597000000E780E0B62A8D97B501002F
:107220009385C583228597000000E780A0B5AA8CCE
:1072300063080D046A8502C097000000E780A09CE7
:1072400001468A852A8D97800100E780C001824728
:107250002A846307FD029307F5FF63E3FA0263964E
:107260000C0281474147B386970083C60600B1E60A
:107270008507E39AE7FE17B501001305659595BBF1
:1072800017B5010013050589ADB38A85668597009A
:107290000000E78080A211E517B501001305C5893C
:1072A00089BBB7E70400FC47268541468A8582975B
:1072B000268597F0FFFFE780A02113150401418187
:1072C000A68597D0FFFFE780E07A17B50100130588
:1072D000E58805B317B501001305C58919BB17B5B6
:1072E00001001305258B31B3938617001306F004B4
:1072F000E365D6D0DA9717E6FF1F231BD6602380FD
:10730000E70001B397B501009385C58B0A85978087
:107310000100E78060DC814C1304B100414DB3876C
:10732000940103C607002285E285850C9780010041
:10733000E78000D40904E394ACFF97A5010093858E
:1073400065E6228597800100E78000D959B18280E7
:10735000E5CD854763FAC70E83C7150003C705004F
:10736000A207D98F13978700A183D98FC2073167EE
:10737000C1831307C7556399E70C97E7FF1F83D7AE
:10738000C7536383A70C797122D426D206D64AD07C
:107390004ECE3284AE842AC697000000E780208853
:1073A00035ED93070007B24563E1870817E7FF1F34
:1073B00003478756894763EAE70697E9FF1F83C9B2
:1073C000A96B93074007B389F902B7E70400FC47AC
:1073D00017E9FF1F130989542286A68513854900E2
:1073E0004A95829797E7FF1F83C707690D4785076F
:1073F000B3F7E7024E99231089002311090017E71C
:10740000FF1F230BF76697E7FF1F9387E75083C79C
:107410000700850717E7FF1F2300F750B2502254DB
:1074200092540259F2494561828022862254B25018
:1074300092540259F24917A501001305A57B456135
:1074400017830100670023A28280011106CE22CC9F
:1074500026CA01C5D54763EFB70017A5010013057C
:10746000657B97800100E780E0B7F2406244D24438
:1074700005618280034705009307500A2A84631838
:10748000F700034715009307A0056307F70017A54A
:1074900001001305A579F1B7034735009307100ADA
:1074A000630EF70059476386E5000347450063050F
:1074B000F70217A501001305A57865B7D1449147D8
:1074C000D1465D476393D400594763FAE50017A599
:1074D00001001305657871B7D5449547D5B737E7EF
:1074E00004007847B305F4000A85414602972694C4
:1074F00083471400034504008A85A2075D8D97D059
:10750000FFFFE780205795B741110D658D4506C6F1
:1075100097C0FFFFE780A08FB71700408D6623A6B6
:10752000D70A17E5FF1F130565551387C70A938709
:10753000870A1CC15CC5856689675CC958C114C5CA
:1075400018C9B7E70400B24003A3871E41010283B4
:1075500097E7FF1F83C7075489E7171300006700E9
:107560006366828097E7FF1F83C7D75299EF411167
:1075700006C697100000E780E05BB240854717E73A
:10758000FF1FA309F750410182808280411126C26A
:10759000AE848D4522C406C62A8497C0FFFFE780CB
:1075A0006091B717004099C803A5C70C418D23A669
:1075B000A70CB240224492444101828003A5870C6B
:1075C000418D23A4A70CF5B7834705000347150099
:1075D000A207D98FC2076177C18713072720639A53
:1075E000E700834525003705040017030000670006
:1075F00023FA828017E6FF1F1306064A8147B286E8
:107600001303F00FA9483308F6000348080013F7E6
:10761000F70F6307A80C630668008507E39517FF5B
:107620002947B387E6002380A70097E7FF1F9387CA
:1076300067475DA8411113D765001347170006C6B9
:1076400093F63500058B954791CA054699476387A0
:10765000C60009469D476383C600A14713F645004F
:107660003336C00093F68503050685C2A145638BBA
:10767000B604E145638AB604930580026388B604C4
:10768000930580036393B600914697E5FF1F23801F
:10769000F56897E5FF1F238BC56697E5FF1FA38756
:1076A000D566BE8517A501001305055F977001001B
:1076B000E780607BB240854717E7FF1FA309F764A7
:1076C000410182808546D1B78946C1B78D4675BFD5
:1076D00017A501001305C55E177301006700A378A5
:1076E00017E7FF1F1307073CBA972380B700E1474E
:1076F000E302F5F493077002E30CF5FC82802A871D
:1077000023800500814717E5FF1F1305E53813089F
:10771000F00F2946B306F50083C606006396E6021D
:1077200097E6FF1F93860638B69783C7070005457F
:107730002380F5009947636EF7029D4763FDE700DC
:10774000E147630DF7008280638506018507E393B7
:10775000C7FC0145C5B7238005008280B7370040CC
:1077600003C7370083C7050093F70704D98F238029
:10777000F5008280797126D24AD097E4FF1F83C436
:10778000E46A17E9FF1F1309A96906D622D44ECE71
:1077900052CC56CA5AC8B307990083C7070093F75B
:1077A000F70FA5C79387140093F7F70F0D47636191
:1077B000F70C17E7FF1F230BF76697E7FF1F938769
:1077C000A766A69783C707001307100293F7F7036E
:1077D0006389E7226363F70A054463808720E382B5
:1077E000076809476389E71413070002E387E75234
:1077F000B7E700E03707400023A0E71801000100C9
:10780000CA942380040023A0E710B787004003C771
:107810006700058BE308077297E6FF1F83C62661A2
:107820000547E393E67029472381E702094723834D
:10783000E7022385E70297E7FF1FA38B074C97E733
:10784000FF1FA386075EB7870040A381070017E7E5
:10785000FF1FA301074C05472383E700B2502254C2
:1078600092540259F249624AD24A424B456182809F
:1078700097E7FF1F238C075A89B7130730026386E7
:10788000E70A63E6E71413074002638AE708130771
:107890000003E39FE7F497E7FF1F9387A758A69796
:1078A00003C70700A1471377F70FE313F71617EA8B
:1078B000FF1F130AEA1F83476A0097E6FF1F238F03
:1078C000F64297E7FF1F83C7171F91C7FD5797E63B
:1078D000FF1F2385F64297E5FF1F83C5751D97E7B8
:1078E000FF1FA38DB74097E7FF1F83C7671C93F95E
:1078F00007089306000493F70706639DD74A93078A
:10790000A0096387F51463E4B7109307F005638457
:10791000F548930750096382F52801440DABFD57E4
:1079200017E7FF1F230BF73CE1B5FD5717E7FF1FD4
:107930002304F73C75BD17A501001305E5499770B1
:107940000100E780206A97E7FF1F9387A74DA6975E
:1079500003C40700814917EAFF1F130AEA2D1374B5
:10796000F40F97AA0100938AAA4763C7890429459F
:1079700097700100E7800054854717E7FF1FA30BAE
:10798000F72A17E7FF1F2308872A17E7FF1F23019E
:10799000F73837E700E0B70640002320D71801008A
:1079A0000100378600408347A60293F7370F23056F
:1079B000F6022320D7102DBDB3073A0183C5070077
:1079C0005685850997700100E780E04979BF8547B2
:1079D00017E7FF1F2300F72621BD17E7FF1F130737
:1079E000674426970347070097E6FF1FA382F61810
:1079F00097E6FF1F238FE61617E7FF1F230AF730CE
:107A0000C5BB854717E7FF1F2304F716D5B39307B8
:107A1000400A638DF5349307200B6388F53693078E
:107A2000100AE39CF5EE83072A00014463D1074264
:107A300097E7FF1F83C7F70793F63700638E061A91
:107A40000546638EC62209466399C61A1D4775A26C
:107A500017E5FF1F0345E505C94717EAFF1F034A5E
:107A60005A0597E5FF1F83C5E50417E4FF1F03448C
:107A700074046319F510CD476316FA109307700864
:107A8000639CF5021307300FB7170E006308E4007C
:107A90001307900DB7B704006314E40817E7FF1F3E
:107AA0002324F726BE8517A501001305E53397703B
:107AB0000100E780403B95B593078008639DF50082
:107AC00033048040B77746001374F40F938787CD53
:107AD000B3D78702E1B793079008639AF5003304A0
:107AE000804091671374F40F9387C766D5B79307E7
:107AF000A008639BF50033048040B7173D00137462
:107B0000F40F93870790E9B79307B008639AF500DD
:107B10003304804091671374F40F938797D04DBF5F
:107B200093F5F5078D47639BF50033048040B797C5
:107B30005B001374F40F938707D859BF8947639B81
:107B4000F50033048040B7770B001374F40F93876C
:107B5000071BBDBF8547639AF50033048040DD678E
:107B60001374F40F938767E3A5B789E93304804062
:107B70008D671374F40F938777DC99BFF167938750
:107B8000072029BF97000000E78000A7A285528543
:107B900097000000E78040A649B39305610017E510
:107BA000FF1F034505F117E4FF1F034494F09700FE
:107BB0000000E78000B59305710022859700000062
:107BC000E78020B43C0017E7FF1F2329F7248347F1
:107BD00061002304F10083477100A304F100894789
:107BE00017E7FF1F230CF7108357810017E7FF1FCC
:107BF0002310F7EC0944A1AC154793F64700B336C0
:107C0000D00093F78703850685C32146638BC7069B
:107C10006146638AC706130680026388C706130697
:107C200080036393C700914717E6FF1F2300D60E1A
:107C300097E6FF1FA38CF60C97E7FF1F2389E70C3D
:107C400017E7FF1F034707E79376070497E7FF1F30
:107C500083C757E68DEE1377770C93067008630C95
:107C6000D7021377F7078D46631ED70AB307F04094
:107C7000B7955B0093F7F70F938505D881A819474F
:107C8000ADBF854755B7894745B78D4771BF930647
:107C900070086311D7021307300FB7150E00638900
:107CA000E7021307900DB7B504006383E7021307DB
:107CB000700845BF9306800C6311D702B307F040EC
:107CC000B775460093F7F70F938585CDB3D5F502C9
:107CD00097E7FF1F23AAB702F9B39306900C631A24
:107CE000D700B307F040916593F7F70F9385C5660A
:107CF000F1BF9306A00C631BD700B307F040B71584
:107D00003D0093F7F70F93850590C9B79306B00C24
:107D1000E319D7F4B307F040916593F7F70F938514
:107D200095D06DB78946631BD700B307F040B77590
:107D30000B0093F7F70F9385051B49BF8546631A20
:107D4000D700B307F040DD6593F7F70F938565E340
:107D5000B5BF09EBB307F0408D6593F7F70F938537
:107D600075DCADB7F165938505209DB783472A0083
:107D7000C18B99C7854717E7FF1F2304F7F871BE2A
:107D800097E7FF1F238F07F649BE854717E7FF1FB9
:107D9000A30FF7F659B63C0017E7FF1F2320F7089B
:107DA0000947930700032314F10097E6FF1F238779
:107DB000E6F42DBD63990758A94763EBB74417A7AD
:107DC00001001307A7EA8A05BA959C41BA978287F2
:107DD00017E4FF1F0344F4CD094A630C440F636C9E
:107DE0008A0885476309F40A9307F00F17E7FF1F16
:107DF0000347C7F063F6E70017E7FF1F2300F7F01C
:107E000017EAFF1F034A8AEF930700041374FA0F5F
:107E100063F447011304000497E7FF1F93870700EB
:107E200083AA0700228617E5FF1F130565C8D685BC
:107E3000330A8A40A29A97700100E78060F797E7BB
:107E4000FF1F238D47EB97E7FF1F23A957FD97E7F8
:107E5000FF1F83C7B7EA15476399E762B7E700E0FA
:107E60003707400023A0E71801000100B786004053
:107E70002380860285A58D47630CF40A9947E31594
:107E8000F4F697A701009387E7E417E7FF1F23277E
:107E9000F7F8A947A1BF17E7FF1F034747F997E77F
:107EA000FF1F9387A7E7494697A50100938585EBB8
:107EB0006306870097A501009385C5E63E85977008
:107EC0000100E780E0EE17E7FF1F2329A7F4C94769
:107ED00031BF97E6FF1F83C686F5054797E7FF1F6B
:107EE0009387C7E36394E6023E851306700297A565
:107EF00001009385A5E497700100E78060EB17E728
:107F0000FF1F232DA7F093077002CDB53E85130602
:107F1000300497A501009385A5DC97700100E780E8
:107F200020E917E7FF1F232BA7EE930730047DBD41
:107F300097E5FF1F83C5E5B717A50100130505ECFD
:107F400097700100E78020F2854A17EBFF1F034B73
:107F50000BEE97E5FF1F83C5C5B517A501001305F7
:107F6000E5E963185B0B97700100E780C0EF97E7C6
:107F7000FF1F83C707B4B5CBE368F4E617A401007D
:107F8000130484E2638C670117A40100130444E224
:107F90006386470117A40100130404E32285977048
:107FA0000100E78080141375F50F9307150086070D
:107FB00017E7FF1F2304F7D68D4717E7FF1FA30F0F
:107FC000F7D497E7FF1F938767D50147BE861376DF
:107FD000F70F89076365A60297E7FF1F23A0D7E481
:107FE00097E7FF1F83C787D311B597A70100938732
:107FF000A7D417E7FF1F2323F7E29147C5BB33063A
:10800000E40003460600A380070005072380C7009D
:108010007DBF97700100E78000E597E7FF1F83C7EA
:1080200047A9E1D7E362F4DC17A401001304C4D428
:10803000638C570117A40100130484D4638647019D
:1080400017A40100130444D5228597700100E7802E
:10805000C0091375F50F93071500860717E7FF1F73
:10806000230EF7CA8D4717E7FF1FA309F7CA97E743
:10807000FF1F9387A7CA0147BE861376F70F8907AC
:10808000E37CA6F43306E40003460600A380070061
:1080900005072380C700D5B797E5FF1F83C565A1F6
:1080A00017A50100130545D697700100E780A0DBF6
:1080B00097E7FF1F83C757C693E7470017E7FF1FE0
:1080C000A30CF7C483472A0017E7FF1FA304F7C4D4
:1080D000A9B017A50100130565D497700100E780CA
:1080E00060F097E7FF1F9387E7C283C7070017E792
:1080F000FF1F230FF79A17E4FF1F034424C03334F4
:108100008000B1B317A50100130585D29770010057
:10811000E78040ED97E7FF1F83C717C093E707018C
:1081200017E7FF1FA30AF7BE83472A0017E7FF1FC1
:108130002302F7BE6FF06FFE17A50100130585D06F
:1081400097700100E78000EA03470A007D8B51EF3A
:10815000B787004003C767021377C70B1367270071
:108160002383E70203C7A7021377C70B1367270010
:108170002385E70203C7E7021377C70B13672700BE
:108180002387E70203C727031377C70B136727006B
:108190002389E702854717E7FF1F230BF79C17E7A3
:1081A000FF1F2309F7A817E7FF1F2307F7B417E7F7
:1081B000FF1F2304F7B497E7FF1FA38B079A97E7E6
:1081C000FF1FA38907A697E7FF1FA38707B297E7BB
:1081D000FF1FA38407B297E7FF1FA38B07B297E7A0
:1081E000FF1FA38607C46FF04FF389476312F7029E
:1081F00097E7FF1F83C7078C9146638CD70863E01E
:10820000F604638EE70C6369F70A05476380E70E9F
:10821000FD5717E7FF1FA303F7AE37074000B7E787
:1082200000E023A0E71801000100B7860040130614
:10823000F0FC2381C60223A0E7106FF06FDB130769
:1082400020086382E7086362F70213071008E391CE
:10825000E7FC378700408347670293F7C70B93E734
:1082600027002303F7026FF04FEB130730086389F1
:10827000E70213074008E39DE7F83787004083478C
:10828000270393F7C70B93E727002309F7026FF043
:10829000CFE8378700408347270393F73707F5B7C1
:1082A000378700408347E70293F7C70B93E7270020
:1082B0002307F7026FF06FE6378700408347E70236
:1082C00093F73707F5B7378700408347A70293F73F
:1082D000C70B93E727002305F7026FF00FE43787FA
:1082E00000408347A70293F73707F5B73787004069
:1082F0008347670293F73707ADB717A5010013054A
:1083000065B597700100E780E0CD97D7FF1F238107
:10831000077AD5B317A501001305C5B497700100FE
:10832000E78040CC97D7FF1F2394077897E7FF1F7C
:108330009387C79C03C40700894763F387000944F8
:108340001374F40F29B613070002E393E7EC639963
:10835000090A638FF500930720026381F50817A5CA
:1083600001001305A5B397700100E780C0AF4DB5BC
:1083700017A501001305C5AF97700100E78080C6FF
:10838000014417AB0100130BEBAFA14AB3078A00FE
:1083900083C507005A85050497700100E780A0ACEB
:1083A000E31654FF179501001305C5E5977001000A
:1083B000E78040C317D4FF1F0344C46F11E497D76D
:1083C000FF1FA38A076C61B48947E313F4E4854770
:1083D00017D7FF1FA301F76C6FF02FD417D6FF1F1D
:1083E0000346366D97D5FF1F83C5A56C17A5010001
:1083F0001305C5A997700100E780E0A66FF0EFD1E3
:10840000638FF50493071002E39BF5F497D5FF1FE4
:1084100083C5456A17A50100130545A9977001009A
:10842000E78060A497E7FF1F23AA479F97E7FF1FF6
:108430009387878D944383D7470017E7FF1F034730
:10844000078D17D6FF1F2325D6661D4497D6FF1F1D
:108450002392F66697D7FF1F238FE764CDBA97D58F
:10846000FF1F83C5256517A501001305A5A59770F6
:108470000100E780409F97D7FF1FA38E076097D723
:10848000FF1F239707626FF0EFF62547E388E79C0D
:1084900019476391E702B786004023808602B7E759
:1084A00000E03707400023A0E71801000100130691
:1084B00000FC41B31307100A6391E702B78600403E
:1084C00023808602B7E700E03707400023A0E718C3
:1084D00001000100130680FCA9BB1307A009E38F6C
:1084E000E7FC1307400AE38BE7FC13072002E3874E
:1084F000E7960547E384E796B7E700E037074000D3
:1085000023A0E718E392099601000100B786004016
:1085100023808602130620FC29BB17D7FF1F0347C1
:10852000F77D6308F71E63E7E7029547630EF70ED2
:1085300099476308F704B786004023800602B7E72F
:1085400000E03707400023A0E718010001001306F0
:10855000A0FCC5B19307F005630AF7009307500923
:108560006306F70093071002E317F7FCB7E700E094
:108570003707400023A0E71801000100B78600403C
:1085800051BF97D9FF1F83C9697793070004CE8A2B
:1085900063F43701930A000497E7FF1F9387078866
:1085A00003AA070013F4FA0F2286D28517D5FF1FFE
:1085B0001305055097600100E780807FB3878940ED
:1085C000529417D7FF1F230BF77297E7FF1F23A7BC
:1085D0008784638E0902B787004023805703B7E67C
:1085E00000E03706400023A0C6180100010003C7C1
:1085F0002702134707042381E70203C727021377E3
:10860000C70F2381E70223A0C6106FF06F9EB786C5
:10861000004023800602B7E700E03707400023A0B0
:10862000E71801000100FDB5378700408347370098
:1086300097D6FF1F83C6166E93F70708D58FA30141
:10864000F700B7064000B7E700E023A0D718010005
:1086500001001306A0FC2301C70223A0D7106FF06E
:108660002F9997D7FF1F9387E77BA69783C70700AC
:1086700093F7F70FD9CF97D7FF1F83C7477BD1EB6E
:1086800017D7FF1F03479767930700026313F70885
:1086900097D7FF1F9387C74103AB070097DAFF1FE8
:1086A00083CA4A4117DAFF1F034ADA4097D9FF1FEE
:1086B00083C96940D2875687CE865A8697D5FF1FD1
:1086C00083C5753D17A5010013054581976001001D
:1086D000E780607997D7FF1F23A8676397D7FF1FAD
:1086E0002386576397D7FF1FA382476397D7FF1F40
:1086F000238F376197D7FF1F238F8738B7E700E0B5
:108700003707400023A0E71801000100B7860040AA
:10871000D1B3B7E700E03707400023A0E718010016
:108720000100B786004025B529472381E7020947A4
:108730002383E7022385E7022387E7022389E702F1
:108740006FF06F8F03C76700118B6309079083C7B2
:108750005700918BB5CF17D7FF1F0347476D85474C
:108760006313F70697D7FF1FA383E75A97D7FF1F17
:108770002380074097D7FF1F238E074A97D7FF1FF5
:10878000238C075697D7FF1F2389075697D7FF1FBC
:10879000A380073E97D7FF1FA38E074897D7FF1FD9
:1087A000A38C075497D7FF1FA389075497D7FF1FA0
:1087B000A380075697D7FF1FA38B0766B787004094
:1087C00011476FF06F8917D7FF1F2306F72C79BF6A
:1087D000854717D7FF1F230DF73817D7FF1F230B28
:1087E000F74417D7FF1F2309F75017D7FF1F23069A
:1087F000F75069BF854717D7FF1F230BF73617D7E9
:10880000FF1F2309F74217D7FF1F2307F74E17D77C
:10881000FF1F2304F74E17D7FF1FA30B073417D7EB
:10882000FF1FA309074017D7FF1FA307074C97D7C0
:10883000FF1FA384074C8280411106C697000000E9
:10884000E78080FBB787004023800700130740FCC8
:108850002386E7001307C004A386E70017D7FF1F8E
:10886000130707252398E70017D7FF1F130747288B
:10887000239AE70017D7FF1F1307C733239CE7008E
:1088800017D7FF1F1307473F239EE7002947238180
:10889000E70209472383E7022385E7022387E702EC
:1088A0002389E702A3810700130700F8A380E700EC
:1088B000130790022380E700B716004003D7A601F4
:1088C0001367070C239DE6007D572383E7000D47C0
:1088D0002381E700B706400037E700E02320D710E8
:1088E00003C7170013671700A380E700B24097D7AC
:1088F000FF1F2391074241018280411106C6970064
:108900000000E78060EFB78700402380070013076F
:1089100000FC2386E7003147A386E70017D7FF1F37
:10892000130707192398E70017D7FF1F1307471CE2
:10893000239AE70017D7FF1F1307C727239CE700D9
:1089400029472381E70209472383E7022385E702BA
:10895000A3810700130700F8A380E7001307900224
:108960002380E700B716004003D7A6011367070C62
:10897000239DE6007D572383E7000D472381E70011
:10898000B706400037E700E02320D71003C71700E1
:1089900013671700A380E700B24097D7FF1F239B00
:1089A000073641018280F1679387072017D7FF1FA1
:1089B000232CF734854717D7FF1F2319F734A14716
:1089C00017D7FF1F2305F73497D7FF1FA38107345D
:1089D00097D7FF1F238E073297D7FF1FA38D070A54
:1089E00097D7FF1F2389070A814717D5FF1F130554
:1089F000A50AFD5517D6FF1F1306C60A2947B30659
:108A0000F5002380B600B306F60023800600850734
:108A1000E397E7FE97D7FF1F2384074097D7FF1FF1
:108A2000A380074097D7FF1F238D073E97D7FF1FCF
:108A3000A387072C97D7FF1FA385072C97D7FF1F66
:108A40002380072C97D7FF1F238B072A97D7FF1F59
:108A5000238A072A97D7FF1FA384072A97D7FF1FC8
:108A60002381072A97D7FF1FA38D073A828017D744
:108A7000FF1F0347C73B85476316F7001703000036
:108A80006700E3E717030000670043DB411122C4DE
:108A900006C617D7FF1F0347873985472E8613F46D
:108AA000F50FAA856317F70417D5FF1F1305851463
:108AB00097600100E780C02F97D7FF1F238C071610
:108AC000B787004023848702B7E600E037064000FE
:108AD00023A0C6180100010003C7A7021377C70F20
:108AE0002385E702B240224423A0C610014541017C
:108AF000828017D5FF1F1305A50397600100E7804B
:108B0000202B97D7FF1F23850706B78700402382B6
:108B10008702B7E600E03706400023A0C618010030
:108B2000010003C767021377C70F2383E7025DBF06
:108B3000411106C697000000E78020E7B2404101DE
:108B4000170300006700E3F2411106C697F0FFFF2C
:108B5000E78080C297D7FF1F83C79701A1CB97D526
:108B6000FF1F83C5050189C917D5FF1F13058500A0
:108B700097E0FFFFE780003597D7FF1FA38A07FE26
:108B800097D7FF1F2386071837E700E0B706400096
:108B90002320D71801000100378600408347660272
:108BA00093F7370F2303F6022320D710B240410179
:108BB000828017D5FF1F0345E5153335A00082805D
:108BC00041C9D9C597D7FF1F83C7C714D1C30111A6
:108BD00022CC4AC84EC656C25AC006CE26CA52C475
:108BE0002E89AA890144930A0004371B0300637786
:108BF0002403B3078940C207C183BE8463F4FA002B
:108C000093040004C204C180130A1BD497D7FF1F2A
:108C100083C707F69DE37D1A631C0A00F240624495
:108C2000D2444249B249224A924A024B05618280AB
:108C300097F0FFFFE78040B4D1BF338589002694C9
:108C4000A685420497000000E78080E4418045B794
:108C50008280411106C622C429C12E8495C997D7A6
:108C6000FF1F83C7270B95CB97D7FF1F83C747F0FD
:108C70008DC713070004AE876374B7009307000421
:108C8000139407014180A28597000000E78040E02F
:108C90002285B2402244410182800144D5BF97D74A
:108CA000FF1F9387671C18429C4383D645000345EA
:108CB000070083C5C700035646006396A50083D509
:108CC000E700638DD502011106CE2386A700239706
:108CD000D700B705CF00DC4B9385757D05077D1662
:108CE0002EC2230001003AC42316C1002317D1006D
:108CF00099C30A858297F240056182808280DC4DAB
:108D0000DC4B81CFB7E70400904503A3870591456D
:108D100017D5FF1F03458515028382806D713C08BE
:108D20003EC6B707E500232291103EC8AA843C083E
:108D30003285232611103ECA2324811023202111BD
:108D40002E8997300000E780605C2A8497950100A7
:108D50009385451C17850100130545E297600100C6
:108D6000E7806010A285179501001305252B9760F9
:108D70000100E780400F294597600100E7808013DC
:108D8000B705CB009385757D680097100000E780DC
:108D90008065A285680097300000E7808049014720
:108DA00081467000CA85268597200000E7800089EB
:108DB00005CD2A84979501009385C5151785010077
:108DC0001305C5DB97600100E780E009A2851795D0
:108DD00001001305652597600100E780C00829455B
:108DE00097600100E780000D8320C11003248110EB
:108DF00083244110032901105161828097D7FF1FFE
:108E00009387870618429C43797122D406D603487B
:108E1000070083C807012A8483D64500035546000E
:108E20006396080183D82701638DD8022388070140
:108E300005072399D7003708CC00DC4B1308787D51
:108E40003ACC1307F5FF42CA23080100231EE100B4
:108E5000231FD10099C7080832C62EC48297324614
:108E6000A245228597000000E78080EBB250225493
:108E7000456182806D713C083EC0B707E5003EC287
:108E80003C083EC423261110232481102322911074
:108E9000231701002318010023190100231A0100E0
:108EA000231B010097A7FF1F83D7475799E3C1678B
:108EB000FD172316F10097A7FF1F83D7475691EBA5
:108EC00097D7FF1F938747FA9C439C43DC4783D780
:108ED000070017A4FF1F13046454584C2317F10014
:108EE00083574400484B2318F10031E19795010066
:108EF0009385450917850100130545C89760010052
:108F0000E78060F6179501001305050997600100D9
:108F1000E78060F5294597600100E780A0F983208C
:108F2000C11003248110832441105161828097A7CE
:108F3000FF1F83C7174F89EBB7E70400BC57829721
:108F40005C4C23AA0700E1BFFD1797A6FF1FA38A69
:108F5000F64C03560701834704014C470A85230B4F
:108F6000F10097300000E780E02997D7FF1F938733
:108F7000A7EF9C430147814688430A866C009710FF
:108F80000000E780A06BAA8429C197950100938512
:108F900065FF17850100130565BE97600100E78036
:108FA00080ECA685179501001305C5FF97600100A9
:108FB000E78060EB294597600100E780A0EF584CFF
:108FC000B7E70400BC57484B9DBF97A7FF1F83C757
:108FD0005745F5D7B7E70400BC4F1044854517D572
:108FE000FF1F0345A5E882971DBF5C4EDC4BB9CF40
:108FF000B1CD411122C417850100130525B82E8477
:1090000097950100938545F606C697600100E780B5
:1090100080E5A28517950100130585FB9760010087
:10902000E78060E4294597600100E780A0E8B7E7A2
:1090300004002244B24003A3870517D5FF1F034550
:10904000E5E2130640069145410102838280411109
:1090500022C417A4FF1F1304243A1C4C06C689C758
:10906000DC4399C34C488297584CB7E70400BC577F
:10907000484B82975C4CB240224423AA070041012E
:10908000828017A7FF1F130727398347070093061E
:10909000F00B850793F7F70F63E9F60097A6FF1F1C
:1090A000238CF636034507008280930700F8FDB74E
:1090B000835745006386071001114AC817A9FF1F8F
:1090C0001309C93552C4032AC90106CE22CC03278D
:1090D0004A0126CA4EC656C2F15735E31307D00DD2
:1090E000FD57636EC704B7E9040083A709072A8404
:1090F0001305860042054181B284AE8A8297232AF5
:10910000AA000325C9015C49A9E797950100938549
:10911000A5E317850100130565A697600100E780A8
:1091200080D4179501001305E5F297600100E780F0
:1091300080D3294597600100E780C0D7DD57F24012
:109140006244D2444249B249224A924A3E8505616C
:10915000828093874400B705CF002319F5009385DB
:10916000757D310597100000E780E0270325C901D0
:1091700083456400310597300000E780800B0325AC
:10918000C9012686D685310597300000E780800723
:109190007146A2854A8597600100E78060C150440E
:1091A00019CA83A78905854517D5FF1F034505CC37
:1091B0008297814769B797000000E780E0CBD5BF71
:1091C000FD573E858280411126C297A4FF1F9384DC
:1091D000E424D84C22C437E404003C54484B06C66F
:1091E0008297DC4C0323C4052244B240924423AA54
:1091F000070017D5FF1F034565C785454101028359
:10920000411126C297D4FF1F938404C69C4006C612
:1092100022C44AC0D5C3DC43C5C35CC12300B5002A
:109220002A8497950100938565CD17850100130564
:10923000E59497600100E78000C32945976001002D
:10924000E78040C79C4023A4070023A2070097A7FC
:10925000FF1F9387671ADC4FDC4B91C72955970096
:109260000000E78000DF97A7FF1F9387271BDC4FD5
:10927000DC4B89C797000000E78020F537E9040040
:109280008327C905894517D5FF1F034525BE82974A
:109290008327C905914517D5FF1F034525BD829733
:1092A0009C4003A347016309030022852244B24086
:1092B0009244024941010283B2402244924402494D
:1092C000410182800111328506CE22CC26CA2E842D
:1092D00097300000E7808003AA849795010093856A
:1092E00025C5178501001305658997600100E78092
:1092F00080B7030784000356640083554400A686A4
:10930000179501001305C5CE97600100E780A0B551
:10931000294597600100E780E0B997A7FF1F83C741
:10932000070E639D9700014597000000E78060D21B
:1093300081450A8597000000E780C0ECF240624456
:10934000D244056182806D7123248110232611107F
:109350002322911093F745002E84638707143C085D
:109360003EC0B707E5003EC23C083EC423170100DB
:109370002318010023190100231A0100231B0100F7
:1093800097A7FF1F83D7470799E3C167FD172316E8
:10939000F10097A7FF1F83D7470691EB97D7FF1FD1
:1093A000938787AC9C439C43DC4783D7070017A770
:1093B000FF1F130767042317F100544F835747001B
:1093C0002318F100DC4AA1E797950100938585BA3F
:1093D000177501001305857A97600100E780A0A842
:1093E00017950100130545BB97600100E780A0A712
:1093F000294597600100E780E0AB134544008320D6
:10940000C11003248110832441105161828097A7E9
:10941000FF1F83C7D7FE2555D9C3FD1717A6FF1F0A
:10942000A30FF6FC03D6060183470701CC460A8545
:10943000230BF10097300000E780C0DC97D7FF1FB7
:10944000938787A29C4317A7FF1F1307E7FA9796F6
:109450000100938666B788430A866C009710000067
:10946000E780C01DAA8451D997950100938585B0E6
:10947000177501001305857097600100E780A09EB5
:10948000A685179501001305E5B197600100E780F7
:10949000809D294597600100E780C0A1268597003F
:1094A0000000E78000BB91BF93F725009DC7B7E799
:1094B0000400BC47414681452808829725559700FE
:1094C0000000E78000B928089305F00F970000001E
:1094D000E78040D3134524001DB793F715000145DD
:1094E00099DF97000000E78020991345140001BF21
:1094F0005C4D411106C688C317D7FF1F2326F79678
:10950000B7E7040083A70708170500001305E5E384
:109510008297B24097D7FF1F238AA7940145410144
:10952000828001113335A000A307A100B7E7040032
:1095300083A7471706CE1306F10085451305503063
:109540008297F240056182808280411122C417D443
:10955000FF1F034424931335140006C69700000030
:10956000E78060FC17950100130585BB09E417959A
:1095700001001305E5B92244B2404101176301001F
:109580006700638E797122D4A30F010037E40400D1
:109590008327841726D24AD006D6AA842E8913059B
:1095A00050309305F10132C6829732468347F1016C
:1095B00093150601C18185CB01452EC69700000099
:1095C000E78060F683274417B2454A86268582974E
:1095D000054597000000E78000F5B25022549254F0
:1095E000025945618280832744174A8626858297DF
:1095F000EDB741119397050122C406C626C2C18763
:109600002E8463D40702B7E40400FC5417A5FF1F9F
:109610000345C5E3829719C1BC5482972165218D0A
:10962000B240224492444101828093F715008DC7D5
:10963000B7E7040083A7471A17A6FF1F130606E023
:1096400097D5FF1F9385458317A5FF1F034505E0A9
:10965000829713451400E9B793F7250099CFB7E730
:109660000400BC4F13060064894517A5FF1F03457E
:10967000E5DD82971345240065B793F7850085CF14
:1096800097D7FF1F83C7C78085E7B7E7040003A804
:10969000871A1307401F97A7FF1F83C727DB814641
:1096A00013064006994517C5FF1F0355E57D02982F
:1096B00013458400B5B793F745000145B5D3B7E42A
:1096C000040083A7041817C5FF1F0355E57B829785
:1096D000BC4C13060064914517A5FF1F034505D731
:1096E0008297134544002DBF97C7FF1F83D7C779C3
:1096F0006398A70217C7FF1F2319B77817C7FF1F63
:109700002316C77817C7FF1F2313D7782E86179500
:109710000100130525A6BE85175301006700A37439
:1097200017950100130585A6176301006700838B59
:109730000357450097C7FF1F83D70775631EF704BC
:10974000C1674111F91722C417C7FF1F232EF772F3
:1097500037E4040097C7FF1F23AA077297C7FF1FAC
:10976000A382077297C7FF1F238407727C4C06C62B
:10977000894517A5FF1F034565CD82977C4C914510
:1097800017A5FF1F034585CC82972244B2404101B3
:10979000170300006700A3DB179501001305059F61
:1097A00017630100670003847D15954763E2A71CDA
:1097B00017970100130787930A053A951C41011179
:1097C00022CC06CEBA972E84828717950100130506
:1097D000659C97600100E780E080A1A203C7250097
:1097E00099476311F7022E8597000000E78080F407
:1097F00083456400179501001305C59A9750010031
:10980000E780606697B7FF1F238407BA17950100AA
:109810001305059B7DBF03C7250095476319F70214
:10982000C16717C7FF1F03572766F91703D5A500A0
:109830006309F702B7E7040083A7C7178297179554
:1098400001001305E59897500100E780A07985474E
:1098500017B7FF1F230EF7B4179501001305C5991D
:109860008DBF97C7FF1F2391A76283D7E50097C6D7
:10987000FF1F239CF66083D7050197C6FF1F239720
:10988000F66083D7250197C6FF1F2392F66097C71E
:10989000FF1FA389075E631BE502B7E70400BC4F07
:1098A000096613060690A14517A5FF1F034505BAD3
:1098B00082970356E4008355A40017950100130511
:1098C000659297500100E780005A51B79307700FD7
:1098D0002316F100B7E7040083A7870D17A6FF1F23
:1098E0000346C6B66C0082974DF9854717C7FF1F20
:1098F000A30AF7585DB7179501001305A590D1BDD0
:1099000083C5250091476392F50217950100130561
:10991000E59097500100E780E06C97000000E78039
:1099200000C3F24062440561828099476392F50268
:10993000228597000000E780E0DF834564001795EB
:1099400001001305258697500100E780C051D1BF63
:109950009547639AF50083471400E1F317950100DA
:109960001305058EBDB5179501001305E58DE1BF03
:109970008280411122C417A4FF1F130464AEAA867B
:1099800017860100130606782285C14506C6975042
:109990000100E78060660357440097A7FF1F938785
:1099A00027AD2393E700035764002394E700B240F8
:1099B000224441018280411106C697000000E780E1
:1099C00080FBB7E7040083A7871417A6FF1F1306C1
:1099D00026A9D54501458297B2404D4697A5FF1F60
:1099E000938505A913057030410117030000670036
:1099F000A3B961712324811A37E404008327040882
:109A00002326111A2322911A2320211B232E3119D8
:109A100017050000130525BE829717A9FF1F13091C
:109A2000E9A2994785442300A900231CF1009785EA
:109A300001009385257193074006177501001305F2
:109A4000E513231CF1082308910097C9FF1F938990
:109A5000C9E697500100E780004183D509001785CA
:109A600001001305256D97500100E780C03F29458F
:109A700097500100E780004403D5090089699700E9
:109A80000000E78040EF8327441710088545130541
:109A9000503082978327441717A6FF1F1306469D51
:109AA000CD451305703082978327441717A6FF1FF3
:109AB0001306069AB545130560308297832744172D
:109AC00030088945130510318297832744173009E0
:109AD0008945130520318297832744159385099082
:109AE0000D458297832744159385099011458297E8
:109AF000A3059100230691002308910002CD230CB9
:109B00000100832784163009914513057040829720
:109B1000832784161306B1008545130500408297FC
:109B2000832784167000854513051040829783278C
:109B300084163008854513052040829783278416B4
:109B400010088545130550408297832704157D55DD
:109B50008297832744137D5582977D5597A0FFFFF9
:109B6000E780E0B48327440C829797A0FFFFE7804B
:109B700040908327841417A6FF1F1306668ED545D1
:109B80000145829789471306700F814528092306EE
:109B9000F1009780FFFFE780C0598D47130600084A
:109BA00081452808230CF1089780FFFFE780605863
:109BB0009147230CF100977701009387A7ED984315
:109BC00083C747003AC8230AF10097C0FFFFE78028
:109BD000007E70008545054597A0FFFFE78040B4F3
:109BE00030099305700F094597A0FFFFE78040B348
:109BF0003008930500080D4597A0FFFFE78040B2AD
:109C000010089545114597A0FFFFE78060B1C16737
:109C100017C7FF1F13074727F9171CC32322070085
:109C200017A5FF1F1305458297A0FFFFE78020AE11
:109C30008327C41D17C5FF1F1305852382973C4842
:109C400003450900854582978320C11A0324811AA0
:109C50008324411A0329011A8329C1195D61828075
:109C6000C16717C8FF1F03582822F9176301F808B6
:109C70003DCDB5CD011126CAB7E4040083A78412F7
:109C800022CC2E862315B10006CE2A8401478146B8
:109C9000ED45428582972AC611ED1785010013050F
:109CA000654B97500100E780E033F2406244D244B4
:109CB00005618280FC440356A100A28582972C0096
:109CC00017C5FF1F0355451C97A0FFFFE780E0B0B5
:109CD00069DD178501001305254997500100E780CC
:109CE000603083A7C412ED45280082977DBF828033
:109CF000411106C61DC985471797FF1FA30FF774AB
:109D000035469795FF1F9385A57413056030979787
:109D1000FF1F2385077497000000E780E086B240AC
:109D2000410117030000670083829797FF1FA386F6
:109D30000772F9B797C7FF1F83C78715A9EFC167D8
:109D400017C7FF1F03574714F9176306F70441119C
:109D5000854722C417C7FF1F230CF71237E40400FE
:109D60007C4C06C6A1451795FF1F0345256E8297BB
:109D70000323841A2244B2409797FF1F83C7076DBD
:109D800017C5FF1F035545101307401F8146314675
:109D900099454101028382806D712324811023261D
:109DA000111023229110328401CD8947630AF502F4
:109DB0008320C110032481108324411051618280CB
:109DC0001785010013050549AE8497500100E7800F
:109DD0006021A285268597C0FFFFE780E08BC9BF81
:109DE000B7E70400FC472800829717850100130598
:109DF000254797500100E780E01E8347810039C462
:109E00001307000B6380E7021387A7051377F70F8B
:109E10008D4663EDE602A285280097C0FFFFE7802C
:109E2000C0FA79B78547E3F587F883459100177540
:109E300001001305A50BB335B00097A7FF1F2389B9
:109E4000B73E97500100E78000029DB7034791009D
:109E5000A207D98F35671307D7556385E70863686D
:109E6000F7022D671307B7556387E70631671307B6
:109E7000C755638AE70429671307A7556394E70268
:109E8000A285280097C0FFFFE780402315B73967F8
:109E90009306E7656381D70863E9F6001307E75582
:109EA0006384E706A28528003DB73D679306F75512
:109EB000638AD7061307F766E396E7FE97C0FFFFAE
:109EC000E780803DF5B50146A285280097C0FFFFD9
:109ED000E780A01AF1BDA285280097C0FFFFE780A8
:109EE000E019F9B58947E3F587EC97000000E780B2
:109EF000A0E49305E4FFC205C1811305A10097907A
:109F0000FFFFE78020306DB5A285280097C0FFFFD6
:109F1000E780801D71BDA285280097C0FFFFE78004
:109F2000402879B597C0FFFFE780C03051B5C167C1
:109F300017C5FF1F035545F5F9176307F500B7E788
:109F4000040003A3C71702838280854717C7FF1F3A
:109F5000230AF7F2014517F3FFFF6700C35C17837D
:109F6000FFFFE70263182A8408452E89B28919C9C0
:109F700000C1971500009385A58661059730010003
:109F8000E780800181447D5A97100000E780E03926
:109F900063C7A404814497100000E780003A63C8B7
:109FA000A40497C7FF1F9387E7EE9C43DC47B307E2
:109FB000F94091872302F400638309048327C900D1
:109FC000B307F4409587A302F4001C4C89C79C4753
:109FD00099C3228582971783FFFF670023145C448F
:109FE000139714008504BA972390470171BF1C484A
:109FF000139714008504BA972390070069BF83273D
:10A0000089000547B307F4409587A302F4008357FE
:10A010000400638EE7028DC309476384E7040D479C
:10A02000E395E7FA97870100938747761CCC9787DB
:10A0300001009387A77611A8978701009387873C33
:10A040001CCC978701009387E73C5CC8BDBF97870E
:10A050000100938727281CCC9787010093878728C6
:10A06000EDB797870100938727771CCC978701006E
:10A0700093878777D9BF95E51783FFFFE7026308CA
:10A08000004618448347940075839D8B6317F7003F
:10A0900097100000E78060B448C41783FFFF670093
:10A0A000830882801783FFFFE702030413893500CA
:10A0B000C16442094111AA890144F11413590901EB
:10A0C000054A2EC697100000E7802026B245634857
:10A0D000A400014541011783FFFF6700230483A704
:10A0E000090013171400BA9783D707006388B700D5
:10A0F0006394970063742A010504E1B70545D9BF4D
:10A100001783FFFFE70263FDAA892E89328BB6848D
:10A110003A8ABE8A97A00000E78020FB71C9268595
:10A1200097200000E78020098D4763E7A7007D5551
:10A130001783FFFF6700E3FD83DB440097100000F7
:10A14000E780A0242A8497100000E7804025930729
:10A15000740031443305850263CDA70297100000D7
:10A16000E780A02297100000E78020222A84971021
:10A170000000E780C0229307740031443305850254
:10A1800063C3A70497100000E780202093074500D1
:10A1900029A897100000E780802033058502130767
:10A1A000F0179307C017E35FA7FA2D55E3C277F9BD
:10A1B00063040B02D6865286A6854A859720010045
:10A1C000E78020BAB5B797100000E780401D33053F
:10A1D00085029307C5FFD1BF832749001385C900B6
:10A1E00083D5270097000000E78000EC61F581B778
:10A1F00069553DBF97C7FF1F2390A7CA97C7FF1F89
:10A20000938747C9904381470C463307F5004207BF
:10A2100041836393B70082805446139847008507B3
:10A22000C2962390E600D5B797C7FF1F938787C6CE
:10A230009C4303C58700828017C5FF1F0355C5C512
:10A2400082801783FFFFE702C3EBC1671387D7FF45
:10A25000630BE502636AA700F1176300F50201458D
:10A260001783FFFF670023EC1387E7FF6302E50214
:10A27000FD171D8D13351500E5B797500000E780D9
:10A28000C0267D15C5BF97500000E78040FBD5BFB5
:10A2900097500000E78060F9EDB71783FFFFE702F2
:10A2A00043E64111AA8401442EC697100000E780BE
:10A2B000C008B2456348A400014541011783FFFF70
:10A2C000670063E69C48131514003E95835705000C
:10A2D000E385B7FE0504C9BF03485500814693F7DF
:10A2E000F60F63E5070181473E85828058459397C5
:10A2F0005600BA9703D727006316B70003D70700A5
:10A30000E304C7FE8506E1BF834645000147937716
:10A31000F70F63E4D700814711A81C4513165700B7
:10A320000507B29703D60700E313B6FE3E85828089
:10A330001783FFFFE70243DB93170501C18797CA25
:10A34000FF1F938A2AB5635BF00883A70A00C04702
:10A350009C4703570400198D420541816368F5004D
:10A36000014422851783FFFF670043DB12052A940F
:10A37000CDBFDC4713944900014A3E948347440013
:10A380006341FA02014A834754006349FA0285098E
:10A39000C20993D9090183A70A009847E3EBE9FCB6
:10A3A000C1B71C4413195A00A6853E994A859700E7
:10A3B0000000E780C0EE05E1050AC9B75C44131947
:10A3C0005A00A6853E994A8597000000E78020ED57
:10A3D00019E1050A4DBFE30C09FA61B7AA84814966
:10A3E0005DBF1783FFFFE702C3D11C452A8481E7C5
:10A3F0009307C5001CC51C44231204001CC093070E
:10A40000F00F63EDB70093F5F50F2285972000005C
:10A41000E78020E21783FFFF6700E3D093940501F4
:10A42000C167C18063F9F500A685228597200000E9
:10A43000E78040E5C5B7C18193F5F50F22859720E8
:10A440000000E78000DFA685228597200000E780D6
:10A4500040E0C9B797C7FF1F9387C7A3884382808F
:10A460001C4599C797C7FF1F23A6A7A20145828055
:10A470007D55828097C7FF1F9387C7A19843834765
:10A480004500484792073E9582801783FFFFE70209
:10A4900043C7617100451C183EC6B70780013EC81E
:10A4A0001C183ECA8357440002CE02D002CC231EA1
:10A4B000F100834784002A8902D22301F1023C087B
:10A4C0003ED402D697000000E78000FB83570500CA
:10A4D0002316F10297500000E78060C42307A10211
:10A4E0005C4003556400F18313F717008347F102C2
:10A4F00052055181F99BD98FA307F10297100100F2
:10A50000E780807539CDAA840355050097A0000027
:10A51000E78080BC83D704002AD26800231CF100A6
:10A5200083D72400231DF1001C4803D647008C4329
:10A5300097200000E78000CD8347B400CA861786C5
:10A5400001001306A6D28117A305F4006C00481081
:10A5500097200100E780E0805D611783FFFF6700BF
:10A5600083BC2155D5BF1C45B1CF03C5A700894683
:10A5700013576500630BD7028D46630ED7028546DD
:10A580006300D702130740063305E50203C7B7008F
:10A59000418B15CB83C7B700BD8B3355F540828007
:10A5A0001375F5031307803EC5B709671375F503E7
:10A5B00013070771D1BF372709001375F503130778
:10A5C000077CD9B7014582801783FFFFE70263B399
:10A5D00003A98500630C09048347B900AE8493F78F
:10A5E000070E85C303459900930520030D810505DA
:10A5F000B305B5028844610597300100E780E0A902
:10A6000035A02E8597000000E78020F62A8419CD1A
:10A6100097000000E780605C8325C900B307B54060
:10A6200063FA87002E94B305A440E9F51783FFFF72
:10A63000670063AF85457DBF1783FFFFE70263AC0B
:10A640002A8403D50500011132C636C43AC22EC091
:10A6500002CA02CC02CE97A00000E780E0A78245A4
:10A660002ACA22852ECC97000000E780E0E003573D
:10A670000500231EE10097500000E78040AAA24693
:10A6800032469247230FA10036874C08B2862285B6
:10A69000014697000000E780E0A605611783FFFFF1
:10A6A000670063A81783FFFFE702A3A561711C1869
:10A6B0003EC6B70780013EC81C183ECA3C0800458C
:10A6C0003ED4AA8402CC02CE02D002D202D6970097
:10A6D0000000E78060DA8357050035592316F10240
:10A6E00097500000E780A0A32307A10209C4835765
:10A6F000440081EB21594A855D611783FFFF6700A4
:10A7000083A2035564005205518197100100E78030
:10A71000A0542A8965D18347B40093F7070E99C7DF
:10A720001305840197300100E78060998357440046
:10A73000231EF100834784002301F1025C4003558E
:10A740000900D98313F7070883471102231CA100CE
:10A7500093F7F707D98FA300F10283572900231D30
:10A76000F1005C40F18313F717008347F102F99B76
:10A77000D98FA307F10297A00000E780E0952AD2C5
:10A7800035D9834794006800139757008347B40076
:10A79000FD8BD98FA305F4001C4803D647008C43DA
:10A7A00097200000E78000A6A687178701001307FF
:10A7B000E7AB740005464C10268597000000E78043
:10A7C00060942A890DD98347B400A685FD8BA30523
:10A7D000F40097000000E78060DF31BF1783FFFFC0
:10A7E000E7022392832485FE2A844111268597005F
:10A7F0000000E78080D7834734FF93F7070E8DCBA7
:10A800002AC6268597000000E78060C809CD8347E7
:10A8100034FFB245FD8BA309F4FE91C52285973024
:10A820000100E780808741011783FFFF6700A38F46
:10A830007DD98327C4FF2685829775F5834734FF2A
:10A8400093F7070E91C7228597300100E780208794
:10A85000032584FE97000000E78000E5E9B7178331
:10A86000FFFFE70203879C4141112A8903C70700C4
:10A8700089472E84935667006380F6040D466388EB
:10A88000C6049307F0076304F7022E8597200000A3
:10A89000E780C0A7AA848149C16B130C490097B710
:10A8A000FF1F9387275F9C43984763E4E9044101B6
:10A8B0001783FFFF6700A38503D745008547E3F8AB
:10A8C000E7FE2E8597200000E780A0A9E1B703D717
:10A8D0004500E3FEE7FC2E8597200000E78000A3FB
:10A8E000AA84228597200000E78060A4C204C98C56
:10A8F0005DB7DC470355A900139A49003E9A9317A8
:10A900000501C187635DF00083570A006397A702C2
:10A9100063E774038327CA00034D5A002DA0A16783
:10A920002167A98F1307F7EFE374F7FE6397090018
:10A9300097000000E780209161FD85098DB783278E
:10A940008A00034D4A00835DA90003576900216A0C
:10A95000138BC7003AC6814A33CA4D01631E5D019D
:10A9600097B7FF1F938787539C43E1DBA2866286DC
:10A97000814526858297D1B7A1679387F7EF930C1E
:10A980004BFF63F24703B2455A8597F0FFFFE7801C
:10A99000A0710DC103278B00104709CE10436382BD
:10A9A000C4023107D5BFEE85668597000000E780B9
:10A9B000008F71F993861A0093FAF60F130B0B02AE
:10A9C00071BF835644005C43E3E9F6F622853AC63C
:10A9D00097100000E780807DA1679387D7042A8ABB
:10A9E000035D4400324763E897008347D90093E74B
:10A9F00007F8A306F9001C4766852286E285829740
:10AA0000C1670844FD17337AFA00529508C0231233
:10AA1000A40125B797B7FF1F9387C747984381477E
:10AA200015C31447814763FFD500939745004C47F2
:10AA3000BE9519C903C7550081476375E600DC451B
:10AA40001606B2973E85828003C745008147E37BA7
:10AA5000E6FE16069C45F5B71773FFFFE702C368CD
:10AA6000AA892E8A814497BAFF1F938AAA4283A794
:10AA70000A00984763E6E4001773FFFF6700036A64
:10AA8000DC471394440001493E9413BB14008347F0
:10AA90004400634BF900014913BB14008347540081
:10AAA000634FF9008504E1B70844931759005287B2
:10AAB000DA860146A2853E9582990509C9BF4844B8
:10AAC000931759005287DA860546A2853E958299EA
:10AAD0000509E9B71773FFFFE702A362814517F580
:10AAE000FFFF1305054897B7FF1F2397073A970005
:10AAF0000000E780A0F61773FFFF6700C36297B7F7
:10AB0000FF1F938727399C4395C31773FFFFE70205
:10AB1000435F814517F5FFFF1305A544970000002B
:10AB2000E780C0F31773FFFF6700E35F828017734E
:10AB3000FFFFE702635B37E40400832784124111BF
:10AB40002315E100AE893289368A3A86814601476B
:10AB5000ED45AA8482972AC621C90356A100D28551
:10AB600097400100E780C0248327C413CE85268543
:10AB70008297058905C98327440D231421010146C5
:10AB80002C00268582972A8401C9B7E7040083A791
:10AB9000C712ED4528008297228541011773FFFFF8
:10ABA0006700C3574944D5B76554FDB75C41FD17ED
:10ABB0005CC182801773FFFFE702A354B7E704006C
:10ABC000FC5F829795473305F50281450D81177328
:10ABD000FFFF670043551773FFFFE7028352B7E794
:10ABE0000400FC5F829795473305F5020D811773CA
:10ABF000FFFF670043531773FFFFE7028350B7E778
:10AC0000040083A7870B0355050082971773FFFF86
:10AC1000670063511773FFFFE702A34E035505005A
:10AC20003287AE861796FF1F0356A68A97B5FF1F79
:10AC30009385052797000000E780A0EF1773FFFFBB
:10AC40006700634E1773FFFFE702A34BB7E70400EB
:10AC500083A7C71782971773FFFF6700C34C17734B
:10AC6000FFFFE702034AB7E7040083A7871397B5FE
:10AC7000FF1F9385E522829701451773FFFF670049
:10AC8000834A1773FFFFE702C347B7E7040083A7B0
:10AC9000C71F81451785FF1F0355A57F829717732F
:10ACA000FFFF670043481773FFFFE7028345B7E7DD
:10ACB000040083A7871397B5FF1F9385651F8297AD
:10ACC00001451773FFFF670003461773FFFFE70295
:10ACD0004343B7E7040083A7C71F81451795FF1FAC
:10ACE0000355258182971773FFFF6700C3431773CE
:10ACF000FFFFE70203412E8597800000E780E0AF69
:10AD000097800000E780E0EC1773FFFF6700A34126
:10AD10001773FFFFE702E33E97800000E780E0F64D
:10AD20001773FFFF670023405C49E1175CC95CC5EE
:10AD300083572501A1072319F50083570501A107B2
:10AD40002318F5008280F1473305F50297B7FF1FFE
:10AD5000938707189C433E9582808D476315F608BC
:10AD600003D74600854763F0E7081773FFFFE70244
:10AD70004339368536842E8997100000E7800059C4
:10AD800029C98357440093140501C18063E39704E4
:10AD9000228597100000E7806057FD14231294006D
:10ADA0009307A0026300F5029307B0026307F50260
:10ADB00093079002631FF500228597000100E7804A
:10ADC000C08501A80146CA85228597A00000E780BA
:10ADD00060B01773FFFF67000335228597100000EE
:10ADE000E780C003FDB7828097B6FF1F9386860E6B
:10ADF0009C42014599CF9843D44217B6FF1F232B9D
:10AE0000E60C6396D70097B6FF1F23A7E60C1385C1
:10AE1000C7FE82801773FFFFE702A32E9700000092
:10AE2000E780A04B7144330585029145979000005F
:10AE3000E78020E911E565551773FFFF6700A32E32
:10AE400097B7FF1F23A4A70897000000E780E048FA
:10AE500033058502914597900000E78080E661DD2B
:10AE600097B7FF1F23A6A70697000000E780E046DC
:10AE700097B7FF1F2396A70497000000E780E045DF
:10AE800097B7FF1F239FA702977701009387474338
:10AE900017B7FF1F232AF70297070000938707E9D8
:10AEA00017B7FF1F2320F702014579B71773FFFF7C
:10AEB000E7022325AA8517B5FF1F13056500971024
:10AEC0000000E780C05B1773FFFF6700C32517739F
:10AED000FFFFE702032397000000E78060FD971063
:10AEE0000000E780405B97B7FF1F9387A7FE9C4356
:10AEF00091CF1387C7FE19CB83D5C7FF17B5FF1FA7
:10AF00001305C5FD97200100E78020191773FFFF87
:10AF1000670063211773FFFFE702A31E970000007D
:10AF2000E780C0EC09CD834785002A8493F70704A6
:10AF300099EB0355E50097000000E78080F917734F
:10AF4000FFFF6700431E8347C5009304450117B9FF
:10AF5000FF1F130929F885E3832709005CC997B708
:10AF6000FF1F23A997F683274900F1FB97B7FF1F1F
:10AF700023A497F6E9B7FD172306F500610597802E
:10AF80000000E780C0D68307840063CB07048347B3
:10AF9000840093E707F82304F400B7E704009C5FFC
:10AFA00082974205A94741813375F50283478400A2
:10AFB00093F707FCC98F2304F4008347D4003E9520
:10AFC0001C402318A40089CF984319CB8347C400A1
:10AFD0005040814585073305F502420541810297BE
:10AFE000832709005CC897B7FF1F23A597EE832727
:10AFF000490089E797B7FF1F23A097EE8347C40056
:10B000009DDF8355040117B5FF1F130525ED97201C
:10B010000100E780800825B71773FFFFE702630E82
:10B0200097B7FF1F9387C7109C4701448583858B83
:10B0300085E3AE84B2853A8697100000E780804BA6
:10B040002A8419C597100000E780C041829408CC7B
:10B0500022851773FFFF6700030D1773FFFFE702D9
:10B06000A30841112E8932C6AA8997000000E78003
:10B07000C031324713060502CA8697050000938542
:10B08000C5CC17B5FF1F1305A5E397000000E780A7
:10B09000E0F82A8425C99304C50097000000E780E2
:10B0A000E0411946AA85268597100000E7808015A3
:10B0B0008545268597100000E7806011177501000F
:10B0C0001305C51D4E958345050026859710000084
:10B0D000E78020165C4831468145A1075CC85CC406
:10B0E00083572401E1172319F40083570401E11762
:10B0F0002318F4001C4C3E859770FFFFE780600327
:10B10000A3042501228541011773FFFF6700030196
:10B110001773FFFFE702E3FE4111AA842EC632C473
:10B1200097100000E7806036004DB2452246834705
:10B1300084000CC050C093F7F70393E7070423047F
:10B14000F40023180400268597100000E780803162
:10B1500083479400A9462317A40013D73700050797
:10B160003307D7029D8B85072306F400A306E4006E
:10B1700083C70401D8488507230FF7FE17B7FF1FC1
:10B18000130747D55843232A04009307440129E3B2
:10B1900017B7FF1F2322F7D417B7FF1F232CF7D2AF
:10B1A00017B4FF1F130484D3228597200100E78082
:10B1B00000E11C44858B5D8D19E581452285972032
:10B1C0000100E78080ED41011773FFFF6700A3F5E1
:10B1D0001CC317B7FF1F2321F7D0D9B71773FFFF81
:10B1E000E70223F297050000938565B701459700B4
:10B1F0000000E78000B001451773FFFF6700A3F26E
:10B200001773FFFFE702E3EF97000000E78080B0CD
:10B210001773FFFF670023F18347C500A5E317738A
:10B22000FFFFE70203EE2A840355E50097000000C4
:10B23000E78000C821C18347840093F7F7FB23040C
:10B24000F4001C4091C7DC4381C74C400145829704
:10B2500097000000E78080B917B5FF1F130505C8E8
:10B2600097200100E780A0E50355E4009700000067
:10B27000E78020C61773FFFF6700E3EA8280177339
:10B28000FFFFE70203E897B7FF1F9387A7C497055F
:10B290000000938565C817B5FF1F130525C423A0BB
:10B2A000070023A2070097200100E780E0CE177374
:10B2B000FFFF670043E71C4D91CFDC4381CF17733D
:10B2C000FFFFE70203E48345070082971773FFFF40
:10B2D000670063E5828097B7FF1F938767C29C432F
:10B2E00003C50700828097B7FF1F938767C19C4300
:10B2F00003C51700828097B7FF1F938767C09C43E1
:10B3000003C52700828097B7FF1F938767BF9C43C1
:10B3100003C54700828097B7FF1F938767BE9C4392
:10B3200003C53700828097B7FF1F938767BD9C4393
:10B3300003C55700828097B7FF1F938767BC9C4364
:10B3400003C56700828097B7FF1F938767BB9C4345
:10B3500003C57700828097B7FF1F938767BA9C4326
:10B3600003C58700828097B7FF1F938767B99C4307
:10B3700003C59700828097B7FF1F938767B89C43E8
:10B3800003C5A700828097B7FF1F938767B79C43C9
:10B3900003C5B70011E11D45828097B7FF1F938752
:10B3A00027B69C4303C5C700828097B7FF1F9387CA
:10B3B00027B59C4303C5D700828097B7FF1F9387AB
:10B3C00027B49C4303C5E700828097B7FF1F93878C
:10B3D00027B39C4303D50701828097B7FF1F93874C
:10B3E00027B29C4303C52701828097B7FF1F93872D
:10B3F00027B19C4303D54701828097B7FF1F9387EE
:10B4000027B09C4303D56701828097B7FF1F9387BE
:10B4100027AF9C4303D58701828097B7FF1F93878F
:10B4200027AE9C4303C5A701828097B7FF1F938770
:10B4300027AD9C4303C5B701828097B7FF1F938751
:10B4400027AC9C4303C5C701828097B7FF1F938732
:10B4500027AB9C4303C5D701828097B7FF1F938713
:10B4600027AA9C438857828097B7FF1F938747A9D5
:10B470009C4303D5C702828097B7FF1F938747A8D5
:10B480009C4303D5E70219E11305800C828097B72E
:10B49000FF1F9387E7A69C4303C50703828097B7E6
:10B4A000FF1F9387E7A59C43C85B828097B7FF1F68
:10B4B000938787A48843828097B7FF1F938707A449
:10B4C0008843828019E17D558280F5DE984265DFF0
:10B4D000FDD917B7FF1F1307A7C51847AA877155CE
:10B4E000058B631D072403C507001547E37DA7FCF3
:10B4F00003C737001305F0057D171377F70FE364D3
:10B50000E5FC03C35700E30003FC83C86700E38C3A
:10B5100008FA03C77700494579171377F70FE364F3
:10B52000E5FA03C7A70011481305F7FF1375F50FD8
:10B53000E36BA8F803CE97000D481305FEFF1375C3
:10B54000F50FE362A8F803C8B7006309080065189F
:10B550001378F80F1305600DE36705F703C5C700FF
:10B56000794879151375F50FE36FA8F403C8D70070
:10B570000D457D181378F80FE36705F503D807012B
:10B58000930E40175118420813580801E3ED0EF3CB
:10B5900003C8E7007D181378F80FE36605F303C8C6
:10B5A00027017D181378F80FE36F05F103C88700B2
:10B5B000C54E75181378F80FE3E70EF103D867014D
:10B5C000856E938EBEE06D18420813580801E3ECB7
:10B5D0000EEF03D847016D18420813580801E3E441
:10B5E0000EEF03D887017918420813580801E36C5D
:10B5F00005ED03C8A7017D181378F80FE36505ED85
:10B6000003C5B7011D487D151375F50FE36DA8EA55
:10B6100003C5D701714879151375F50FE365A8EADD
:10B6200003D5E7011308E00F7D1542054181E36C66
:10B63000A8E803C50702494879151375F50FE364B7
:10B64000A8E8C85301C937C834005915130858BFB2
:10B65000E36BA8E603A8870237C53400130555BF7E
:10B660005918E36205E717B5FF1F2329C58803C6EC
:10B67000050117B5FF1F2325F5880545E375C5E4CA
:10B6800003D82501D04933760603E31E06E203C63C
:10B690001501E30A06E217B6FF1F232FB68483C500
:10B6A000270001466387A50003C61700F14533064E
:10B6B000B60283C707039305C00272971A071307E0
:10B6C000C70516031A9796084697B387B7024155E0
:10B6D0003E973297420741836362E8061773FFFF84
:10B6E000E70223A2368597800000E780A0689700D4
:10B6F0000100E78020482A8497A00000E780805A54
:10B700002A9497F00000E78060262A949790000022
:10B71000E780A0812A9497F0FFFFE780E06F2A94EA
:10B7200097400000E78060932A9497700000E780BC
:10B73000A09C22951773FFFF6700E39E828017731A
:10B74000FFFFE702039C4111A307A10097A000009F
:10B75000E780A0C59305F100170500001305E5B5C6
:10B7600097F0FFFFE780802F014541011773FFFF2E
:10B770006700639B1773FFFFE702239617B4FF1F51
:10B780001304049B0328840079599368180097B424
:10B79000FF1F23A3149B1378180063100802BA84B8
:10B7A000BE89368B328A2E89AA8A97F0FFFFE780FE
:10B7B000E0A77D15269519E531594A851773FFFFD6
:10B7C0006700239597F0FFFFE78040A67D1526953B
:10B7D000A167E353F5FE97B7FF1F938727CC9843E4
:10B7E0003E8C814B01CB014597F00000E78020445F
:10B7F000933B15004A85DA865686D28597900000DD
:10B80000E780C04D2A8911CD1C44F99B17B7FF1F53
:10B810002324F79283270C00CDD3E3800BFA829781
:10B8200069BF268597B7FF1F23A6079097F0FFFFF4
:10B83000E780809C4146CE8517B5FF1F1305C5984C
:10B8400097300100E780C05697D00000E78040990C
:10B850000325040B97D00000E780009D054597D095
:10B860000000E78000A4054597000000E78060ED38
:10B87000A9B797B7FF1F9387A78B9C47858BEDC709
:10B880001773FFFFE702E38717B5FF1F1305059244
:10B8900097B7FF1F23AE078897B7FF1F23AC078812
:10B8A00097B7FF1F23AA078897200100E780208110
:10B8B00097500000E780E0F597100100E780A04C6A
:10B8C00097100100E780A05297B7FF1F9387C784A6
:10B8D0009C4391C7054597800000E780402097A7CB
:10B8E000FF1F9387276D9C4399C741657D1597700E
:10B8F0000000E78040A297F00000E780E03D97D08D
:10B900000000E780808F97B7FF1F938727979C439E
:10B91000139717016356070097F00000E78000AD0A
:10B9200097B7FF1F23A2078A97B7FF1F23A0078A95
:10B9300097B7FF1F23AE078897B7FF1F23AC078871
:10B9400097000000E780008C97000000E7800072FD
:10B9500097F0FFFFE780401897F00000E78040D69F
:10B960001763FFFF6700237C828097A7FF1F9387E1
:10B97000277C884382801763FFFFE70283789780E4
:10B980000000E780607597800000E780C07717634C
:10B99000FFFF670043791763FFFFE702E3742A8420
:10B9A0009304140201112E85B289A685214636C65C
:10B9B0003A8997300100E780403D0DE9B2463808EA
:10B9C0002686CE851305940497500000E7806041D9
:10B9D00021462C084A8597300100E780003B13354B
:10B9E000150005611763FFFF670043730145D5BF6D
:10B9F0001763FFFFE702E3709305450617A5FF1FD6
:10BA00001305455097100100E78020691763FFFF79
:10BA1000670063711763FFFFE702A36E41112EC633
:10BA200097F0FFFFE780601BB24588C141011763B3
:10BA3000FFFF6700436F1763FFFFE702E36AAA8413
:10BA40002E8497800000E780006CAA8985452285B6
:10BA500097000000E780E07D83C7E4011389940824
:10BA600099E313890403CE85228597000000E780BF
:10BA7000407C214693051902228597000000E7804B
:10BA8000607897A7FF1F9387A76A8C43228597103A
:10BA90000000E780C08221469385840222859700BA
:10BAA0000000E78020761763FFFF670023671763B6
:10BAB000FFFFE7028362397197F00000E780E0B48E
:10BAC0009305400661E997800000E780006063020B
:10BAD000051497A7FF1F83C7A74413B7170097A69E
:10BAE000FF1F238FE642014499CFC16417A9FF1FAE
:10BAF000130909649309400EFD1497000000E780C4
:10BB0000C0866342A40A97F0FFFFE780000D4169F9
:10BB1000B7290900096AFD7A2A8B81447D19938926
:10BB2000F97B130A0A71938A8AC797000000E7809D
:10BB3000C08363D7A4041304400EB387840217A7FD
:10BB4000FF1F1307E75E0324070B3E948357C401CE
:10BB50006382270B18403307EB4063EAE900834711
:10BB600044008507B3874703D6976365F708014606
:10BB70008145094597F0FFFFE780604EAA8B29E5D4
:10BB800097400000E780808385476317F506896545
:10BB90009385057117A5FF1F1305C5369710010082
:10BBA000E780A04F95A0B30734030327090BBA978A
:10BBB00003D7C7016308970003C75700A382070094
:10BBC0002382E700050415BF9305C5002285970071
:10BBD0000000E78080E65E852286976501009385F8
:10BBE000256D97F0FFFFE780E0525E85971000001B
:10BBF000E780608A850415BF97A7FF1F9387475387
:10BC00009C478D83858BC1F721611763FFFF670018
:10BC1000435001468545094502D002D202D402D6DE
:10BC200097F0FFFFE780A043AA8479DD97F000003A
:10BC3000E780E09C1389C4002A8481454A859700E7
:10BC40000000E780005F0C4041464A8597000000F5
:10BC5000E780405B832944006385090C4E8502D848
:10BC600002DA02DC02DE97300100E78000482ACECB
:10BC7000141005462C0808184ECC97500000E78099
:10BC8000E00A1375F50F51ED8355840093E5250007
:10BC90004A8597000000E780E05E11460C104A8557
:10BCA00097000000E78000560146976501009385E4
:10BCB000A560268597F0FFFFE780C04526859700A1
:10BCC0000000E780407D5C40A1D3014685450D45DD
:10BCD00097F0FFFFE780A038AA841DD5484013895C
:10BCE000C40097300100E78040402AC64A8597008B
:10BCF0000000E780404C3246636FC5004C404A85E7
:10BD000097000000E780005001468145268597F0A6
:10BD1000FFFFE7802040268597000000E780A0779E
:10BD2000E5B583558400ADB71763FFFFE702633DB8
:10BD300097A7FF1F9387C73F9C471DC193E78700C5
:10BD400017A5FF1F1305051C17A7FF1F2326F73E86
:10BD500097100100E78040321763FFFF6700A33CA4
:10BD6000DD9B17A7FF1F2329F73C97300000E780D2
:10BD7000E0647DF117A5FF1F1305C518971001009A
:10BD8000E780E033D1BF1763FFFFE7020335416966
:10BD9000AA892E8AB28A368BBA8B814417ACFF1FD0
:10BDA000130C0C39930C400E7D1997F0FFFFE780C0
:10BDB000C05B63C4A40001443DA033849403832783
:10BDC0000C0B3E948357C401638627055A87D68699
:10BDD0005286CE851305040397000000E780E0BB80
:10BDE00001C923800B0022851763FFFF67006332C0
:10BDF0008347F40185C35A87D6865286CE851305BC
:10BE0000940897000000E78040B909C58547238062
:10BE1000FB00D1BF850451BF835745006380071ED7
:10BE20001763FFFFE702432C01112A8497000000EB
:10BE3000E780C04D09C985476309F50605611763A9
:10BE4000FFFF6700A32D97E00000E780007C7DF5F1
:10BE5000835744004947ED9BE392E7FEC1452285A5
:10BE600097000000E7804033AA84228597000000F5
:10BE7000E780204F0357440002CE91472A89631A76
:10BE8000F700228597000000E780A0513C082ACCEB
:10BE90003ECE97E00000E78080765C55C5D37408FD
:10BEA0004A86A6850545829751BF03574400D1476E
:10BEB000E3F6E7F8032A0400C169014997AAFF1FC6
:10BEC000938A0A27130B400EFD1997F0FFFFE780B6
:10BED000C049634FA90E2285032A04009700000081
:10BEE000E780C042A1452A89228597000000E780AB
:10BEF000A02AAA84228597000000E780804A144087
:10BF00002A86AA8978082685CA8597000000E780D6
:10BF1000C0E7AA8405D503C7F40189476315F70074
:10BF20008347C10181DF5546D28513856400973070
:10BF30000100E780E0E7014597800000E780C01935
:10BF400001C583D7C401A5E797A7FF1F9387471EA5
:10BF50009C4793551900858913D73700058B01CF6E
:10BF60008983858B6399B70001452EC69700000031
:10BF7000E780C0DBB2454E8597800000E780601FF8
:10BF80000346C1012A849375190026859790000005
:10BF9000E780E03935C1268597800000E780E0180A
:10BFA000268511C0014597800000E780004C97303E
:10BFB0000000E780A0408547E312F5E883C75400FE
:10BFC0001307F00FE38CE7E68507A382F400BDB505
:10BFD000B304690383A70A0BBE9483D7C401638BA0
:10BFE00037015546D2851385640097300100E780FC
:10BFF000C0D955DD0509D1BD5DD86DB78280176305
:10C00000FFFFE702630E97800000E780000C05C188
:10C01000C164014417A9FF1F130989119309400E38
:10C02000FD1497F0FFFFE7804034634EA40017A58E
:10C03000FF1F130525ED97100100E780E00317634C
:10C04000FFFF6700A30D330534038327090B3E95DB
:10C050008357C5016388970023120500978000006D
:10C06000E780A00C050475BF97A7FF1F9387470CB7
:10C070009C478D83858B8DE31763FFFFE702630881
:10C0800017A5FF1F130505E897100100E78020039F
:10C090001763FFFF6700230982801763FFFFE70232
:10C0A0004306970500009385C5A017A5FF1F13053C
:10C0B00065E597100100E78020EE1763FFFF67003A
:10C0C00083061763FFFFE702C3038841B7E7040055
:10C0D000BC5B050542054181829709C58547230060
:10C0E000F50005051763FFFF6700E30383C7F5FF4E
:10C0F0002E858507A38FF5FE828083C7F5FFFD1788
:10C1000093F7F70FA38FF5FE99EF1763FFFFE70291
:10C1100043FFB7E70400BC571385F5FF8297176309
:10C12000FFFF6700430082801C41035745008D8F4D
:10C13000BA951CC12312B5003E85828093D7850035
:10C14000A2051441DD8D835745001387E6FF18C112
:10C1500089072312F50013D685004111238FB6FEFF
:10C16000A38FC6FE4101828018419307F7FF1CC1CF
:10C170008357450085072312F500A30FB7FE828081
:10C18000835745008D8F2312F5001C41BE950CC1CD
:10C190002E858280AA8703D7470008410D8FAA9574
:10C1A0002392E7008CC38280184108453305A740DD
:10C1B000828083574500035765001D8F1C41084549
:10C1C0003385A7403305A74082801763FFFFE7024E
:10C1D00043F341112EC62A8497000000E780A0FD9A
:10C1E000B2456373B50001A0835744000840BE9573
:10C1F0002312B4003E9541011763FFFF6700A3F2CD
:10C200001763FFFFE702E3EF41112E84B28532C6C8
:10C2100097000000E780A0FB3246A285973001001E
:10C22000E78000B941011763FFFF6700C3EF1763A1
:10C23000FFFFE70203ED2E84854597000000E780AD
:10C2400000F9230085001763FFFF6700C3ED176344
:10C25000FFFFE70203EB41112317B1008945970067
:10C260000000E780C0F68347E1002300F500834724
:10C27000F100A300F50041011763FFFF6700A3EA87
:10C280001763FFFFE702E3E793D78500A20541119B
:10C29000DD8D2317B100894597000000E78020F36A
:10C2A0008347E1002300F5008347F100A300F50078
:10C2B00041011763FFFF670003E71763FFFFE70212
:10C2C00043E41397850193D78501C166938606F0F1
:10C2D000D98F13D78500758FD98FA2053707FF0037
:10C2E000F98D4111DD8D2EC6914597000000E78044
:10C2F00000EE6C00114697300100E78060AB410111
:10C300001763FFFF670023E21763FFFFE70263DFA6
:10C310001C41854503C4070097000000E78080E6C4
:10C3200022851763FFFF670003E01763FFFFE70243
:10C3300043DD1C414111894503C7070083C717002E
:10C340002307E100A307F10097000000E78080E3E6
:10C350000355E10041011763FFFF6700C3DC17636A
:10C36000FFFFE70203DA1C414111894503C70700BB
:10C3700083C717002307E100A307F100970000001F
:10C38000E78040E08357E100410113D58700A20711
:10C390005D8D420541811763FFFF6700C3D81763B6
:10C3A000FFFFE70203D60C4141112A8411466800C1
:10C3B00097300100E780C09F9145228597000000DB
:10C3C000E78040DCB247C166938606F01397870189
:10C3D00013D58701598D13D78700758F598DA20703
:10C3E0003707FF00F98F5D8D41011763FFFF67007D
:10C3F00083D31C45BE950CC18280AE87944391E6E1
:10C40000584101EF0CC15CC1828003C7570013671C
:10C410001700A382E700B687D5B70CC3EDB7AA878C
:10C42000084119CD1841D44398C36313D500D8C32C
:10C430002A87034657009376160081E623200700DB
:10C440008280944381CA8C4203A847008CC36393C3
:10C450000601CCC3799A14C3A302C7003687D1BFA3
:10C460001C45DC471D8DB777DBB6938777DB0985E5
:10C470003305F502420541818280F147B385F5021B
:10C4800048452E9582808347450085072302F500A5
:10C4900082801763FFFFE702C3C62A8409E417639B
:10C4A000FFFF670043C883474400F5DBFD1793F7A0
:10C4B000F70F2302F400E5F71C4403D72700050714
:10C4C0002391E700DC4399C3228582974C4889CDAC
:10C4D00083475400898B99E71C4422859C479C43E1
:10C4E0009C478297232A04000040232004007DB744
:10C4F0001763FFFFE702E3C08357250041112EC6F3
:10C5000081EB0144228541011763FFFF6700A3C14E
:10C51000035705008147F146E305F7FEB385D702CF
:10C52000404585072E948345440008C4F5F5B2477D
:10C53000AA8481E7232A040009A81C456C002285EF
:10C540009C439C43829748C84DDD85472312F400E5
:10C55000B24723200400231804002319F4005C4888
:10C560005CC483D72400FD172391F40061BF1763D7
:10C57000FFFFE70203B997A7FF1F9387A79A884396
:10C580002326050023240500410597100100E780BC
:10C5900000B31763FFFF670003B91763FFFFE702EC
:10C5A00043B617A4FF1F1304E4971C40411199CF11
:10C5B0009C472300B5002AC65CC197000000E780B5
:10C5C00040FB1C40DC4399C332458297410117630D
:10C5D000FFFF670043B50347450029E3584DAA878D
:10C5E0007D551DCF1763FFFFE702A3B11CC3DC47D6
:10C5F00097A6FF1F23A8E692F15613050701239083
:10C60000D700970500009385050297100100E78089
:10C61000A09801451763FFFF6700E3B07D55828056
:10C6200082801763FFFFE702C3AD011161468145B8
:10C6300028009760FFFFE780C0AF97A7FF1F938791
:10C64000678E9C4328009305F00FDC473EC6970099
:10C650000000E780C0F405611763FFFF6700A3AC2B
:10C6600097A7FF1F9387078C9C43D847A1679387A1
:10C67000C702631EF70A397106DE22DC26DA800063
:10C680004AD84ED652D456D23285B2849700000092
:10C69000E780C0C7AA89268597000000E78020C9E7
:10C6A0002318A4FC268597000000E78040C82319C2
:10C6B000A4FC268597000000E78060C783D744006C
:10C6C0000A8A231AA4FC858393F7F70F230EF4FC40
:10C6D0008607BD0793F7073F3301F1408A8A014976
:10C6E0008347C4FD6367F902CE85130584FC232CC0
:10C6F00054FD97000000E78080EA5281130104FC9A
:10C70000F2506254D2544259B259225A925A21617B
:10C710008280268597000000E78060C1931719008A
:10C72000D69705092390A7001379F90F55BF82808A
:10C730009797FF1F9387077F9C43D847A1679387ED
:10C74000A702631AF70A397106DE22DC26DA8000B6
:10C750004AD84ED652D456D23285B28497000000C1
:10C76000E780C0BAAA89268597000000E78020BC30
:10C77000FD572318A4FC26852319F4FC970000001C
:10C78000E780E0BA83D744000A8A231AA4FC858391
:10C7900093F7F70F230EF4FC8607BD0793F7073FC7
:10C7A0003301F1408A8A01498347C4FD6367F90276
:10C7B000CE85130584FC232C54FD97000000E780F0
:10C7C00000DE5281130104FCF2506254D2544259EB
:10C7D000B259225A925A2161828026859700000020
:10C7E000E780E0B493171900D69705092390A700B6
:10C7F0001379F90F55BF82809797FF1F9387877230
:10C800009C43D847A16789076310F70A397106DE90
:10C8100022DC26DA80004AD84ED652D456D232854F
:10C82000328997000000E78060AEAA894A859700A8
:10C830000000E780C0AF835749000A8A2318A4FC90
:10C84000858393F7F70F230CF4FC8607BD0793F756
:10C85000073F3301F1408A8A8144834784FD63E7BF
:10C86000F402CE85130584FC232A54FD97000000B2
:10C87000E780E0D25281130104FCF2506254D2549A
:10C880004259B259225A925A216182804A859700B0
:10C890000000E780C0A993971400D69785042390E1
:10C8A000A70093F4F40F55BF82809797FF1F9387DB
:10C8B00067679C43D847A1679387E704631EF70A1D
:10C8C000397106DE22DC26DA80004AD84ED652D4F0
:10C8D00056D23285B28497000000E78020A3AA894F
:10C8E000268597000000E78080A42318A4FC2685F5
:10C8F00097000000E780A0A3231AA4FC26859700D8
:10C900000000E780C0A283D744000A8A2319A4FC50
:10C91000858393F7F70F230EF4FC8607BD0793F783
:10C92000073F3301F1408A8A01498347C4FD6367A9
:10C93000F902CE85130584FC232C54FD97000000DA
:10C94000E780E0C55281130104FCF2506254D254D6
:10C950004259B259225A925A216182802685970003
:10C960000000E780C09C93171900D6970509239013
:10C97000A7001379F90F55BF82809797FF1F938700
:10C98000675A9C43D847A1679387C704631AF70A7D
:10C99000397106DE22DC26DA80004AD84ED652D41F
:10C9A00056D23285B28497000000E7802096AA898B
:10C9B000268597000000E7808097FD572318A4FC88
:10C9C0002685231AF4FC97000000E780409683D761
:10C9D00044000A8A2319A4FC858393F7F70F230EDA
:10C9E000F4FC8607BD0793F7073F3301F1408A8ABD
:10C9F00001498347C4FD6367F902CE85130584FCB2
:10CA0000232C54FD97000000E78060B95281130188
:10CA100004FCF2506254D2544259B259225A925AEA
:10CA200021618280268597000000E780409093175F
:10CA30001900D69705092390A7001379F90F55BF60
:10CA400082809797FF1F9387E74D9C43D847A16744
:10CA5000DD076317F7041753FFFFE702836A797155
:10CA60003285328497000000E780408A2AC62285FA
:10CA700097000000E780A08B2311A1022285970078
:10CA80000000E780A088B2452300A1022808970093
:10CA90000000E780C0B045611753FFFF6700A3683F
:10CAA00082809797FF1F9387E7479C43D847A167EA
:10CAB000938787046317F7041753FFFFE702636444
:10CAC00079713285328497000000E78020842AC67D
:10CAD000228597000000E78080852311A10222852E
:10CAE00097000000E7808082B2452300A102280859
:10CAF00097000000E780A0AA45611753FFFF670079
:10CB0000836282809797FF1F9387C7419C43D847D2
:10CB1000A1679387A7046312F7021753FFFFE70289
:10CB2000435E01112800814597000000E78020A79F
:10CB300005611753FFFF6700035F82809797FF1F10
:10CB40009387473E9C43D847A16793875702631951
:10CB5000F7021753FFFFE702C35A0111328597F01E
:10CB6000FFFFE780A07A2308A100814528009700F5
:10CB70000000E780C0A205611753FFFF6700A35ABA
:10CB800082809797FF1F9387E7399C43D847A16717
:10CB90009387E702631BF7041753FFFFE70263560F
:10CBA00001113285328497F0FFFFE7804078AA8434
:10CBB000228597F0FFFFE7808077854709E9228586
:10CBC00097F0FFFFE78080744205B337A00028008C
:10CBD0008145231891003ECA97000000E780209C01
:10CBE00005611753FFFF6700035482809797FF1F6B
:10CBF000938747339C43D84799476313F7081753E4
:10CC0000FFFFE702035079713285328497F0FFFF0E
:10CC1000E780C06F2AC6228597F0FFFFE78020716A
:10CC20002310A102228597F0FFFFE780206E2301E9
:10CC3000A102228597F0FFFFE780406DA301A102CA
:10CC4000228597F0FFFFE780606C2302A102228516
:10CC500097F0FFFFE780806B2313A102228597F0F6
:10CC6000FFFFE780A06AB2452314A10228089700BD
:10CC70000000E780C09245611753FFFF6700A34A99
:10CC800082809797FF1F9387E7299C43D847A16726
:10CC90009387C7036313F7081753FFFFE702634641
:10CCA00079713285328497F0FFFFE78020662AC6CB
:10CCB000228597F0FFFFE78080672310A10222857D
:10CCC00097F0FFFFE780A0662311A102228597F06D
:10CCD000FFFFE780A0632302A102228597F0FFFFF8
:10CCE000E780C062A302A102228597F0FFFFE780E0
:10CCF000E0612303A102228597F0FFFFE780006136
:10CD0000B245A303A102280897000000E78020890C
:10CD100045611753FFFF6700034182801753FFFFF0
:10CD2000E702233E01112A8497F0FFFFE780005EAF
:10CD3000AA84228597F0FFFFE780605F228597F045
:10CD4000FFFFE780C05E035744008D4763F7E700AD
:10CD5000228597F0FFFFE780805D228597F0FFFF37
:10CD6000E780E05C2800A68597000000E78020832C
:10CD700005611753FFFF6700033B9797FF1F9387DA
:10CD8000671A9C43D847A167FD07631FF700175335
:10CD9000FFFFE7020337328597000000E78040F885
:10CDA0001753FFFF6700233882809797FF1F9387F1
:10CDB00067179C43D847A167E5076315F708175322
:10CDC000FFFFE702033479713285328497F0FFFF69
:10CDD000E780C0532AC6228597F0FFFFE7802055E1
:10CDE000228597F0FFFFE78080542310A10222855F
:10CDF00097F0FFFFE780A053520551812311A10254
:10CE000022852302010297F0FFFFE7802050A30252
:10CE1000A102228597F0FFFFE780404F2303A10284
:10CE2000228597F0FFFFE780604EB245A303A10281
:10CE3000280897F0FFFFE780807645611753FFFFD2
:10CE40006700632E82809797FF1F9387A70D9C43EF
:10CE5000D847A1679387E703631FF7001753FFFFC6
:10CE6000E702232A328597000000E78060EB175322
:10CE7000FFFF6700432B82809797FF1F9387870AE6
:10CE80009C43D847A16793874704631EF702175353
:10CE9000FFFFE702032779713285328497F0FFFFA5
:10CEA000E780C0462AC6228597F0FFFFE78020482A
:10CEB000B245280897F0FFFFE780606E4561175381
:10CEC000FFFF6700432682809797FF1F93878705A0
:10CED0009C43D847A167938787026310F7041753D1
:10CEE000FFFFE702032279713285328497F0FFFF5A
:10CEF000E780C0412AC6228597F0FFFFE780004106
:10CF0000B2452300A102280897F0FFFFE7802069BF
:10CF100045611753FFFF6700032182801753FFFF0E
:10CF2000E702231E011197F0FFFFE780203EAA854C
:10CF3000280097F0FFFFE780806605611753FFFF29
:10CF40006700631E9797FF1F9387C7FD9C43D847D1
:10CF5000A167D107631FF7001753FFFFE702631AAA
:10CF6000328597000000E780A0FB1753FFFF6700A2
:10CF7000831B82809797FF1F9387C7FA9C43D847EC
:10CF8000A167C507631FF7001753FFFFE702631789
:10CF9000328597000000E780A0F81753FFFF670075
:10CFA000831882809797FF1F9387C7F79C43D847C2
:10CFB000A167B907631FF7001753FFFFE702631468
:10CFC000328597000000E780A0F51753FFFF670048
:10CFD000831582809797FF1F9387C7F49C43D84798
:10CFE000A167AD07631FF7001753FFFFE702631147
:10CFF000328597000000E780A0F21753FFFF67001B
:10D00000831282809797FF1F9387C7F19C43D8476D
:10D0100089476318F7021753FFFFE702830E0111D8
:10D02000328532C897F0FFFFE780402EAA8528009E
:10D0300097F0FFFFE780A05605611753FFFF6700D9
:10D04000830E82809797FF1F9387C7ED9C43D84735
:10D05000A1678D076311F7041753FFFFE702630A07
:10D0600001113285328497F0FFFFE780202A1306F2
:10D070006100AA844C00228597300000E780C0231D
:10D080002800A68597F0FFFFE780605105611753E0
:10D09000FFFF6700430982809797FF1F9387C7E8C8
:10D0A0009C4381CFDC4391CB1753FFFFE70263051D
:10D0B00082971753FFFF6700030782801753FFFF14
:10D0C000E702230479713C08AE843ED2A165B7071C
:10D0D0000A002A843ED448103C08DD053ED636C4FA
:10D0E00032C63AC297D0FFFFE780E02F12474810C0
:10D0F000BA8597F0FFFFE780C01332464810B2852B
:10D1000097F0FFFFE780E014A2464810B68597F03D
:10D11000FFFFE7800012501001478146A685228557
:10D1200097D0FFFFE780805145611753FFFF6700ED
:10D1300083FF1753FFFFE702C3FC01117C000329A3
:10D14000C501AE843ECAA165B70707002A843ECC5C
:10D1500048087C00C5053ECE97D0FFFFE780A02899
:10D160008345D900480897F0FFFFE780800C5008FE
:10D1700001478146A685228597D0FFFFE780004CB6
:10D1800005611753FFFF670003FA1753FFFFE7021C
:10D1900043F783C7950093F7F707A384F50097003B
:10D1A0000000E78040F91753FFFF6700C3F71753EC
:10D1B000FFFFE70203F579713C08AE843ED2A1651A
:10D1C000B70709002A843ED448103C0893854504DB
:10D1D0003ED632C636C497D0FFFFE780C020A246B5
:10D1E0004810B68597F0FFFFE780A004324648104C
:10D1F000B28597F0FFFFE780C005501001478146D8
:10D20000A685228597D0FFFFE780404345611753ED
:10D21000FFFF670043F11753FFFFE70283EE83C769
:10D22000950041112A8493F7F707A384F50032850E
:10D230002EC697F0FFFFE780800F85672AC46370D2
:10D24000F50297700000E78020E92246B24509ED1B
:10D2500011478146228597000000E78060E6410182
:10D260001753FFFF670023EC01478346F501DDB745
:10D270001753FFFFE70243E701113C003ECAB7071F
:10D280000A003ECC3C003ECE83C79500AA89328579
:10D2900093F7F707A384F5002E8497F0FFFFE7804C
:10D2A00000098567637DF504A165AA8493858504DB
:10D2B000480897D0FFFFE78000132685977000008D
:10D2C000E78080E12A8929E19145480897F0FFFF2E
:10D2D000E78020F6A685480897F0FFFFE78060F713
:10D2E000CA85480897F0FFFFE780A0F40147814610
:10D2F0005008A2854E8597D0FFFFE7802034056156
:10D300001753FFFF670083E18145480897F0FFFF4F
:10D31000E78020F20349090275BF1753FFFFE702B8
:10D32000A3DC79711C103ECAB7070F003ECC404DFC
:10D330001C10AA84AE894808994532C636893ECE6B
:10D3400097D0FFFFE780200A32464808B28597F061
:10D35000FFFFE78000EE630C0902A545480897F03F
:10D36000FFFFE780C0E62546CA8597200100E780D9
:10D3700020A4500801478146CE85268597D0FFFF1F
:10D38000E780C02B45611753FFFF670023D9835502
:10D39000C402480897F0FFFFE780A0EB0355E402C2
:10D3A000814505C5854785456301F502C167FD17C0
:10D3B0009305F00F630BF5007D1597700000E78073
:10D3C000208E9305150093F5F50F480897F0FFFFA1
:10D3D000E78020E683450403480897F0FFFFE780D5
:10D3E00040E583451403480897F0FFFFE78060E4B9
:10D3F00083552403480897F0FFFFE78080E58355B5
:10D400004403480897F0FFFFE780A0E49DB7175357
:10D41000FFFFE70203CF83C795008146014693F7DC
:10D42000F707A384F50097000000E78040EF17534B
:10D43000FFFF670043CF1753FFFFE70283CC7971EB
:10D440003E841C103ECA2E89B7070F00A1653ECC52
:10D45000FD051C10AA84480842C03AC23ECE36C41C
:10D4600032C697D0FFFFE78000F832464808B28501
:10D4700097F0FFFFE780E0DBA2464808B68597F00B
:10D48000FFFFE78000DD12474808BA8597F0FFFFED
:10D49000E78020DC0248630C08029145480897F0B9
:10D4A000FFFFE780C0D21146A28597200100E780E8
:10D4B0002090500801478146CA85268597D0FFFFF6
:10D4C000E780C01745611753FFFF6700C3C5894553
:10D4D000480897F0FFFFE78080CF834704002300D0
:10D4E000F50083471400A300F500E1B71753FFFFD1
:10D4F000E70283BF83C7950001112A8A93F7F707D4
:10D50000A384F5003285AE8432C697F0FFFFE78032
:10D5100000E232462A89328597F0FFFFE78000DF7C
:10D5200085676373F902AA894A8597700000E780CE
:10D53000A0BA2A8419ED114781464A86A6855285EC
:10D5400097000000E780C0B705611753FFFF670031
:10D55000E3BC9387E9FF93F7F70F0547E366F7FE10
:10D560008347F50195EB8947E380F9FE8346F40193
:10D57000528501474A86A68597000000E78040B49F
:10D58000A167D90748083ECC230A010002CE9700C4
:10D590000000E780A0B04DBF639EE7008947639E0F
:10D5A000F90093071020231FF50097700000E78013
:10D5B000C0B76DBF0947E39BE7FA8D47E398F9FAD7
:10D5C000228597700000E78080DF9797FF1F938781
:10D5D000A7B49C4399E79797FF1F9387A79D9C4308
:10D5E00099C703D5040097800000E780A0CE231FD1
:10D5F000040022855DBF1753FFFFE70283B00111CE
:10D600003C003ECAB7070B003ECC3C003ECE83C771
:10D6100095002A89328593F7F707A384F500AE8435
:10D6200097F0FFFFE780A0D093170501C187635AE9
:10D63000F006A1652A849385E502480897D0FFFF8C
:10D64000E78060DAA285480897F0FFFFE78060C0B6
:10D650009797FF1F938707969C43A9EB0144937507
:10D66000F40F480897F0FFFFE780A0BC9355844073
:10D6700093F5F50F480897F0FFFFE78080BB9355BF
:10D68000044193F5F50F480897F0FFFFE78060BA73
:10D69000014781465008A6854A8597D0FFFFE7805D
:10D6A000E0F905611753FFFF6700E3A74165854671
:10D6B0000546A2857D1597500000E78060BD59DDC5
:10D6C000510597000100E780808F13044006334422
:10D6D000850271B71753FFFFE702A3A20111B70735
:10D6E00006003EC683C7950021642A8993F7F70791
:10D6F000A384F500AE8428009305A4040AC40AC8D4
:10D7000097D0FFFFE78020CE300001478146A685F5
:10D710004A8597D0FFFFE78060F297E0FFFFE78040
:10D72000801513049404480822CC230A010002CE79
:10D7300097000000E780809605611753FFFF6700A0
:10D74000839E1753FFFFE702239AC1642A8901448D
:10D750009799FF1F9389C99D130A8002FD1497E0D2
:10D76000FFFFE78080C16347A40001451753FFFF17
:10D770006700C39AB307440303A7C90ABA9703D73C
:10D7800007006306970083D72700638427010504F9
:10D79000F9B70545E1BF1753FFFFE702E3942A8A73
:10D7A0002E8999C123A0050081498144978AFF1FD2
:10D7B000938ACA77614B97E0FFFFE78040C263C757
:10D7C000A4004E851753FFFF67004395338464031D
:10D7D00083A70A003E948357040099E76304090075
:10D7E000232089008504C1BF4146D285130544002A
:10D7F00097100100E780605975F5A289E5B71753C6
:10D80000FFFFE702638E39717C083ED4B7070A0038
:10D810003ED67C083ED883C795002A8A328593F786
:10D82000F707A384F5002E8932C697F0FFFFE78043
:10D8300000B085676373F5083246AA84328597F095
:10D84000FFFFE780A0AC8547AA8963E8A706A1652A
:10D8500093858504281097D0FFFFE780C0B8268500
:10D8600097700000E78040872A8429ED91452810B1
:10D8700097F0FFFFE780E09BA685281097F0FFFF59
:10D88000E780209DCE85281097F0FFFFE780609A03
:10D89000014781463010CA85528597D0FFFFE78047
:10D8A000E0D9A1679387770448183EDC230A010278
:10D8B00002DE97F0FFFFE780607E21611753FFFFD4
:10D8C0006700C3858145281097F0FFFFE7806096C9
:10D8D000A685281097F0FFFFE780A0979797FF1F76
:10D8E000938787BB9C4381CB22856389090097D0AE
:10D8F0000000E78040248345040271B797D0000000
:10D90000E780C022CDBF1743FFFFE702E37D83C757
:10D9100095004111AA8993F7F707A384F500328592
:10D92000AE84328A97F0FFFFE78060A08567637F4F
:10D93000F5022A8997600000E780007A2A849146E0
:10D9400031C58347F50105476387E70291C70D4756
:10D950006366F704AD461DA89305050303250A0079
:10D96000414697100100E78040420DE9410117430D
:10D97000FFFF6700A37A9305950803250A00414637
:10D9800097100100E7806040814669F54A86A685C8
:10D990004E8597000000E780C081C9BF83250A003B
:10D9A0001305940897700000E780A02919C1C146AB
:10D9B000F1BF9787FF1F938727769C4399E7978747
:10D9C000FF1F9387275F9C4399C72285978000009C
:10D9D000E780208A69FD8547A30FF400228597B070
:10D9E0000000E7806084228597600000E780E07394
:10D9F0004E8581464A86A68597F0FFFFE780607BCB
:10DA0000A1679387570448003EC42302010002C661
:10DA100097F0FFFFE780806891BF1743FFFFE702A1
:10DA2000C36B83C795004111AA8993F7F707A384B5
:10DA3000F50032852E89B28A97F0FFFFE780208FAC
:10DA400085676374F50EAA8497600000E780C0685C
:10DA50002A840DED416B014A978BFF1F938B4B6D11
:10DA6000130C400E7D1B19A833048A0383A70B0BEC
:10DA70003E948357C40163836705050A97E0FFFF5F
:10DA8000E780A08EE342AAFE95460DA08357C5010C
:10DA9000639697029305050303A50A004146971074
:10DAA0000100E780802E994611E181462686CA85CD
:10DAB0004E8597F0FFFFE780C06F85A883A50A0019
:10DAC0001305040397700000E780A017C14679FD95
:10DAD0002285231E940097A00000E780E074228531
:10DAE00097600000E78060649797FF1F9387C79A4D
:10DAF0009C43A9C323000402228597D00000E7803D
:10DB000040F04E8581462686CA8597F0FFFFE78064
:10DB1000406AA1679387070448003EC423020100BE
:10DB200002C697F0FFFFE780605741011743FFFFF0
:10DB30006700235E89472300F402E1B7397106DEEE
:10DB400022DC4AD8800052D456D25AD026DA4ED699
:10DB50005ECE2E8A32892A8B97D0FFFFE780E07D48
:10DB60000605710541998A8A3301A140232224FCCC
:10DB7000231404FC97D0FFFFE780207C83479A00A2
:10DB80000605350593F7F7072315A4FCA304FA004F
:10DB90004A85232624FC97E0FFFFE780407993170E
:10DBA0000501C1876340F0025681130104FCF25065
:10DBB0006254D2544259B259225A925A025BF24BE1
:10DBC00021618280AA844A8597E0FFFFE780207662
:10DBD000AA894A8597E0FFFFE7806075A165938574
:10DBE000C5022A89130544FC97C0FFFFE780A07F88
:10DBF000268597C0FFFFE780E073854511C94A86F7
:10DC0000CE8597C0FFFFE780606DAA8B21E989452B
:10DC1000130544FC97E0FFFFE780A061A68513058C
:10DC200044FC97E0FFFFE780C062CE85130544FC0B
:10DC300097E0FFFFE780E061CA85130544FC97E0A9
:10DC4000FFFFE780006101478146130644FCD2854F
:10DC50005A8597D0FFFFE780609EB9B781451305CD
:10DC600044FC97E0FFFFE780C05CA685130544FCF9
:10DC700097E0FFFFE780E05DCE85130544FC97E069
:10DC8000FFFFE780005DCA85130544FC97E0FFFFB6
:10DC9000E780205C814497D0FFFFE780006AE3D4EF
:10DCA000A4FA83A70B0113971400BA9783D5070032
:10DCB00099C5130544FC97E0FFFFE7808059850470
:10DCC000D9BF797106D622D44AD000184ECE52CC94
:10DCD00056CA26D25AC8AE893289AA8A97D0FFFF7F
:10DCE000E780A0650605690541990A8A3301A140CC
:10DCF000232A24FC231C04FC97D0FFFFE780E06369
:10DD000083C7990006052D0593F7F707231DA4FC8B
:10DD1000A384F9004A85232E24FC97E0FFFFE780C7
:10DD2000006193170501C187634FF0005281130111
:10DD300004FDB250225492540259F249624AD24A26
:10DD4000424B45618280AA844A8597E0FFFFE780C5
:10DD5000005EA1659385A5022A89130544FD97C03D
:10DD6000FFFFE7804068268597C0FFFFE780805C63
:10DD7000854509C9CA8597C0FFFFE78020592A8BCE
:10DD800029E18945130544FD97E0FFFFE780604ADC
:10DD9000A685130544FD97E0FFFFE780804BCA8509
:10DDA000130544FD97E0FFFFE780A04A0147814645
:10DDB000130644FDCE85568597D0FFFFE780008887
:10DDC000B5B78145130544FD97E0FFFFE780604646
:10DDD000A685130544FD97E0FFFFE7808047CA85CD
:10DDE000130544FD97E0FFFFE780A046814497D0EC
:10DDF000FFFFE7808054E3DBA4FA83270B0113972E
:10DE00001400BA9783D5070099C5130544FD97E020
:10DE1000FFFFE78000448504D9BF1743FFFFE702F7
:10DE2000432E83474500404DD5EFFD575DC48346E3
:10DE3000940009476363D70A0346B400854663EE3E
:10DE4000C6088306E40063CA06085C45F9562390B9
:10DE5000D7009787FF1F83C7A70D99E3A304E400AA
:10DE60009787FF1F938707159C4381E78947A30680
:10DE7000F4009787FF1F938727629C4381E78947B8
:10DE80002306F4009705000093854506AA84130530
:10DE9000040197F00000E7802010FD57231AF402D8
:10DEA00081471CDC01489787FF1F23AF87069787B0
:10DEB000FF1F9387A707232E040304C0804397D036
:10DEC000FFFFE780C05161463306C50281452285C8
:10DED0009740FFFFE780E02581473E851743FFFF1E
:10DEE00067006324FD57D5BF1743FFFFE702632197
:10DEF0002A840355450297600000E780E01D19E57C
:10DF0000231E04001743FFFF6700E3218357E4014A
:10DF1000F5DB930504FF174501001305A57397E092
:10DF20000000E780E014F9BF1743FFFFE702631D1D
:10DF30002E89A16541119385E5032A8436C432C632
:10DF4000BE843AC297C0FFFFE780E04912472285AE
:10DF5000BA8597E0FFFFE780C02D32462285B28563
:10DF600097E0FFFFE780E02EA2462285B68597E086
:10DF7000FFFFE780002E630309029145228597E0A9
:10DF8000FFFFE780C0241146A68597100100E780B7
:10DF900020E241011743FFFF6700E318894522850E
:10DFA00097E0FFFFE780A02283C704002300F5006D
:10DFB00083C71400A300F500E9BF1743FFFFE70282
:10DFC000431483C79500444D054793F7F707A3848F
:10DFD000F5001C42411183C707006367F7062E84D2
:10DFE0002A89B1C003C7D400630FF7021787FF1F48
:10DFF000130747FC184305C3A386F40097A000004D
:10E00000E780404A83C7D40099E741657D15974072
:10E010000000E780403083D72403918B89C797E0C5
:10E020000000E780C0134A85A28597F0FFFFE780D4
:10E030008010A167C10748003EC42302010002C648
:10E0400097F0FFFFE780800541011743FFFF67005E
:10E05000830D1743FFFFE702C30A03D745008D472F
:10E06000AA8441112E8432892E8563E3E70297E06A
:10E07000FFFFE780C02BAA8523000900268597C0F3
:10E08000FFFFE780A02841011743FFFF6700A309B6
:10E0900097E0FFFFE780A0292AC6228597E0FFFFCF
:10E0A000E780E028B24585472A862300F9002685C7
:10E0B00097C0FFFFE7808022F9B7397106DE22DCC6
:10E0C00026DA80004ED652D456D24AD85AD05ECEE6
:10E0D000AE89B284AA8A97D0FFFFE78000250605A3
:10E0E0001305250241990A8A3301A140232224FC09
:10E0F000231404FC97D0FFFFE780202383C79900F7
:10E1000006054D0593F7F7072315A4FCA384F90032
:10E110002685232624FC97E0FFFFE7804021931704
:10E120000501C1876340F0025281130104FCF250E3
:10E130006254D2544259B259225A925A025BF24B5B
:10E1400021618280AA8B03AB040097C0FFFFE780A8
:10E15000601E51E583D7440001498544F11793B708
:10E160001700A301F4FC834734FCA165C9C793855C
:10E17000E504130544FC97C0FFFFE780C026A68591
:10E18000130544FC97E0FFFFE780A00ADE85130536
:10E1900044FC97E0FFFFE780C00B834734FC114647
:10E1A00091E30946DA85130544FC97E0FFFFE78019
:10E1B00060058144630A0900416B7D1B97D0FFFF16
:10E1C000E780A01663CCA40201478146130644FCF5
:10E1D000CE85568597C0FFFFE7804046B1B7A6853C
:10E1E000130634FC97000000E780E0E69334150046
:10E1F0002A8986048DBF9385C504A5BF8327C900DE
:10E2000013971400BA9783D5070063886501130537
:10E2100044FC97E0FFFFE780C003850445B7174340
:10E22000FFFFE70283EB79711C103EC4B7070F00B4
:10E230003EC61C103EC883C79500AA8A328593F754
:10E24000F707A384F500AE89328497E0FFFFE780EB
:10E25000000E93170501C187635AF0062A8A2285AA
:10E2600097E0FFFFE780A00C2A895285032B04006A
:10E2700097C0FFFFE780000C39ED835744008144CD
:10E280000544F11793B71700A303F100834571000C
:10E29000DA872287CA865286280097000000E78026
:10E2A000E0C8014781463000CE85568597C0FFFF04
:10E2B000E780C038A1679387D70348083ECC230A7C
:10E2C000810026CE97F0FFFFE78040DD45611743D0
:10E2D000FFFF670003E4A2851306710097000000AA
:10E2E000E78060D7AA84094455D13544E30055FB43
:10E2F0004A8597F0FFFFE78000450D4441D901446E
:10E3000097D0FFFFE7806002634DA400C16B01441A
:10E31000FD1B97D0FFFFE7804001634EA40015442A
:10E32000B5B7DC4413171400BA9783D7070063838B
:10E3300027030504F1B7D84493171400BA9703D7FD
:10E340000700631B770123902701268597A0000013
:10E35000E78080DB01441DBF050465BF1743FFFF55
:10E36000E70283D883C7950041112A8A93F7F707FC
:10E37000A384F50032852E89328497E0FFFFE78081
:10E3800000FB93170501C1876353F006AA89228514
:10E3900097E0FFFFE780A0F92311A1004E85832AB3
:10E3A000040097C0FFFFE780E0F839E58357440099
:10E3B00085440144F11793B71700A300F100034807
:10E3C000110003572100D6875285CE862686CA853E
:10E3D00097F0FFFFE7806006A167F10748003EC4A1
:10E3E0002302910022C697F0FFFFE78020CB410176
:10E3F0001743FFFF670083D2A28513061100970021
:10E400000000E78040C52A84894455D983572100FC
:10E4100011678544BA97C2071167C1831307F7EFE5
:10E42000E36FF7F89787FF1F938707CF9C4381CB54
:10E4300085451305210097500000E780207583551E
:10E4400021002285814497C0FFFFE78040E525D960
:10E4500023100500228597A00000E78040CD85B7F6
:10E460001743FFFFE70263C783C7950041112A8B5B
:10E4700093F7F707A384F50032852E8A328497E05C
:10E48000FFFFE780C0EA93170501C1876351F006DB
:10E49000AA8A228597E0FFFFE78060E92A895685EE
:10E4A000832B040097C0FFFFE780C0E831E5835766
:10E4B000440081440544F11793B71700A301F1000C
:10E4C00003483100DE875A854A87D6862286D28560
:10E4D00097F0FFFFE78060F6A167ED0748003EC4B4
:10E4E0002302810026C697F0FFFFE78020BB410191
:10E4F0001743FFFF6700E3C1A285130631009700B1
:10E500000000E78040B5AA8409445DD99167CA97A5
:10E51000C2071167C1831307F7EF0544E362F7FAF7
:10E52000CA8597C0FFFFE78080D7014451F9814930
:10E5300097D0FFFFE78060E063DBA90098489397DE
:10E540001900BA9703D7070005EF2390270197D04A
:10E55000FFFFE78080DE1544E384A9F6268597A0B7
:10E560000000E780C0BC9787FF1F9387E7BA9C43F2
:10E570000144B9D74A8597500000E780C05889B751
:10E5800085097DB71743FFFFE70203B679713E8423
:10E590007C083EC82E8AB7071400A1653ECAE5056F
:10E5A0007C08AA89080836C4428932C6BA8AC68459
:10E5B0003ECC97C0FFFFE78000E3CA85080897E0DC
:10E5C000FFFFE78000C732460808B28597E0FFFFEB
:10E5D000E78020C8A246630A09049D45080897E021
:10E5E000FFFFE780C0BE1D4681459740FFFFE780E3
:10E5F00040B463890A089145080897E0FFFFE78067
:10E6000000BD1146A68597000100E780607A1008DA
:10E6100001478146D2854E8597C0FFFFE780000203
:10E6200045611743FFFF670063AFB685080897E0B1
:10E63000FFFFE78000C21C400808D8439355C7017C
:10E64000858912075183B205D98D97E0FFFFE780D6
:10E6500040C01C40080883C5870097E0FFFFE780A3
:10E6600040BD1C40080883C5A70097E0FFFFE78076
:10E6700040BC1C40080883C5970097E0FFFFE78077
:10E6800040BB85BF8945080897E0FFFFE78020B4BD
:10E6900083C704002300F50083C71400A300F5001E
:10E6A000BDB71743FFFFE70223A483C795004111BD
:10E6B000AA8993F7F707A384F5003285AE843284E4
:10E6C00097E0FFFFE780A0C693170501C187635D50
:10E6D000F0042A89032A040097C0FFFFE78080C561
:10E6E00019E9835744000548F11793B71700A307AA
:10E6F000F100814631A81306F100A28597000000C1
:10E70000E78060951DC51C459DC783D6470001481D
:10E710000347F10093078500D2884A86A6854E8577
:10E7200097000000E78040E641011743FFFF6700C4
:10E73000E39E09487DBF1D486DBF1743FFFFE702F9
:10E74000A39A65715C083EC4B7077B013EC65C08AE
:10E750003EC883C795002A8A328593F7F707A384BA
:10E76000F500AE8997E0FFFFE78040BA8357E100EC
:10E77000E1C78945280097C0FFFFE780C0C68145F3
:10E78000280097E0FFFFE780C0AA97C0FFFFE7805F
:10E79000A0CC9787FF1F938727D09C431774FF1F38
:10E7A00003440479AA843334800099C31364240099
:10E7B0009787FF1F938707809C4399C31364440086
:10E7C0009787FF1F938747959C4399C313648400E1
:10E7D00083D504002800014997E0FFFFE78060A788
:10E7E00083D52400280097E0FFFFE78080A683D52B
:10E7F0004400280097E0FFFFE780A0A597D0FFFF27
:10E80000E780A0AE93150501C181280097E0FFFFC6
:10E81000E78020A4A285280097E0FFFFE78060A39F
:10E820009C446360F902014781463000CE855285E1
:10E8300097C0FFFFE78080E059611743FFFF670043
:10E84000E38DDC441314490028003E9497E0FFFF59
:10E85000E780609683474400034754008907060712
:10E86000BA978607E36AF5FC835524002800814A9D
:10E8700097E0FFFFE780E09D83454400280097E094
:10E88000FFFFE780009B83455400280097E0FFFFCF
:10E89000E780209A8347440063C9FA00814A83478E
:10E8A000540063C1FA020509A5BF1C4413975A001E
:10E8B0002800BA9783D50700850A97E0FFFFE78015
:10E8C0004099C9BF032BC40093975A0028003E9B70
:10E8D00083552B00850A97E0FFFFE78080978355DB
:10E8E0000B00280097E0FFFFE780A0964DBF17437D
:10E8F000FFFFE70203815C4993E717005CC997A01B
:10E900000000E78020B61743FFFF6700C38117337D
:10E91000FFFFE702037F2E84814597F0FFFFE7802A
:10E92000C0E705C583570500FD172310F50009C48E
:10E93000835725002310F40097000000E78060FB58
:10E9400001451733FFFF6700037E31457DD8231053
:10E950000400C5BF1733FFFFE702037983C79500A3
:10E9600041112A8A93F7F707A384F50032852E898F
:10E97000328497E0FFFFE780809B93170501C187F2
:10E980006356F006AA89C145228597E0FFFFE7801C
:10E99000A0802A8B4E85832A040097C0FFFFE78062
:10E9A000609931E983574400231101000544F117B0
:10E9B00093B71700A300F1008144034811000357E7
:10E9C0002100D6875285CE862286CA8597F0FFFF22
:10E9D000E780A0A6A1679387170248003EC42302E0
:10E9E000810026C697E0FFFFE780406B41011733A7
:10E9F000FFFF6700A37213061100A28597F0FFFFC7
:10EA0000E7806065AA8409E523110100094475B710
:10EA1000930521005A8597000000E78080EF835717
:10EA200021002A84D9DB9777FF1F9387E76E9C43E9
:10EA300081CB85451305210097500000E780001524
:10EA4000835521002685314497C0FFFFE78020854C
:10EA50002DD523100500268597900000E780206DB6
:10EA60000144A1BF1733FFFFE702A36941112E89BB
:10EA70006C00AA8402C697F0FFFFE78000D20DC1A8
:10EA80000357050005072310E50097000000E78005
:10EA900040E681473E8541011733FFFF6700A368C9
:10EAA0003247954765DBCA85268597300000E780A9
:10EAB000400DC147E34005FE3244854741462310DF
:10EAC000F40083570900A685130544002311F400C0
:10EAD00097000100E780C02D228545BF1733FFFF57
:10EAE000E702836083C795004111AA8A93F7F7076D
:10EAF000A384F5003285AE89328497E0FFFFE7807A
:10EB0000008393170501C1876356F0062A8AC14521
:10EB1000228597D0FFFFE7802068AA845285032BC7
:10EB2000040097C0FFFFE780E08031E9835744008D
:10EB3000231101008544F11793B71700A300F100DA
:10EB400001440348110003572100DA875685D28615
:10EB50002686CE8597F0FFFFE780208EA1679387FA
:10EB6000070248003EC42302910022C697E0FFFF3F
:10EB7000E780C05241011733FFFF6700235AA28587
:10EB80001306110097F0FFFFE780E04C2A8409E5A7
:10EB900023110100894475B726859305210097004C
:10EBA0000000E78060ECAA8449FD8355210022859E
:10EBB00097B0FFFFE780A06E49F5014997C0FFFFBE
:10EBC000E780A077635DA900184893171900BA97EA
:10EBD00003D707000DEF035721002390E70097C0EC
:10EBE000FFFFE7808075630625039777FF1F9387F4
:10EBF000A7529C4399C70355210097500000E78016
:10EC000080F0228597900000E78060521DBF0509C3
:10EC100075B795443DB705C19307F00F630FF50035
:10EC2000C547630CF5009307F5FF05453315F5005F
:10EC30004205418182800145828041657D15828047
:10EC4000B9E91733FFFFE702C34B034506033284DC
:10EC500097000000E78060FC9305803EB305B50295
:10EC6000C205C18181CD0357E402854763F8E700FF
:10EC70001305040197E00000E78020428357E40277
:10EC800041677D176385E700FD172317F4021733EB
:10EC9000FFFF6700434982801733FFFFE702E3432A
:10ECA000004283C79500444D0349140093F7F707CA
:10ECB000A384F50083470400220911673369F90032
:10ECC000A167B347F90041112A8BAE8A63ECE70EC6
:10ECD000834724001307C00EB91793F7F70F637328
:10ECE000F71003473400C14763EEE70E8347440043
:10ECF0001307E00793C707086371F70C8349840083
:10ED000083477400A209B3E9F900856763F7F90A3C
:10ED1000034A6400834754004E85220A336AFA008E
:10ED200097500000E780403B61C123962403834B4A
:10ED30003400137AFA00239A340323887403239946
:10ED4000440393890401631C090023A60402239849
:10ED500004024E8597E00000E78060363DA003493D
:10ED600024004A8597000000E78020EB2397A40247
:10ED7000834744004E85A388F402E38D0BFCE30B2C
:10ED800009FC97E00000E780202F97900000E780C3
:10ED9000007381460146D6855A8597E0FFFFE780DC
:10EDA0000058A167938797033EC4230201004800DF
:10EDB00002C697E0FFFFE780602E41011733FFFF97
:10EDC000670023358544A2862686D6855A8597E036
:10EDD000FFFFE780C054A167938797033EC42302D7
:10EDE0009100F1B7BD44C5B79144F1BF1733FFFFA0
:10EDF000E702832F01111C08404D3EC2B7070F00E8
:10EE00003EC41C083EC62A89AE8997C0FFFFE78032
:10EE1000A0DA585C1C5C6346B70E6394E50063E2BD
:10EE2000A70E3385A740B3B7A700B305B7401306B5
:10EE3000803E81469D8D97000100E78080B7931446
:10EE40000501C180A1659385C503480097B0FFFF08
:10EE5000E78060598145480097D0FFFFE780603D1B
:10EE600083550404480097D0FFFFE780803E835518
:10EE70002404480097D0FFFFE780A03D814589CC5E
:10EE8000C167FD179305F00F6388F400268597503E
:10EE90000000E780E0E0AA85480097D0FFFFE78008
:10EEA000403903554404814501CDC167FD179305E1
:10EEB000F00F6307F50097500000E78060DEAA8539
:10EEC000480097D0FFFFE780C036834564044800C0
:10EED00097D0FFFFE780E03583457404480097D062
:10EEE000FFFFE7800035500001478146CE854A8507
:10EEF00097B0FFFFE780807405611733FFFF67005D
:10EF0000E321814481B71733FFFFE702831F83C7E3
:10EF1000950093F7F707A384F50097000000E780BA
:10EF200020ED1733FFFF670003201733FFFFE702D1
:10EF3000A31B83C795004111404D93F7F707A384A6
:10EF4000F5002A8A3285B284AE8997D0FFFFE78028
:10EF5000003E2A8B268597D0FFFFE780403D2A8917
:10EF6000268597D0FFFFE780603A93170B0163CAAD
:10EF70000702E177CA97C207C183116763E3E7021B
:10EF800093070910C207C1831307B00F637BF70013
:10EF900093170901C187AA8A634AF000C54763FE37
:10EFA000570141011733FFFF6700431797B0FFFF79
:10EFB000E780C028E31725FFD5B763080B02630677
:10EFC0000902814463890A02B7077F0023106405A0
:10EFD000231124057CC0568597000000E780E0C31C
:10EFE0009304803EB304950239A0B7077F00232025
:10EFF00004047CC081440355240497E00000E780AA
:10F00000A0A3A1C497C0FFFFE78000BB269593D7BC
:10F01000F44133379500AE97BA9708DC5CDCCE85B7
:10F02000528597000000E780A0DC99E023220404C9
:10F03000A1679387B70348003EC42302010002C6BC
:10F0400097E0FFFFE7808005A9BF814701481CDCEE
:10F05000232E0403E9B71733FFFFE702830A97C0A3
:10F06000FFFFE780C037E1473305F5029145975030
:10F070000000E78000C5E55711C59777FF1F23A75C
:10F08000A7EA81473E851733FFFF6700C30985471D
:10F090001777FF1F230EF7E882801733FFFFE70281
:10F0A00043069777FF1F938727E880433DC0835728
:10F0B00004046390A70683572404639CB70436892D
:10F0C000B28497C0FFFFE78020AF5C5C63C3B704E6
:10F0D0006395B7001C5C63EEA7028347640463F387
:10F0E000F400A6872303F4048347740463F39700B2
:10F0F000A687A303F4048357440441677D176385FF
:10F10000E70085072312F4043C4481C7CA8526859D
:10F1100082971733FFFF670003019777FF1F9387DD
:10F12000A7E09C43014599C303C58700828017333C
:10F13000FFFFE70203FD0111B70707003EC683C7C3
:10F140009500584D0AC493F7F7070AC8A384F50041
:10F150002A89AE8411CB1C4283C707002304F70021
:10F1600097900000E7800034216493055402280042
:10F1700097B0FFFFE780202797000000E78020FA84
:10F18000AA85280097D0FFFFE780A00A300001473A
:10F190008146A6854A8597B0FFFFE780204A130481
:10F1A0004402480822CC230A010002CE97E0FFFF68
:10F1B000E780C0EE05611733FFFF6700C3F6173322
:10F1C000FFFFE70203F401117C003ECAB707070006
:10F1D0003ECC7C003ECE83C795002E84AA8493F754
:10F1E000F707A384F500A16593855502480897B0F9
:10F1F000FFFFE780401F97000000E78040F2AA85EC
:10F20000480897D0FFFFE780C002500801478146B9
:10F21000A285268597B0FFFFE7804042056117333E
:10F22000FFFF670043F09777FF1F9387E7CF9C436B
:10F23000094599C303C5970082809777FF1F93877D
:10F24000A7CE9C43094599C303C5D7008280977711
:10F25000FF1F938767CD9C43014599C303C5A70052
:10F2600082801733FFFFE70223E80111B707080088
:10F270003EC683C79500404D0AC493F7F7070AC8F6
:10F28000A384F5002A89AE8429C41442854703C7A4
:10F29000060063E0E70A83479400094681496380DA
:10F2A000C702B307F740A304E400B339F00083C7F3
:10F2B00016002305F40097900000E780A01E035776
:10F2C0002403058B19C76386090097D00000E780E7
:10F2D00000E9216493058402280097B0FFFFE780CE
:10F2E000801097000000E78040F4AA85280097D09E
:10F2F000FFFFE78000F497000000E78080F5AA8513
:10F30000280097D0FFFFE780C0F201478146300018
:10F31000A6854A8597B0FFFFE78040321304740248
:10F32000480822CC230A010002CE97E0FFFFE780C5
:10F33000E0D605611733FFFF670043DE1733FFFF99
:10F34000E70223DC01117C003ECAB70708003ECC6F
:10F350007C003ECE83C795002E84AA8493F7F707DE
:10F36000A384F500A16593858502480897B0FFFF47
:10F37000E780600797000000E78020EBAA85480837
:10F3800097D0FFFFE780E0EA97000000E78060EC9D
:10F39000AA85480897D0FFFFE780A0E950080147F9
:10F3A0008146A285268597B0FFFFE7802029056169
:10F3B0001733FFFF670023D79777FF1F9387C7B6E1
:10F3C0009C43014599C303C5B70082801733FFFFF3
:10F3D000E70223D30111B70707003EC683C7950094
:10F3E000404D0AC493F7F7070AC8A384F5002A8999
:10F3F000AE8405C81C42054783C707006368F7064B
:10F400000347B400630FF700A305F40097900000D2
:10F41000E78040098347B400B9CF97D0FFFFE7806A
:10F4200040BE21649305B400280097B0FFFFE78039
:10F4300080FB97000000E78060F8AA85280097D03D
:10F44000FFFFE78000DF014781463000A6854A853F
:10F4500097B0FFFFE780801E2904480822CC230ACA
:10F46000010002CE97E0FFFFE78040C3056117333C
:10F47000FFFF670043CB97D0FFFFE78020BF55B762
:10F480001733FFFFE702E3C701117C003ECAB7074D
:10F4900007003ECC7C003ECE83C795002E84AA8414
:10F4A00093F7F707A384F500A165AD05480897B069
:10F4B000FFFFE78040F397000000E78020F0AA8577
:10F4C000480897D0FFFFE780C0D650080147814623
:10F4D000A285268597B0FFFFE780401605611733A8
:10F4E000FFFF670043C49777FF1F9387E7A39C4301
:10F4F000094599C303C5C70082801733FFFFE702A0
:10F5000043C001117C00AE843ECAA165B707070065
:10F510002A843ECCD1057C0048083ECE97B0FFFF40
:10F52000E78060EC97000000E78020FCAA8548088F
:10F5300097D0FFFFE780E0CF500801478146A685BE
:10F54000228597B0FFFFE780600F05611733FFFF4B
:10F55000670063BD1733FFFFE702A3BA83C79500B7
:10F5600093F7F707A384F50097000000E78020F9E0
:10F570001733FFFF670023BB1733FFFFE702C3B654
:10F5800083C795000329C501411193F7F707A384A9
:10F59000F5001C4283C90700854763E63707977764
:10F5A000FF1F938767EF9C432E84AA8485CF970023
:10F5B0000000E78080F389476306F50263040902CF
:10F5C0008347C90063803703230639019790000001
:10F5D000E78040ED83572903898B89C797D00000C6
:10F5E000E780E0B72685A28597000000E78020F13C
:10F5F000A167CD0748003EC42302010002C697E080
:10F60000FFFFE780A0A941011733FFFF670003B1A7
:10F610009777FF1F938747919C431D4599C303C567
:10F62000E70082801733FFFFE702A3AD0111B707A0
:10F6300007003EC683C79500584D0AC493F7F707E5
:10F640000AC8A384F5002A89AE8415C71C4283C763
:10F65000070093968701E18663C4060685466381A9
:10F66000D7068346E7006388F6002307F7009790E4
:10F670000000E78020E321649305E400280097B0B0
:10F68000FFFFE78040D697000000E780A0F8AA853A
:10F69000280097D0FFFFE780C0B9014781463000BE
:10F6A000A6854A8597B0FFFFE78040F935044808F2
:10F6B00022CC230A010002CE97E0FFFFE780009EE4
:10F6C00005611733FFFF670003A61733FFFFE7024B
:10F6D00043A301117C003ECAB70707003ECC7C0063
:10F6E0003ECE83C795002E84AA8493F7F707A384A0
:10F6F000F500A165B905480897B0FFFFE780A0CEE7
:10F7000097000000E78000F1AA85480897D0FFFF26
:10F71000E78020B2500801478146A285268597B030
:10F72000FFFFE780A0F105611733FFFF6700A39F8C
:10F730001733FFFFE702439BAA8401441769FF1FA9
:10F740001309C97EE14997C0FFFFE78040C96344C0
:10F75000A400014519A833053403832709003E9509
:10F76000835725006397970011051733FFFF670044
:10F77000E39A0504C9BF032E8500630A0E121773AE
:10F78000FF1F130363990323030063150300294339
:10F790006390061203234E01631503001D43639912
:10F7A00007101733FFFFE7024393C689428A3E8959
:10F7B000BA8AB684328BAE8B2A84B5E103554E00EB
:10F7C00019E501431A851733FFFF67008394A1678A
:10F7D000A98F116763FBE70097000000E78080F5C1
:10F7E000814597F0FFFFE780C0120844B70700E0AB
:10F7F0005841F98F18455CC1B707001FF98F1CC528
:10F800005C4991C7610597E00000E780408BE38A7F
:10F8100009FA228597900000E78060C65DB73285BF
:10F8200097C00000E78040430D4349DD1C44116749
:10F8300003D54700A167A98F63FBE700970000008D
:10F84000E78040EF814597F0FFFFE780800C0323BE
:10F85000840093164B01D1828347B30003566300A3
:10F860008588FD8BA305F300FD777D8E558EFD7693
:10F87000FD16B204F18E83274301C58E2312730156
:10F880002313D3002304530123052301A3044301BD
:10F89000BDDF228597B0FFFFE78020CDAA85084411
:10F8A000B5D1610597D00000E780207F8DB71D435B
:10F8B0001A8582801733FFFFE70203830569AA8454
:10F8C000AE89328A0144FD5A7D1997C0FFFFE78057
:10F8D000C0A56347A40001451733FFFF67000384F9
:10F8E000D84493171400BA9703D70700631F370350
:10F8F0002390570163070A00268597900000E78050
:10F90000A0809C449DC383D76700B3F72701639E03
:10F910003701D28801488147014781460146814528
:10F92000268597000000E78040E5050479BF17238E
:10F93000FFFFE702637B79711C103EC4B7070F001D
:10F940003EC61C103EC883C79500AA8A328593F72D
:10F95000F707A384F5002E89328497D0FFFFE78054
:10F96000009D93170501C187635AF006AA89228575
:10F9700097D0FFFFE780A09B2A8A4E85032B0400C7
:10F9800097B0FFFFE780009B39ED83574400814427
:10F990000544F11793B71700A303F10083457100E5
:10F9A000DA872287D2864E86280097E0FFFFE7801D
:10F9B000E057014781463000CA85568597B0FFFF62
:10F9C000E780C0C7A1679387F70348083ECC230AA6
:10F9D000810026CE97D0FFFFE780406C456117235A
:10F9E000FFFF6700A373A2851306710097E0FFFF76
:10F9F000E7806066AA84094455D1528597E0FFFFED
:10FA0000E78060D40D4459D90546D28526859700F4
:10FA10000000E78060EA2A8451B71723FFFFE7025E
:10FA2000436E835507000346270041112A842E8523
:10FA300032C62EC497E0FFFFE780E0D001C932460E
:10FA4000A245228597000000E78000E741011723C7
:10FA5000FFFF6700436D1723FFFFE702036883C7BB
:10FA600095004111AA8A93F7F707A384F500328520
:10FA7000AE89328497D0FFFFE780608B9317050132
:10FA8000C1876357F00AC1452A8A228597C0FFFFC4
:10FA9000E78080702A8D228597D0FFFFE78020893C
:10FAA0002A89228597D0FFFFE7804086930705F8D3
:10FAB00093F7F70F1307E007AA8B637BF7062285FE
:10FAC00097D0FFFFE78080842A8C228597D0FFFFA4
:10FAD000E780C083AA8C5285032B040097B0FFFFF8
:10FAE000E780408539E983574400231101008144B0
:10FAF000F11793B71700A300F10005440347110065
:10FB000083562100938784005685DA88228852869E
:10FB1000CE8597F0FFFFE78020A7A167E90748009F
:10FB20003EC42302810026C697D0FFFFE78000571E
:10FB300041011723FFFF6700C35D13061100A28573
:10FB400097E0FFFFE7802051AA8409E52311010017
:10FB500009446DB7930521006A8597F0FFFFE780A0
:10FB6000A0F02A8441FD835521009356C900131645
:10FB7000490185486688E2875E87858A51822685A5
:10FB800097000000E78060BF2A848DBF1723FFFF26
:10FB9000E702A35483C7950041112A8B93F7F70717
:10FBA000A384F5003285AE89328497C0FFFFE780D9
:10FBB000007893170501C1876352F00A2A8A2285CB
:10FBC00097C0FFFFE780A076AA8A228597C0FFFF33
:10FBD000E780E0752A89228597C0FFFFE7800073E0
:10FBE000930705F893F7F70F1307E0072A8C63775D
:10FBF000F706228597C0FFFFE7804071AA8C228517
:10FC000097C0FFFFE78080702A8D5285832B040008
:10FC100097A0FFFFE780007239E5835744008544D1
:10FC20000144F11793B71700A301F1000347310016
:10FC3000930784005A85DE882688D6865286CE852C
:10FC400097F0FFFFE78040948D4748003EC42302B1
:10FC5000910022C697D0FFFFE7804044410117235F
:10FC6000FFFF6700034BA2851306310097E0FFFFFB
:10FC7000E780603E2A84894455D99356C9001316FB
:10FC8000490185486A88E6876287858A5182D685D8
:10FC900097000000E78060AEAA8449BF1723FFFFEA
:10FCA000E70283442A8981440144617A916A176B8F
:10FCB000FF1F130B6B4697B0FFFFE780006863C719
:10FCC000A40022851723FFFF67004345832709000F
:10FCD00093991400CE9703D50700330745014207D7
:10FCE00041836364570305C103270B0019C785458A
:10FCF0003E8597400000E78060E9832709000504FE
:10FD0000CE972390070085047DB797000000E78019
:10FD100060A2832709000504CE972390070065D5CC
:10FD2000814597F0FFFFE780C0BEF1BF1723FFFFBB
:10FD3000E702833B83C7950041112A8A93F7F707AF
:10FD4000A384F50032852E89328497C0FFFFE780B7
:10FD5000005E93170501C187635AF004AA89832ABC
:10FD6000040097A0FFFFE780E05C31E58357440083
:10FD700085440144F11793B71700A301F10003482C
:10FD80003100D68752850147CE862686CA8597D010
:10FD9000FFFFE780806AA167F50748003EC42302A1
:10FDA000910022C697D0FFFFE780402F4101172323
:10FDB000FFFF6700A336A2851306310097E0FFFF1F
:10FDC000E78060292A8489445DD99767FF1F93875C
:10FDD000A7349C4381CF044997B0FFFFE780E055EB
:10FDE000AA85268597400000E78040DA13050401C4
:10FDF00097000000E780C0EA228597800000E78036
:10FE000000338144ADBF1723FFFFE702032D83C7F3
:10FE100095004111AA8A93F7F707A384F50032856C
:10FE2000AE8932842311010097C0FFFFE780205084
:10FE300093170501C1876354F0062A8AC1452285BC
:10FE400097C0FFFFE7804035AA8B5285032B040043
:10FE500097A0FFFFE780004E21E9835744008544C7
:10FE60000144F11793B71700A300F10003481100F4
:10FE700003572100DA875685D2862686CE8597D00D
:10FE8000FFFFE780805BA1679387270248003EC49D
:10FE90002302910022C697D0FFFFE7802020410176
:10FEA0001723FFFF6700E326A2851306110097E0E2
:10FEB000FFFFE780401A2A8489444DD99767FF1FC6
:10FEC0009387872598433E8901CF044997B0FFFF68
:10FED000E780A046AA85268597400000E78000CBF2
:10FEE0001305040197000000E78080DB97B0FFFF57
:10FEF000E780A04495443DD9930521005E8597F0A5
:10FF0000FFFFE78060B6AA8435F11C480357210043
:10FF100022852390E70097800000E7804021832717
:10FF20000900A9D70355210097400000E780A0BD34
:10FF300035BF1723FFFFE702431A83C7950041111E
:10FF4000AA8A93F7F707A384F5003285AE89328435
:10FF500097C0FFFFE780A03D93170501C18763515C
:10FF6000F0062A8A228597C0FFFFE780403C2A8955
:10FF70005285032B040097A0FFFFE780A03B31E5EB
:10FF80008357440085440144F11793B71700A30138
:10FF9000F10003483100DA8756854A87D2862686E3
:10FFA000CE8597D0FFFFE7804049A167F907480059
:10FFB0003EC42302910022C697D0FFFFE780000EC7
:10FFC00041011723FFFF6700C314A2851306310008
:10FFD00097E0FFFFE78020082A8489445DD9916774
:10FFE000CA97C2071167C1831307F7EF8544E3621D
:10FFF000F7FA9767FF1F938727129843BE8B01CFAD
:020000040001F9
:10000000044997B0FFFFE7804033AA8526859740D3
:100010000000E780A0B71305040197000000E78007
:1000200020C897B0FFFFE780403195443DD11C4880
:10003000228581442390270197800000E780200FCC
:1000400083A70B00B9D74A8597400000E780A0AB93
:1000500089B71723FFFFE702C30A2A844105B28448
:1000600097000000E780C0C311C52285978000007B
:10007000E780E00B81460146A68522859780000037
:10008000E780C04E1C4C89C7DC4799C32285829704
:100090001723FFFF670023099767FF1F9387C7E8B0
:1000A0009C43014599C31385070182809767FF1F11
:1000B000938787E7884382801723FFFFE702630463
:1000C0009317C600DD8DC2054111C1812A8432C655
:1000D00097C0FFFFE780E0173246228511829375B3
:1000E000F60F97C0FFFFE780C01441011723FFFF01
:1000F000670063031723FFFFE70203FF79713C08E2
:100100003ED2B7070C003ED43C083ED683C79500CC
:10011000AE842A8993F7F707A384F500A165938538
:100120003504481097A0FFFFE780E02BC165FD155F
:100130000144176AFF1F130AAAFF930A400EAE89F3
:100140002E8B2EC697B0FFFFE78020224205931723
:1001500004014181C183B24563E9A702C167FD176C
:100160006387F500481097C0FFFFE780800E5010AE
:1001700001478146A6854A8597A0FFFFE780004C8E
:1001800045611723FFFF670063F933075403832793
:100190000A0BBA9703D6C701630A3601638A350191
:1001A000481097000000E78060F1DA85050451BF30
:1001B000B285EDBF1723FFFFE70223F279717C08B8
:1001C0003EC8B70711003ECA7C083ECC83C79500E5
:1001D000AA89328593F7F707A384F5002E8997C083
:1001E000FFFFE780C01485676378F504A165AA84E2
:1001F0008905080897A0FFFFE780E01E2685974045
:100200000000E78060ED133415000A04A285080899
:1002100097C0FFFFE780E001A685080897C0FFFFB1
:10022000E780200325CC014781461008CA854E850A
:1002300097A0FFFFE780804045611723FFFF67001D
:1002400043EDB30754030327CA0ABA9703D707003D
:10025000631C970003D62700638065050808970094
:100260000000E780A0E5DE8505042EC697B0FFFFFD
:10027000E780A0104205931704014181C183B24574
:10028000E3E1A7FCC167FD17E38FF5F8080897C005
:10029000FFFFE78000FC41BFB285F9B7C165FD15DE
:1002A0000144176AFF1F130AAAE8930A80022E8BE3
:1002B000AE8B65BF1723FFFFE702A3E41841834716
:1002C000170083460700A207D58FD207D18323905A
:1002D000F50083472700034717008D45A207D98FF4
:1002E00091832310F60097C0FFFFE780A0E9172352
:1002F000FFFF670043E31723FFFFE702E3DEC1646C
:1003000001441769FF1F1309A9E293098002FD1434
:1003100097B0FFFFE78060066347A40001451723FD
:10032000FFFF6700A3DF330534038327C90A3E9527
:1003300083570500E38597FE0504D9BF1723FFFF08
:10034000E70283DA2A8AAE89B284B68A974000002F
:10035000E78080D819E591473E851723FFFF6700A6
:10036000E3DB2A894E8597C00000E780E08E2A846F
:10037000638E0A048D476DD103570500C547E31D01
:1003800047FD0347F9018546AD47E317D7FC83478F
:10039000450081CF4146A6855D0597F00000E780C6
:1003A000C09E814755D9AD4745BF1309650123025A
:1003B000E500CA85268597100000E780606231C19C
:1003C000A547E38B0AF82302040079B705C18357D8
:1003D0000500E39247F94146A685190597F000000C
:1003E000E780A09A81472DD99947BDB74E859700E0
:1003F0000000E78080F02A84954739DD1309550015
:100400004DBF4146A6852310440123113401130535
:10041000190097F00000E780A099228597800000DE
:10042000E780A0EA81470DBF1723FFFFE70263CDF6
:1004300079717C003ECCB7070A003ECE7C003ED0EE
:1004400083C79500B2842E8493F7F707A384F50041
:100450001306A1002A892C00268597000000E7805A
:10046000A0E5A16528088D0597A0FFFFE780A0F70C
:1004700090408355A10003558100854697000000F8
:10048000E78000ECAA84AA85280897C0FFFFE780D0
:1004900040DA0356A1008355810028089700000028
:1004A000E780C0C1300801478146A2854A8597A0F0
:1004B000FFFFE780A018854748103ED42302910231
:1004C00002D697D0FFFFE78060BD45611723FFFF8D
:1004D000670063C51723FFFFE702A3C279717C00A1
:1004E0003ECCB7070A003ECE7C003ED083C79500C5
:1004F000B2842E8493F7F707A384F5001306A100B6
:100500002A892C00268597000000E780E0DAA165A3
:1005100028088D0597A0FFFFE780E0EC9040835509
:10052000A10003558100814697000000E78040E16B
:10053000AA84AA85280897C0FFFFE78080CF0356CA
:10054000A10083558100280897000000E78000B7CC
:10055000300801478146A2854A8597A0FFFFE780C2
:10056000E00D48102302910202D402D697D0FFFF7B
:10057000E780C0B245611723FFFF6700C3BA1723A6
:10058000FFFFE70203B897000000E78060DB172356
:10059000FFFF670043B99767FF1F93872799884339
:1005A00082801723FFFFE702C3B58357250041115F
:1005B000AE842A842307B10017F5FFFF13052546F3
:1005C0006C002316F10097A0FFFFE780204991C43B
:1005D000228597800000E780E0D6FD572310F400C5
:1005E000130620028145130554009720FFFFE78082
:1005F00040B441011723FFFF6700E3B21723FFFF59
:10060000E70283AE79717C003ECCB7070A003ECE8C
:100610007C003ED083C79500AA89AE8493F7F70784
:100620003285A384F5001306A1002C00970000007A
:10063000E78080C803558100114497400000E7809F
:10064000A0A915C50355A100014497B00000E7809B
:10065000A06011CD035705008357810045446318FE
:10066000F700854597000000E780E0F30144216929
:1006700093053900280897A0FFFFE780C0D6A28520
:10068000280897C0FFFFE780C0BA0356A100835532
:100690008100280897000000E78040A23008014749
:1006A0008146A6854E8597A0FFFFE78020F9481078
:1006B0004AD42302810202D697D0FFFFE780009E32
:1006C00045611723FFFF670063A51723FFFFE702BC
:1006D000A3A19767FF1F938727852A8488432E89C4
:1006E00015C5035745038357C4016311F702232639
:1006F000050223180502410597D00000E780209CE1
:100700006306090097800000E78060DB81449769F9
:10071000FF1F9389E9A1130A800297B0FFFFE780CA
:10072000C0C563C4A4049767FF1F9387A7889C4331
:1007300099C70355C40197200000E780C0BD630737
:100740000900228597800000E780C0A01306400EB4
:10075000814522859720FFFFE780A09DFD57231E3E
:10076000F4001723FFFF6700639B3385440383A7CF
:10077000C90A3E95035705008357C4016317F70064
:10078000CA8597000000E78000E2850479B7172347
:10079000FFFFE702639583C795004111AA8993F78C
:1007A000F707A384F5003285AE8497C0FFFFE7808A
:1007B00000B885676378F5042A8997400000E780D0
:1007C000A091014401CD83D70400314463882701FF
:1007D000854597000000E78080EF01444E85A286A2
:1007E0004A86A68597D0FFFFE780A09CA1679387E4
:1007F000170448003EC42302810002C697D0FFFFC1
:10080000E780C08941011723FFFF67002391172369
:10081000FFFFE702638D9757FF1F9387E7708043C1
:1008200029C4014597C00000E780002181470148A5
:10083000C1641CDC232E0403232004041769FF1F5A
:100840001309098F01449309400EFD1497B0FFFF6F
:10085000E780A0B1634FA400814517F5FFFF1305A2
:10086000857F97A0FFFFE780601F1723FFFF6700CA
:10087000E38A330534038327090B3E958357C5016B
:1008800063879700854597000000E78040E40504F2
:1008900075BF9357050113D78700A380F500931701
:1008A0000501C183A1832380E5002381F500A38195
:1008B000A50082801723FFFFE702A3842300050021
:1008C00083C71500A300F50083C725002301F500A9
:1008D00083C73500A301F50083C745002302F50057
:1008E00083C75500A302F50083C7650093059500F3
:1008F000A30305002303F5002304050032859700B8
:100900000000E78040F91723FFFF6700C38117133A
:10091000FFFFE702637D4111E9540DCD85CD93F9C9
:10092000C5FF2E842A89AA84338AA900B7EA040065
:1009300063189A020D88854411CCB7E704009C5FC8
:1009400082972AC622866C003305390197E00000A1
:10095000E7800046268541011713FFFF6700037CEF
:1009600083A78A039104829793170501C183A1830A
:10097000A38EF4FE93570501238FF4FEA183238EEB
:10098000A4FEA38FF4FE6DB763E6D5021713FFFF35
:10099000E7022377B28741113686BE8536C697E0D7
:1009A0000000E780E040B246410136851713FFFFA3
:1009B00067006377814636858280838705001387C9
:1009C000F5003D05FD8793F77708834607007D1501
:1009D0008606B58FA300F5006307B7007D17834730
:1009E00017009D83DDB782801713FFFFE702637155
:1009F000B7E7040083A7070932872A863A858297DA
:100A0000133515001713FFFF6700E37115C1814708
:100A10008DC11713FFFFE702C36E414697E0000048
:100A2000E780003985473E851713FFFF6700A36FF6
:100A300081473E8582801DCD1713FFFFE702636C5F
:100A4000414681452A849710FFFFE780806E41462A
:100A50008145130504039710FFFFE780806D014770
:100A6000C1672322040438C87CC805451713FFFF5B
:100A70006700636B0145828081473DCDB5CD17137B
:100A8000FFFFE7020368B2842E89130680058145C3
:100A90002A849710FFFFE780C069CA8524C4268591
:100AA00097000000E780C0F64146814522859710F7
:100AB000FFFFE78000683044A28522859700000090
:100AC000E780C0F293040401A28526859700000008
:100AD000E780E0EEA6851305040297000000E7809A
:100AE00000EE228597000000E78020F585473E85CF
:100AF0001713FFFF670023633E8582801713FFFFF4
:100B0000E702835E4111E9540DCD85CD93F9C5FF10
:100B10002E842A89AA84338AA900B7EA040063983C
:100B200044030D88814411CCB7E704009C5F829791
:100B30002AC622866C003305390197E00000E78061
:100B40002027268541011713FFFF6700235D83A738
:100B50008A039104829793170501C183A183A38E11
:100B6000F4FE93570501238FF4FEA183238EA4FE88
:100B7000A38FF4FE6DB765CD1713FFFFE702C356D1
:100B8000B28411E605451713FFFF670023592A8435
:100B90002E890145EDD93C487848B3E6E700E5D613
:100BA0009386F7FFB3B7F6007D17032A4404BA977C
:100BB00034C87CC863050A06C14913050A03B38912
:100BC00049412295637D3601B2862E86A68597001F
:100BD0000000E780A0DB7C40BE9464C065B7CE8691
:100BE0002E86CE8597000000E78040DAC114D294AB
:100BF0004E9923220404A2879306040103C7070029
:100C000003C607038507318FA38FE7FEE398F6FE3F
:100C10003044A285228597000000E78020DD2699D8
:100C2000C1493306994063EC9900A9DCA686A685E4
:100C30001305040397000000E78040D579BF814782
:100C4000B306F4003307F6000347070083C5060028
:100C500085072D8F2380E600E39437FF3044A2857B
:100C6000228597000000E78060D8C1145DBF014570
:100C700082800DC11713FFFFE702A348130680050A
:100C800081459710FFFFE780C04A05451713FFFF16
:100C90006700634901458280814749C5C1C5171373
:100CA000FFFFE7020346FC4141462E84AA84639974
:100CB000C70413860501A2878146C14503C7070003
:100CC00003C507038507298F3305D60003450500B3
:100CD0008506298FA38FE7FEE392B6FE3044A285F6
:100CE000268597000000E78060D0228597000000ED
:100CF000E78060F885473E851713FFFF6700A34232
:100D0000138507031D8E814522959710FFFFE7800D
:100D100040427C40130700F813060402A297238880
:100D2000E70251BF3E8582801713FFFFE702633D54
:100D30006D712E84B284AA859010280036899700A0
:100D40000000E780A0D309EDD55725A050400C4006
:100D5000280097000000E78040E27DD5FD142104C3
:100D6000F5F42C004A8597000000E78020F38147C6
:100D700061DD3E8551611713FFFF6700C33A17130A
:100D8000FFFFE702033841112EC432C62C0005468E
:100D900097000000E78080F941011713FFFF67000B
:100DA00083381713FFFFE702C33501112A842EC6CB
:100DB00002C802CA02CC02CE97E00000E780E0320F
:100DC000B2462A86A285080897000000E78060FBEB
:100DD0001375F50F05611713FFFF6700C334171371
:100DE000FFFFE70203327971B2872A842146230884
:100DF000B10013051101BE853AC436C697E0000064
:100E0000E78000FBB246930591013685970000000C
:100E1000E78060A82285141035460C089700000072
:100E2000E78020F62A84224701E921460C103A8502
:100E300097E00000E780C0F7228545611713FFFFA8
:100E40006700632E1713FFFFE702A32B7171AE84B7
:100E5000AA850A85328497000000E78060BB11C92B
:100E60000A86A685228597000000E78020B8814782
:100E700011E1C5473E854D611713FFFF6700A32AA7
:100E80001713FFFFE702E3241D712A8AB289BE848B
:100E900035468547130511012E8CB68A3A8BC28CD4
:100EA000468D2308F10097E00000E78060F0101005
:100EB0000C085285231F010097000000E780C0F84E
:100EC0002A843DEDA1476313FD089307900591E047
:100ED000E5473546E2851305110113990A012308F8
:100EE000F1001359090197E00000E78060EC135707
:100EF000890093978A00D98F90080C085285231F88
:100F0000F10097000000E78020F42A8415E9A1E4AD
:100F10009387FA0091831379F9003EC663130900A1
:100F20004149668B8144C14B854DB247639F970C05
:100F30006A868C0033855C0197E00000E78040E71B
:100F4000228525611713FFFF6700631C9307900438
:100F5000C9F0A547BDBF834701050947C14B230819
:100F6000F10083471105A58FA308F10093872400A2
:100F7000814463E1FB04014714083386E6008C08D2
:100F8000B386E400BA95DA9683C6060083C50500E9
:100F90000507AD8E2300D600E390E7FE4147639C32
:100FA000E70490080C08528597000000E780C0E92C
:100FB00025D181A0B3069B00BA871008B305F600BF
:100FC00090083E9603C50600034606008507850681
:100FD000298E2380C500E39277FF998F90080C0833
:100FE0005285BE9497000000E78000E689470147DC
:100FF00049D12A84B1B790083E96034606001408EA
:10100000BE962380C600850759BFB2478504638713
:10101000971481471808B306F70098083E9733865F
:10102000F90003470700034606008507318F238038
:10103000E600E39177FF90080C08528597000000C6
:10104000E78080E05DF53546E28513051101230850
:10105000B10197E00000E780A0D513970401418318
:10106000939784002183D98F10180C085285231F71
:10107000F10097000000E78020DD25FD8147101872
:101080003387F9003E960347070003460600B30680
:10109000FB008507318F2380E600E39277FF65A888
:1010A0001808B306F70098083E973386F9000347FF
:1010B0000700034606008507318F2380E600E3E141
:1010C00027FFCA87639E770990080C08528597000E
:1010D0000000E78060D711FD81479800B306F70054
:1010E000900818103E973E960347070003460600F7
:1010F0008507318F2380E600E39177FF3546E2854F
:10110000130511012308B10197E00000E78040CAF0
:10111000139704014183939784002183D98F10187A
:101120000C085285231FF10097000000E780C0D112
:10113000E31105EC814710183387F9003E96034709
:10114000070003460600B306FB008507318F2380A6
:10115000E600E3E227FFC109410BC1BB814785B728
:101160009408BE9683C6060018083E972300D70051
:10117000850789BF638006321713FFFFE70263F517
:1011800059712A84BE89B28B8547354613051102F1
:101190002E8B468C4289BA8A368A2300F10297E068
:1011A0000000E780E0C010180C1022852317010210
:1011B00097000000E78040C963180512A147631F2C
:1011C000FC069307900563930900E5473546DA85E9
:1011D0001305110293140A012300F102C18097E064
:1011E0000000E780E0BC93178A0013D78400D98FF2
:1011F00090080C1022852317F10297000000E78069
:10120000A0C47DE1639209049307FA00BD8891832D
:1012100091E0C144C207C183DE8C814A3EC6414D84
:10122000B24763E2FA0E6286B3854B01881097E0FD
:101230000000E78080B54DC93D557DA0930790041F
:10124000E39609F8A54759B7834701050947C14CFB
:101250002300F10283471105B3C7F900A300F1028F
:1012600093872900814963E1FC0481461810330605
:10127000D7008C083387D900B695569703470700E7
:1012800083C5050085062D8F2300E600E390D7FE79
:1012900041476390E70690080C10228597000000F4
:1012A000E78080BA35D189A0B3863A01BA87101099
:1012B000B305F60090083E9603C5060003460600F7
:1012C00085078506298E2380C500E39297FF338723
:1012D000EC4090080C102285BA9997000000E78036
:1012E000A0B68947014741D165611713FFFF670029
:1012F00003E290083E96034606001410BE96238033
:10130000C600850779B7B247850A93990A01939D6C
:101310008A0093D909016391570F85473546DA85CD
:10132000130511022300F10293D9890097E0000010
:10133000E78000A8B3ED3D0190000C102285231733
:10134000B10397000000E78020B059FD8147A689CE
:1013500063EA970626860C084A8597E00000E78036
:1013600020A581471810B306F700100898083E978B
:101370003E9603470700034606008507318F23800A
:10138000E600E3E197FE639FA90590080C10228513
:1013900097000000E78040AB21F981479810B30621
:1013A000F700900818183E973E960347070003463B
:1013B00006008507318F2380E600E391A7FF4109EE
:1013C000C10CB9BD18089000B306F7003E963387EC
:1013D000FC0003470700034606008507318F238082
:1013E000E600B5B798084E97034707001C10CE9744
:1013F0002380E700850941BF85473546DA85130517
:1014000011022300F10293D9890097E00000E780E0
:10141000209AB3ED3D0190000C1022852317B103F3
:1014200097000000E78040A2E31005EC8147180810
:101430009000B306F7003E963387FC000347070091
:10144000034606008507318F2380E600E391A7FF5E
:1014500041460C084A8597E00000E7806095814787
:101460001810B306F700100898083E973E960347F9
:101470000700034606008507318F2380E600E391CD
:10148000A7FF90080C10228597000000E780C09B02
:101490001DD599BD7D5582801713FFFFE70263C6F6
:1014A00001112A842E8593055100328902C002C29F
:1014B00002C402C69304740097F0FFFFE780A03DCA
:1014C0001D46A6851305910097E00000E780408E39
:1014D00010088A854A8597000000E780E09619ED9C
:1014E00093071400180883C6070003460700850702
:1014F0000507B18EA38FD7FEE397F4FE056117139E
:10150000FFFF670043C21713FFFFE702E3BD2E840E
:101510008C414111AA89838715003289914463D394
:101520000700A1449757FF1F938707F79C43A1C764
:10153000C1CA8D472310F10083C725004A852301C6
:10154000F10083C73500A301F10083C745002302E2
:10155000F10083C75500A302F10083C7650093051E
:101560009100A30301002303F1002304010097F07D
:10157000FFFFE78040320C404A860A8597F0FFFF64
:10158000E78080330328040083564400A6881D08A2
:1015900081470147E51642868A854E8597000000FF
:1015A000E780408E2A8919E5A685228597B0FFFF3E
:1015B000E780E0C14A8541011713FFFF670003B6CA
:1015C0004A860A8597F0FFFFE780002F6DB7171353
:1015D000FFFFE70263B12E848C414111AA89838702
:1015E00015003289914463D30700A1449757FF1F28
:1015F000938787EA9C43A1C7C1C68D472310F1009A
:1016000083C725004A852301F10083C73500A30164
:10161000F10083C745002302F10083C75500A302F0
:10162000F10083C7650093059100A3030100230324
:10163000F1002304010097F0FFFFE780C0250C4074
:101640004A860A8597F0FFFFE7800027835644000B
:10165000032804008A85858EC2061D08C1822312D4
:10166000D400A68881470147E51642864E8597003B
:101670000000E78060B041011713FFFF670003AA75
:101680004A860A8597F0FFFFE78000234DBF1713B6
:10169000FFFFE70203A7B335B000011185052A89D2
:1016A0001315F601336515012308B10093051101E7
:1016B00036843AC632C03EC442C297F0FFFFE7808C
:1016C000801DA2471248425593D68700230BF10094
:1016D0009305910193578800A30AD100A30BF10051
:1016E000230C010197F0FFFFE780E01A3247024622
:1016F00003280400B337E000835644009207914466
:1017000011C2A1444A85A68842860C0897F0FFFFC3
:10171000E78040772A8919E5A685228597B0FFFFE3
:10172000E780E0AA4A8505611713FFFF6700A39FC2
:101730001713FFFFE702439B01113EC68647B335EF
:10174000B0008505AA891315F6015D8D2308B10047
:101750009305110136843A89B28442C446C297F097
:10176000FFFFE780401322489248164593578800B0
:10177000A30AF1009305910193D78800230B01017F
:10178000A30BF100230C110197F0FFFFE780A010DD
:101790003247104083564400B337E00092070328D5
:1017A0000900914891C0A1480C084E85970000009F
:1017B000E780809CAA8401E9835544004A8597B05C
:1017C000FFFFE780C0A0268505611713FFFF6700B4
:1017D000E394AA959307F00F17170100130707EB7F
:1017E0006317B50013C5F7FF1375F50F8280050564
:1017F0008346F5FFB58FBA9783C70700D5B7035760
:10180000450014419307F00F17160100130606E870
:10181000369742074183139506014181631BE5001A
:10182000AD8FB29703C50700130515F313351500E7
:101830008280850603C5F6FFA98FB29783C707008C
:10184000D9BF1713FFFFE702C38BB28736842E86FA
:10185000BA86AA853E85BA8497F0FFFFE78060527A
:10186000634F0500228597E00000E78000882A8604
:10187000A686A285268597F0FFFFE7808050171384
:10188000FFFF6700438A1713FFFFE702E3855D71DF
:101890002A8BAE8A171501001305C5DC2C00B28413
:1018A000368ABA893E8997F0FFFFE780C04F2A84C5
:1018B0005DE134104146DA85280097F0FFFFE780AC
:1018C000404C2A8449E98547A303F100A6C2930747
:1018D00071002408BEC4A68685470D462C18281022
:1018E00002DC02DED6C0BEC697F0FFFFE7800044F0
:1018F0002A8435E183477102A6860D4693F7F707E0
:101900002300FA00C1473EDE2C188947281026DC48
:10191000A303F10097F0FFFFE78040412A8405ED23
:101920004146A6854E8597D00000E78060488D47E8
:10193000A6860D462C182810A303F10097F0FFFF90
:10194000E780C03E2A8401E94146A6854A8597D0B2
:101950000000E780E045228561611703FFFF670013
:10196000E37B1703FFFFE702C37997F70000938734
:10197000E712984383C7470079712A89AE84171507
:1019800001001305A5CE0C083AC42306F10097F018
:10199000FFFFE78040412A8405ED14104146CA85C7
:1019A000080897F0FFFFE780C03D2A8415E114087E
:1019B00015462C00081097F0FFFFE780803C2A8432
:1019C00001E921462C08268597D00000E780403E9B
:1019D000228545611703FFFF6700E3741703FFFFCC
:1019E000E702237297F700009387470B9C477971B2
:1019F000AA842E84171501001305C5C70C083EC61E
:101A000097F0FFFFE780203A0DE914104146A685C4
:101A1000080897F0FFFFE780C03605E1140811467B
:101A20006C00081097F0FFFFE780A03519E58347A9
:101A3000F10193F7F7032300F40045611703FFFF5B
:101A40006700636E1703FFFFE702A36B3688A148A8
:101A500081470147E54697F0FFFFE780A042170363
:101A6000FFFF6700436C1703FFFFE70283693688B7
:101A7000A14881470147E54697F0FFFFE780C06F27
:101A80001703FFFF6700236A1703FFFFE70263677F
:101A900001112A842E850C0832C697F0FFFFE780DB
:101AA000803009ED324797160100938626BB100857
:101AB000C145228597000000E780E0D80561170343
:101AC000FFFF670043661703FFFFE70283634111CF
:101AD000C1472EC032C48A8509463EC23EC697F031
:101AE000FFFFE780A02441011703FFFF6700A36306
:101AF0001703FFFFE702E3604111AE8613061009EA
:101B0000AA850A8502C002C202C402C697F0FFFF7E
:101B1000E780202741011703FFFF6700C360170319
:101B2000FFFFE702035E328797160100938606B532
:101B30002E869305000297000000E780C0D01703AF
:101B4000FFFF6700435E1703FFFFE702835B7971C6
:101B5000C1472ACC2ED032D42C080D4628003ECEC8
:101B60003ED23ED602C402C602C802CA97F0FFFFA8
:101B7000E780C01B45611703FFFF6700C35A1703C7
:101B8000FFFFE70203580111AA842E8417150100F4
:101B9000130545AF8A8597F0FFFFE780C02015E564
:101BA00014084146A6850A8597F0FFFFE780601D6F
:101BB00009ED8347E1010347F101A207D98FCA0765
:101BC000C9836177D98F2310F40005611703FFFFE4
:101BD0006700635515CD1703FFFFE7028352974750
:101BE000FF1F9387273990439745FF1F9385C5387B
:101BF0001745FF1F1305053497D00000E78000C587
:101C00001745FF1F130505331703FFFF6700A35197
:101C10001745FF1F1305053282808DCD1703FFFF87
:101C2000E702234E9747FF1F9387C7349443011160
:101C30002E840A869745FF1F9385053497D00000B0
:101C4000E78040C60A850294014505611703FFFF3E
:101C50006700634D7D5582801703FFFFE702634AEB
:101C600097D00000E78080D19747FF1F23A4A730BB
:101C700017F5FFFF1305E5C997B00000E780C074B2
:101C80001703FFFF6700234A1747FF1F1307C730DB
:101C90009317150008433E95FD572310F5008280E9
:101CA0001703FFFFE702E3452A84084009E517030D
:101CB000FFFF670043471C4158401CC06313E50009
:101CC0005CC08347550023200500F99BA302F50063
:101CD00097A0FFFFE780207CC9BF1703FFFFE70243
:101CE000A3409747FF1F9387272D98432A8411CB42
:101CF0008347350093F7070289C7035505008945D7
:101D000002971305440197B00000E780403B8355DC
:101D100004000355E40097300000E780A00C485809
:101D200019C597A0FFFFE7800077232A0402130557
:101D3000840397000000E780E0F68144B149979062
:101D4000FFFFE780C06D63CBA402834734002320EC
:101D5000040493F727FCA301F40000489790FFFFC9
:101D6000E780E06C13161500814522859700FFFF80
:101D7000E780203C1703FFFF6700433AB387340333
:101D80000329040385043E994A8597000000E780F3
:101D900060F12304090065B78347350093F7070214
:101DA00099E3014582808357E500E39CB7FEC16754
:101DB000FD176316F60005458280054599A81703AF
:101DC000FFFFE702033493170601C187B2842A8418
:101DD00001496359F002835705009DCB01456367B4
:101DE000F600034584003E953325A6001375F50FD4
:101DF0000DA01C4813171900BA9783D70700E38E6C
:101E000097FA05099790FFFFE7806062E343A9FE18
:101E100001451703FFFF670003311703FFFFE702C8
:101E2000A32CAE89AA849790FFFFE78000562A84EE
:101E300097D0FFFFE780A02EAA86014713068401F2
:101E400097050000938585E41745FF1F13050515C9
:101E50009790FFFFE780801C2A8925C98C441304D2
:101E6000C50022859E0593F5050897A0FFFFE78032
:101E7000403CCC4083877400E18163DD070493E537
:101E80000508228597A0FFFFE780A03A0D469385BD
:101E90004400228597A0FFFFE780C03683D5040069
:101EA000228597A0FFFFE780E03D83D524002285AF
:101EB00097A0FFFFE780003D03D6490083A50900F6
:101EC000228597A0FFFFE780E0334A851703FFFFD5
:101ED0006700C32493F5F5076DB71703FFFFE7020B
:101EE000432201112A84328532C697A0FFFFE78082
:101EF000E0279780FFFFE78060348357040017478F
:101F0000FF1F1307E7223246231BF100930700F857
:101F1000A30DF1001C471843231AA1008983858B68
:101F2000B307F740B28548083ECE231C0100230DBD
:101F3000010097000000E78080EE05611703FFFFB6
:101F40006700631E1703FFFFE702031A0041014504
:101F50003DC49304C40026853289AE8997A0FFFF53
:101F6000E780C02495452A8A2685035B040197A053
:101F7000FFFFE7802021268597A0FFFFE780603ED6
:101F80008D45AA8A268597A0FFFFE780A01F26859A
:101F900097A0FFFFE780E03C5C48420A135A0A0121
:101FA000D2975CC423186401814763983A014605BF
:101FB0004D81330625419337160013F5F70F1703AC
:101FC000FFFF6700A3151703FFFFE70203118969ED
:101FD0002A8BAE8B328AB68A81440144314CFD197A
:101FE0009790FFFFE780A04363CDA4009790FFFF89
:101FF000E780E045018D33B5AA001703FFFF6700B6
:1020000043113389840383270B003E9963170A0029
:102010008347890085043E94E1B703560A00DE85B4
:102020004A8533F6C90097000000E780E0F16DD1E2
:102030000545E1B71703FFFFE702A30C01112A844E
:102040007C000355E5003ECAB70707003ECC7C0084
:102050003ECE97200000E78020082A898545480861
:1020600097A0FFFFE78020399945480897A0FFFF18
:10207000E780E015AA844A8597200000E780A00841
:102080002380A4009747FF1F9387870A9C434166DC
:10209000130606F09396870113D78701558F93D6C1
:1020A0008700F18E558FA207B706FF00F58FD98FF5
:1020B00011462C00138514003EC497D00000E78021
:1020C00020CF5008A3820400894522859700000094
:1020D000E780E0E019C9AA851305840397A0FFFFF4
:1020E000E780E0313C4085073CC005611703FFFFF6
:1020F000670063031703FFFFE702A3009790FFFF4A
:10210000E780E0342A8405049790FFFFE7802033BE
:102110003305A402F14791453305F50297200000ED
:10212000E78020BA11E565551703FFFF6700A3FF9D
:102130009747FF1F23AAA7E69790FFFFE78020316C
:102140002A8405049790FFFFE780602F3305A402DF
:102150008945060597200000E780A0B669D5974716
:10216000FF1F23ABA7E29790FFFFE780402E2A8452
:1021700005049790FFFFE780802C3304A402974763
:10218000FF1F239D87E09790FFFFE780402C2A8464
:102190009790FFFFE780A02A930714003385A702DA
:1021A0009747FF1F239DA7DE9707010093874711DD
:1021B0001747FF1F2328F7DE0145BDB71703FFFFB1
:1021C000E70283F2AA842E8901449749FF1F93896D
:1021D00029F6130A80069790FFFFE78040266347A1
:1021E000A40001451703FFFF670043F333054403D1
:1021F00083A709024A86A6853E9597000000E780DE
:10220000E0B919E10504C1BF0545E9BF1703FFFFA8
:10221000E702A3ECAA8A2E8BB28B368C3A8A8144D1
:1022200001448149974CFF1F938C8CF0130D80065D
:102230009790FFFFE780A02063C9A40011E08549C3
:102240004E851703FFFF6700C3EC3389A40383A700
:102250000C025E86D6853E994A8597000000E7808D
:10226000E0B31DC19790FFFFE780601E0544636DDA
:102270004501D2866286DA851305090397000000BE
:10228000E780A0D411C1854985045DB71703FFFF1E
:10229000E70283E5C16441112A8901449749FF1F80
:1022A000938909E9130A8006FD1436C632C42EC28A
:1022B0009790FFFFE780A01892452246B2466348F8
:1022C000A400014541011703FFFF670023E5330523
:1022D000440383A709023E9509C683473500C18B95
:1022E0009DC791C68347350093F707028DC36306E8
:1022F00099008357E500639C27010357050001CB34
:1023000063E7E50083478500BA97E3CDF5FA050456
:1023100069BF1703FFFFE70223DDC1642A89014477
:102320009749FF1F9389C9E0130A8006FD1497900F
:10233000FFFFE780C0106346A4001703FFFF67009C
:10234000E3DD3305440383A709023E958357E50087
:10235000638A970063049900639627019700000041
:10236000E780E0970504E1B71703FFFFE70263D6B4
:1023700089692A8AAE8A328BB68B8144174CFF1F3B
:10238000130C0CDB930C8006314DFD199790FFFF69
:10239000E780E00A63C6A4001703FFFF670023D7A6
:1023A0003389940383270C028355CA015A863E99C8
:1023B0004A8597000000E780609E31C1814D15A0DD
:1023C0003384AD038327090303D60B00D68533F688
:1023D000C9003E94228597000000E780E0B609E935
:1023E000850D9790FFFFE7808003E3CBADFC01A84C
:1023F000228597000000E780E08A2304040085041A
:1024000071B71703FFFFE70243CD4169AA8A014A6A
:10241000174BFF1F130BCBD17D19C14B054C979068
:10242000FFFFE780C0016346AA001703FFFF6700B4
:1024300043CE93098006B3073A0383290B02BE9962
:1024400083D7E900638E270163842A01639A5701C9
:1024500003A4890301E84E8597000000E780C0BD12
:10246000050A75BF83570401639977099304C40073
:10247000268597A0FFFFE78060D385452A8D2685B6
:10248000835C040197A0FFFFE780C0CF268597A05B
:10249000FFFFE780A0E762056185635905048D456C
:1024A000268597A0FFFFE780E0CD8945268597A088
:1024B000FFFFE78020CD8945268597A0FFFFE780B5
:1024C00060CC8545268597A0FFFFE780E0CC834759
:1024D0000500094793F7F707639AE70099452685B2
:1024E00097A0FFFFE78040CBA30285014848337DDA
:1024F0002D01231894016A9548C40040A1BF170319
:10250000FFFFE70203C037E404008327041D82971E
:102510009747FF1F83C7C7AE1715FF1F1305C502D7
:10252000A300F5008327441C82978327841C8146DF
:102530001306F00F8145014582971703FFFF6700DF
:1025400083BE1747FF1F1307A79B18439745FF1F1D
:1025500083C505AB9747FF1F938707A9834687036A
:10256000034697036397D5009747FF1F238AC7A8A1
:10257000828083C587010347A7036317B600974787
:10258000FF1F238FE7A6828003C687016317C7005A
:102590009747FF1F2386D7A6828083C6870113072C
:1025A00050026319D700930760021747FF1F2309E2
:1025B000F7A4828083C68701130660026315D600E4
:1025C00093077002DDB783C7870155BF9747FF1F89
:1025D000938787A1D44B0947638DE6081703FFFF54
:1025E000E70223B21749FF1F1309499D3E84834721
:1025F0000900918B9DCFB7E4040083A7041D829747
:1026000083A7441C1745FF1F1305C59B829783A70B
:10261000841C81461746FF1F0346C69C8145014521
:10262000829721C583470900ED9B1747FF1F2307AA
:10263000F7988347040093F7F70F85CB9147174727
:10264000FF1F232DF79A97000000E78080EB97008B
:102650000000E78040EFB7E70400BC4F41469145DA
:102660001745FF1F0345C59882971703FFFF6700B3
:1026700083AB82801703FFFFE702A3A88D474111B8
:102680006306F504C5476308F50285476310F50244
:102690009747FF1F2388A796B7E70400BC4B930515
:1026A00000101745FF1F0345A594829741011703AA
:1026B000FFFF670043A785471747FF1F2304F794D1
:1026C000B7E70400BC4B93050020E1BF9747FF1F0D
:1026D00093878791D44B1147638DE600B7E70400D9
:1026E00083A7071D8297B7E70400BC4B930500043E
:1026F0004DBF05491747FF1F2322279183C70700B6
:1027000032C62E8493F7F70FD5D3B7E4040083A71E
:10271000041D7D141374F40F8297E37689FCB2458F
:10272000994703C61500E3F0C7FCFC4409061745AA
:10273000FF1F1305658D8297BC4893050008174558
:10274000FF1F0345E58A829779BF1703FFFFE70262
:10275000439B1747FF1F130727894047184B1C400F
:102760009746FF1F23A8F6886316E4001747FF1F4C
:102770002324F788130584FE9790FFFFE78000AAC3
:10278000035564FF9780FFFFE780807297A0FFFFEB
:10279000E78060D01703FFFF6700E3981703FFFF90
:1027A000E70223969747FF1F93870784D84BDC47A0
:1027B00089C797000000E78080F985471747FF1F0A
:1027C000232EF7829737FF1F938787739C439305C8
:1027D00000021745FF1F0345A58183C787031747DD
:1027E000FF1F230FF780B7E70400BC4B8297170346
:1027F000FFFF670043939737FF1F23A9A77E8280BF
:102800001703FFFFE702438E37E404007C4CA14529
:102810001735FF1F0345C57D82977C48A1451735B5
:10282000FF1F0345E57C9734FF1F9384E47B829769
:10283000DC4489EB97000000E78080D91703FFFF95
:102840006700C38D03D567FF9780FFFFE780406671
:10285000AA896DD1D84891476310F7027C4C914505
:102860001735FF1F0345C57882977C48914517357A
:10287000FF1F0345E577829703A9490103D40901A6
:102880008947B7E904001737FF1F2329F77683A785
:10289000091D21044204829783C784011715FF1F75
:1028A000130585CA61191717FF1FA30FF7C883A760
:1028B000491C418082979737FF1F2385077483A7A0
:1028C000C91C814609469375F40F4A85829711E920
:1028D0009747FF1F83C7478389C79700FF1FE7807C
:1028E000A033B7E70400BC4F2146A1451735FF1FB1
:1028F00003450570829799B71703FFFFE7026380CE
:1029000093F7052001112E8481CF97000000E78006
:1029100020E91345042005611703FFFF6700A3802A
:1029200093F70510A9CF9734FF1F9384E46BDC481D
:1029300097000000E78020C11737FF1F1307475C8F
:10294000184383C78401034787036318F700DC44F7
:1029500089C797000000E78080DF85471737FF1F92
:10296000232EF768B7E70400BC4B93050002173528
:10297000FF1F0345E56782971345041069BF93F76E
:102980000508BDC79737FF1F83C71768E9171946A2
:102990009735FF1F938565671305D10093F4F70FF3
:1029A0001739FF1F0349496697C00000E780404080
:1029B00093970401C1831737FF1F13076765231D12
:1029C000F100231CF1009737FF1F9387E7613ACE90
:1029D0003ACAD8432306010009CBDC439315890189
:1029E00054080D46E185680082971345040825B711
:1029F00093F72500A5C39737FF1F9387E75ED84B52
:102A000089476306F7029737FF1F83C7275B13F7D2
:102A1000270011EF918B99CFB7E70400BC4F130645
:102A2000000A89451735FF1F0345855C82971345CA
:102A30002400D5B59737FF1F9387874C9C4383C7E6
:102A400087031737FF1F230DF75A97000000E78011
:102A500060DBF1BF93F7050281CB97000000E780B0
:102A600060DA1345040245BD93F7850081CB9700DA
:102A70000000E780E0D21345840071BD93F7150094
:102A800081CB97000000E780A0B41345140061B526
:102A900093F7450081CB97000000E78060B31345B2
:102AA000440095BD93F7050495C39737FF1F83C76F
:102AB000A75391CB97000000E780A0A49147173758
:102AC000FF1F232DF75213450404B1B593F70501F9
:102AD0000145E38207E49737FF1F9387E750D84B00
:102AE00091476310F7049737FF1F9387274D9C4347
:102AF00013D727008583D98F858B91E7B7E704002B
:102B000083A7071D8297B7E70400FC4F914517354F
:102B1000FF1F0345E54D829785471737FF1F232F7A
:102B2000F74C13450401C5BB9737FF1F238EA75CE5
:102B3000828017F3FEFFE702C35C9737FF1F23ABCA
:102B4000074A9737FF1F23A9074A85471734FF1FF6
:102B50001304043B1737FF1F2322F74A1C4083C787
:102B600087031737FF1F230DF7489790FFFFE78074
:102B7000409329C59717FF1F23ACA79C1C4017053E
:102B800000001305A5D783C787031737FF1F230945
:102B9000F7461717FF1FA309F79A9737FF1FA3855B
:102BA0000744B7E7040083A7070882979737FF1FFA
:102BB0002380A74417F3FEFF6700E356B7C7898E4B
:102BC000938767ED1717FF1F2324F79845BF173723
:102BD000FF1F03476741795555E79737FF1F9387D5
:102BE000A74003C7170005079736FF1FA38EE63ED1
:102BF00003C717008D463377D7029736FF1FA3858B
